:100000000C94A5010C941F020C941F020C941F0267
:100010000C941F020C941F180C949B160C941F0236
:100020000C941F020C941F020C941F020C941F02CC
:100030000C941F020C941F020C941F020C94980C39
:100040000C941F020C941F020C9407170C946B174E
:100050000C941F020C941F020C941F020C941F029C
:100060000C941F020C941F020C941F020C941F028C
:100070000C941F020C941F020C94C4110C943611A2
:100080000C941F020C941F020C941F02D96DE36D97
:10009000EA6DF06DFA6D086ED66DD66DD66DD66DC3
:1000A000176E1D6E206E326E356E406ED66D436ECD
:1000B000496E4C6E526E556E5B6E5E6E666E0A00D9
:1000C00072252E32787C000A0077252E32782000A7
:1000D0000A007C0072252E327820005445524D498A
:1000E0004E414C204552524F523A2063616E6E6F22
:1000F0007420616C6C6F63206D656D6F72790A009E
:1001000025630021214C494E4520544F4F204C4F30
:100110004E4721210A0025632025630025733A20DC
:10012000636F6D6D616E64206E6F7420666F756EA7
:10013000640A000A002563202563000A20756172A5
:10014000742072656164206572723A2025640A0029
:1001500042544E5F5445524D494E414C3A2045520F
:10016000524F523A207768696C6520726561646904
:100170006E672066726F6D20756172740A00666129
:10018000696C65642120636D6473206275666665C1
:10019000722066756C6C210A0072656769737465FC
:1001A00072696E6720636D643A2573200066616929
:1001B0006C656421206E616D6520746F6F206C6FBB
:1001C0006E67210A007265676973746572696E678C
:1001D00020636D643A257320000A0009000A000AB2
:1001E000004E75743A204865617020417661696CF3
:1001F00061626C65203D2025752062797465732EDF
:100200000A006E75743A206572726F723A207573C7
:100210006167653A0A206E7574207468726561645E
:10022000730A206E75742074696D6572730A206E8E
:10023000757420686561700A00257520627974659F
:100240007320667265650A00257520636F756E748C
:1002500065642C20627574202575207265706F723C
:100260007465640A0025303478202535640A002836
:1002700025303458290A002530356C580025303493
:100280005825366C7525366C7520004164647220E3
:100290005469636B7320204C6566742043616C6CF9
:1002A0006261636B0A004E75744576656E745469BD
:1002B0006D656F7574004E7574546872656164572E
:1002C000616B65000A486E646C204E616D6520208C
:1002D0002020205072696F205374612051554520B1
:1002E0002054696D722053746B5020467265654DC1
:1002F000656D0A00202530345800253034582025FB
:100300002D3873202534752025732025303458204E
:100310002530345820253034582025357520257354
:10032000002530345820252D38732025347520259C
:100330007320253034582025303458202530345847
:10034000202535752025730A000085B7806885BF94
:10035000ECE6F0E0808180688083BF9ABE9AC798FF
:10036000C69880EC85BFAF9AA79AAE9AA69A81EEFE
:100370008093008380E48093018385B78F7785BF66
:1003800080E090E09D9B05C0019641F09D9BF8CFD9
:10039000FBCF019619F09D99F3CFFBCF85B780680D
:1003A00085BFAF98A798AE98A69887E089B9809343
:1003B000990011241FBECFEFD0E1DEBFCDBF14E105
:1003C000A0E0B1E0E2E8FFEF00E00BBF02C0079061
:1003D0000D92AA38B107D9F716E1AAE8B4E101C035
:1003E0001D92A936B107E1F78FEF9FEF9EBF8DBF3A
:1003F00029E636E1C901809590958158914038F001
:100400006FEF7EEF621B730BC9010E9435090E94DA
:100410006F09892B41F065E273E08DE096E10E945F
:10042000C87E0E94560920E831E040E050E064EDCB
:1004300073E08EE293E00E94340B0C9400000C9465
:1004400000006F927F928F929F92AF92BF92CF9255
:10045000DF92EF92FF920F931F93CF93DF93CDB76D
:10046000DEB7CC54D0400FB6F894DEBF0FBECDBF80
:1004700080E09BE4A0E0B0E089839A83AB83BC83F7
:100480000E940C4A81E00E94364B0FE313E040E0EB
:1004900060E070E0C8010E9419044091510450913D
:1004A000520460E071E0C80102960E94A518809194
:1004B0005104909152040E944518AE014F5F5F4F66
:1004C00061E071E00E94A9190E94664D83E091E00D
:1004D0009F938F930E9410198DE391E00E94301931
:1004E00085E691E09F938F9383E791E09F938F93AD
:1004F0000E94101981E991E09F938F9388EC91E01D
:100500009F938F930E9410190E94E00B7B018C0136
:100510000E94E90B5B016C01C801B70120E432E4E1
:100520004FE050E00E942A7F39014A01BF92AF920A
:10053000CA01B90120E432E44FE050E00E94EC7EB1
:10054000E61AF70A080B190BC801B70124E630E0D8
:1005500040E050E00E942A7F3F932F937F926F925A
:100560008EEC91E09F938F930E94101987EF91E09A
:100570009F938F930E9410198FE292E00E9430198E
:100580000E94254A8BEB93E00E949F319093F915CE
:100590008093F8154DE050E060E070E00E940E2C72
:1005A000BE016B5F7F4F8091F8159091F9150E9405
:1005B000E42D8E819927982F88272D813327822B30
:1005C000932B9F938F9388859927982F88272F8126
:1005D0003327822B932B9F938F938A859927982F6C
:1005E000882729853327822B932B9F938F938CE425
:1005F00092E09F938F930E941019AE01455F5F4F69
:1006000060E070E08091F8159091F9150E947228D1
:1006100089899A899F938F938F8598899F938F93C8
:100620008E8599279F938F938C859D859F938F931C
:100630008B8599279F938F9383E792E09F938F9366
:100640000E9410198DB79EB788960FB6F8949EBF7A
:100650000FBE8DBFAE014D5E5F4F60E070E08091D8
:10066000F8159091F9150E94F0278A8D99279F938C
:100670008F93898D99279F938F93888D99279F9327
:100680008F938F8999279F938F938E8999279F9313
:100690008F938D8999279F938F938C8999279F9307
:1006A0008F938B8999279F938F9386E992E09F93ED
:1006B0008F930E9410198E01015D1F4F2EE1A8013A
:1006C00060E070E08091F8159091F9150E949E22EB
:1006D0001F930F938DEC92E09F938F930E941019BC
:1006E0004FED52E060E070E08091F8159091F915BF
:1006F0000E9484258BEE92E00E9430198D8199270B
:100700009F938F938E8199279F938F9380E193E09E
:100710009F938F938E01055E1F4F1F930F930E942F
:100720004719B80180915104909152040E949E5340
:100730008091F8159091F9150E9432580E942B581B
:100740000E94D2650E942C620E941E638091510417
:10075000909152040E947B6360E070E081E00E940F
:1007600017588DB79EB74E960FB6F8949EBF0FBE22
:100770008DBF80E090E0C45BDF4F0FB6F894DEBF22
:100780000FBECDBFDF91CF911F910F91FF90EF90E2
:10079000DF90CF90BF90AF909F908F907F906F90A1
:1007A00008958093380308950E94DA0420E033E02E
:1007B00040E050E061E272E083E393E00E94340B9A
:1007C0008EEF0E94B9070E943D080E948407209185
:1007D00038032F3FC1F395B785B7837E822B85BF42
:1007E00085B7806285BF889585B78F7D85BF85B7C2
:1007F000837E9C71892B85BFE6CF0F931F93CF9388
:10080000DF938C01C0918B14D0918C140AC0B80175
:10081000CE0102960E94BE7E892B29F00990D881D4
:10082000C02D2097A1F7CE01DF91CF911F910F919D
:100830000895CF93DF93EC01892B11F161157105B8
:1008400011F07D876C8741114E87CE0102960E9480
:10085000FD03892BA9F4EB89FC89309721F0CE01A7
:100860000995892B69F480918B1490918C1499834C
:100870008883D0938C14C0938B1480E090E002C0E6
:100880008FEF9FEFDF91CF9108958091FC159091AC
:10089000FD15A091FE15B091FF150196A11DB11D8A
:1008A0008093FC159093FD15A093FE15B093FF1552
:1008B0000895CF93DF93EC011B821A82E091FA1521
:1008C000F091FB151AC0288539854A855B8580859E
:1008D0009185A285B385281739074A075B0780F001
:1008E000281B390B4A0B5B0B288739874A875B87A4
:1008F000FB83EA830190F081E02D309721F718C047
:10090000821B930BA40BB50B80879187A287B387BB
:10091000F983E883D383C283EA81FB81309719F09E
:10092000D183C08308C0D093FB15C093FA1503C0D0
:1009300019821882F1CFDF91CF9108950FB6F89404
:100940000F926091FC157091FD158091FE159091AC
:10095000FF150F900FBE0895CF93DF93EC01EA814E
:10096000FB8188819981309719F09183808304C03D
:100970009093FB158093FA15E881F9813097A1F0E7
:100980008A819B819383828380859185A285B385AB
:10099000288539854A855B85820F931FA41FB51F63
:1009A00080879187A287B387CE010E94C808DF9114
:1009B000CF91089585E494E00E94EE0B87B78260A2
:1009C00087BF0895EF92FF920F931F93CF93DF930A
:1009D0000FB6F8940F922091FC153091FD154091BF
:1009E000FE155091FF150F900FBE80918D149091C0
:1009F0008E14A0918F14B091901479018A01E81A95
:100A0000F90A0A0B1B0B20938D1430938E1440931C
:100A10008F14509390144FC088859985AA85BB8503
:100A2000E816F9060A071B07A0F48E199F09A00B08
:100A3000B10B88879987AA87BB870097A105B10565
:100A400021F0EE24FF24870136C0EE24FF24870125
:100A500008C0E81AF90A0A0B1B0B188619861A86B1
:100A60001B86EC85FD85309721F06E857F85CE0154
:100A700009958C819D81AE81BF8188879987AA87DE
:100A8000BB870097A105B10521F4CE010E94AC04FB
:100A900012C0E091FA15F091FB150190F081E02D64
:100AA000F093FB15E093FA15309711F01382128240
:100AB000CE010E945904C091FA15D091FB152097E0
:100AC00031F0E114F1040105110509F0A5CFDF9122
:100AD000CF911F910F91FF90EF9008952F923F9229
:100AE0004F925F926F927F928F929F92AF92BF923E
:100AF000CF92DF92EF92FF920F931F93CF93DF93EA
:100B0000CDB7DEB724970FB6F894DEBF0FBECDBFCA
:100B10000FB6F8940F92A090FC15B090FD15C09000
:100B2000FE15D090FF150F900FBE0E94E90B9B01A0
:100B3000AC01C601B5010E942A7F39014A010E9419
:100B4000E90B1B012C010E94E90B69837A838B83DB
:100B50009C83C401B30128EE33E040E050E00E94E2
:100B6000EC7E7B018C01C401B301A20191010E94C2
:100B7000EC7EA61AB70AC80AD90AC601B50128EE42
:100B800033E040E050E00E94EC7E29813A814B81C5
:100B90005C810E942A7FE20EF31E041F151FC8010C
:100BA000B70124960FB6F894DEBF0FBECDBFDF911C
:100BB000CF911F910F91FF90EF90DF90CF90BF905A
:100BC000AF909F908F907F906F905F904F903F90ED
:100BD0002F900895EF92FF920F931F930FB6F89402
:100BE0000F92E090FC15F090FD150091FE1510910C
:100BF000FF150F900FBE0E94E90B9B01AC01C801CD
:100C0000B7010E942A7FCA01B9011F910F91FF907D
:100C1000EF900895AF92BF92CF92DF92EF92FF9242
:100C20000F93CF93DF936B017C01EA01590180E1BF
:100C300090E00E945508FC01892B81F10FB6F894D1
:100C40000F928091FC159091FD15A091FE15B09129
:100C5000FF150F900FBE8C0D9D1DAE1DBF1D209169
:100C60008D1430918E1440918F1450919014821BEA
:100C7000930BA40BB50B80879187A287B38700FFE6
:100C800005C0148215821682178204C0C482D582E0
:100C9000E682F782D587C487B786A686CF01DF9123
:100CA000CF910F91FF90EF90DF90CF90BF90AF90DA
:100CB00008950F93CF93DF930E940A06EC010097EB
:100CC00011F00E945904CE01DF91CF910F91089548
:100CD000CF92DF92EF92FF920F936A0179010E9407
:100CE0003E0C9701A6010E9459060F91FF90EF90CC
:100CF000DF90CF900895AF92BF92CF92DF92EF92A4
:100D0000FF920F93CF93DF935B016C016115710527
:100D100081059105D1F1C2E0D6E1BE0180910416B2
:100D2000909105160E941F07E0910416F091051698
:100D300083E08787E0900416F090051601E09701A4
:100D40004AE557E0C601B5010E946806F701968B97
:100D5000858B892B19F00E94F80719C0E0910416C1
:100D6000F0910516D08FC78B8091021690910316D3
:100D70009383828381E08787809104169091051682
:100D8000909303168093021602C00E943D08DF91E3
:100D9000CF910F91FF90EF90DF90CF90BF90AF90E9
:100DA0000895CF93DF93DC019B01EC01788F6F8B6B
:100DB0001D821C820FB6F8940F92EB01E881F98135
:100DC0008FEFEF3FF80749F4ED018C819D8101968B
:100DD0009D838C83E0E0F0E015C0309799F00F9090
:100DE0000FBEED019A8908C09F012E5F3F4F028020
:100DF000F381E02D309719F082899817A8F70FB684
:100E0000F8940F92ED01FB83EA83F901B183A0838B
:100E1000EA81FB81309771F084819581892B51F0B3
:100E20008C819D8124813581820F931F9D838C83CA
:100E3000158214820F900FBEDF91CF910895CF934A
:100E4000DF939C01DB010FB6F8940F92ED91FC91BA
:100E500011970F900FBE8FEFEF3FF80731F527C0C6
:100E600082819381E217F307E9F40FB6F8940F92A9
:100E700011969C938E9384819581892B59F0A28140
:100E8000B381109729F084819581ED019D838C8336
:100E9000158214820F900FBEF90113821282108EF8
:100EA000178A05C0DF011296FC013097C9F6DF9161
:100EB000CF910895FB01168A158A82E0878762E048
:100EC00076E1CF010E94D10608950F931F93CF932F
:100ED000DF938C01C0910016D09101160CC0B801AF
:100EE000CE0106960E94BE7E892B11F4CE0107C06A
:100EF0000990D881C02D209791F780E090E0DF9194
:100F0000CF911F910F910895E0910616F091071669
:100F1000309741F0838994890E94C808109207167F
:100F2000109206160895CF93DF93C0910016D091CA
:100F300001160E9484072091041630910516E0E006
:100F4000F6E10AC088819981C217D30719F4918309
:100F5000808304C0FE01EC012097A1F78091041664
:100F6000909105169093071680930616DF91CF9106
:100F700008950F931F93182FE0910416F091051612
:100F8000028962E076E1CF010E941F07E09104161A
:100F9000F0910516128B1F3F49F062E076E18091D7
:100FA0000416909105160E94D10602C00E94930774
:100FB000E0910416F09105168091021690910316A7
:100FC000E817F90719F481E0878709C082E087876D
:100FD0000FB6F8940F920E94F50A0F900FBE802F63
:100FE00099271F910F9108958FEF0E94B9070895D7
:100FF000CF93DF93C0910016D091011620C00FB699
:10100000F8940F928C819D810F900FBE892BA1F0D7
:10101000EF89F88D0FB6F8940F928C819D8101971E
:101020009D838C830F900FBE808191818F5F9F4F36
:1010300019F0CF010E948B090990D881C02D20970B
:10104000F1F60E94E204E0910416F09105168091F9
:10105000021690910316E817F90761F08785813031
:1010600011F482E087870FB6F8940F920E94F50A78
:101070000F900FBEDF91CF910895E0910416F0918B
:10108000051682819381892B69F062E076E1CF01B8
:101090000E941F0762E076E1809104169091051688
:1010A0000E94D1060E94F80708950F931F93CF93D3
:1010B000DF9300919114109192148017910730F0F2
:1010C00080E090E060C0EF01DB012FC0AC014A5F1F
:1010D0005F4F4430510510F444E050E0E0910816B1
:1010E000F091091668E076E1C0E0D0E0A0E0B0E061
:1010F00017C0208131812417350760F02417350788
:1011000011F3209729F0888199812817390710F465
:10111000EF01DB01BF016E5F7F4F0280F381E02DA5
:10112000309739F7CE01209771F128813981CA01B2
:101130000A966A817B818217930770F4FE01E40F9F
:10114000F51F241B350B31832083738362835983FE
:101150004883ED93FC9302C06D937C93E881F98101
:101160000E1B1F0B1093921400939114EC0FFD1F94
:1011700034978FEE9EEBADEABEED80839183A28320
:10118000B383CE010296DF91CF911F910F91089505
:10119000CF93DF93DC0112976D917C911197E091D1
:1011A0000816F0910916C8E0D6E13AC04081518195
:1011B000CF01840F951F8A179B07C1F49A01260F50
:1011C000371F3183208382819381DF01A20FB31FF8
:1011D000A817B90791F58D919C911197280F391F88
:1011E00031832083ED018A819B8125C0AE17BF0723
:1011F00078F4B983A8832D913C911197CD01820F8A
:10120000931F8E179F0779F0ED01FB83EA8315C0CA
:10121000A817B90728F1EF0122960280F381E02D8B
:10122000309721F617C0240F351F11963C932E934B
:1012300082819381FD0193838283809191149091A7
:101240009214860F971F909392148093911480E0CC
:1012500090E008C0FD0113821282B983A883EDCF0C
:101260008FEF9FEFDF91CF910895FC016193719310
:10127000CF010E94C8080895809191149091921412
:1012800008950F931F93CF93DF938C010E9455080D
:10129000EC01009729F0A80160E070E00E94B47EA4
:1012A000CE01DF91CF911F910F91089583E180933B
:1012B0000A168FE480930B1683E580930C1643E1A6
:1012C00050E06AE076E180E090E00E94E70A892B36
:1012D00019F08FEF9FEF089580E090E0089543E1CB
:1012E00050E06AE076E180E090E00E94EA0A892B13
:1012F00079F480910A16833159F480910B168F345A
:1013000039F480910C16833519F480E090E008954B
:101310008FEF9FEF0895CF93DF93DC010FB6F89422
:101320000F92CD91DC9111970F900FBE8FEFCF3FB1
:10133000D80709F43AC0209771F10FB6F8940F92CC
:10134000EA81FB811196FC93EE938C819D81892B20
:1013500071F0309729F08C819D819583848305C03D
:101360008FEF9FEF11969C938E931D821C820F909E
:101370000FBE8D899E89009721F00E94AC041E8AC1
:101380001D8A82E08F8762E076E1CE010E94D1065D
:1013900081E090E00CC00FB6F8940F928FEF9FEFB2
:1013A00011969C938E930F900FBE80E090E0DF919A
:1013B000CF9108950F931F93CF93DF93EC010FB656
:1013C000F8940F92888199810F900FBE2FEF8F3F75
:1013D000920741F40FB6F8940F92198218820F9079
:1013E0000FBE02C0892B19F400E010E012C000E02B
:1013F00010E0CE010E948B09080F191F0FB6F89458
:101400000F92888199810F900FBE01978E5F9F4F39
:1014100080F3C801DF91CF911F910F9108950F9331
:101420001F930E94DA098C010E943D08C8011F9198
:101430000F9108950F931F930E948B098C010E94B6
:101440003D08C8011F910F910895CF93DF93AC0120
:10145000DB010FB6F8940F92CD91DC9111970F90AC
:101460000FBE8FEFCF3FD80799F534C08D899E8985
:101470002A813B818417950741F50FB6F8940F92A6
:1014800011963C932E938C819D81892B81F0EA816A
:10149000FB81309729F08C819D819583848305C0E1
:1014A0008FEF9FEF11969C938E931D821C820F905D
:1014B0000FBE82E08F8762E076E1CE010E94D10606
:1014C0008FEF9FEF9E8B8D8B05C0DE011296E90199
:1014D000209761F6DF91CF910895AF92BF92CF929E
:1014E000DF92EF92FF920F93CF93DF93EC015A01BB
:1014F0006B010FB6F8940F92888199810F900FBEFF
:101500008F5F9F4F51F40FB6F8940F921982188293
:101510000F900FBE0E943D0838C062E076E18091D6
:101520000416909105160E941F07BE0180910416B3
:10153000909105160E94D106E0910416F0910516CF
:1015400083E08787E0900416F0900516A114B1049B
:10155000C104D10461F001E09E0145E25AE0C601F8
:10156000B5010E946806F701968B858B03C0F701D1
:10157000168A158A0E94F807E0910416F091051664
:10158000858996898F5F9F4F19F080E090E004C0B5
:10159000168A158A8FEF9FEFDF91CF910F91FF9001
:1015A000EF90DF90CF90BF90AF900895FC010FB601
:1015B000F8940F92808191818F5F9F4F11F4118277
:1015C00010820F900FBECF010E946D0A08950E94F5
:1015D000E01508950E94001608959F918F910F9035
:1015E0000BBE0F900FBE1F9018952F923F924F92F7
:1015F0005F926F927F928F929F92AF92BF92CF92A3
:10160000DF92EF92FF920F931F93CF93DF938DB7EB
:101610009EB7E0910416F0910516918B808BE091B6
:101620000216F0910316F0930516E093041681E07C
:101630008787E0910416F0910516808991898DBF06
:101640009EBFDF91CF911F910F91FF90EF90DF90A0
:10165000CF90BF90AF909F908F907F906F905F9052
:101660004F903F902F900895CF92DF92EF92FF928C
:101670000F931F93CF93DF938C017B016A01E901E4
:10168000C90149960E945508FC01009719F480E0B1
:1016900090E075C0C80FD91F9E0127503040AE01A1
:1016A0004B515040CE01069668E0D8010D908D0157
:1016B000DC010D92CD016150C1F71E8641505040B2
:1016C000598B488B4F5F5F4FFC8BEB8B8FEE9EEB04
:1016D000ADEABEED80839183A283B3838483958337
:1016E000A683B78380879187A287B38784879587EE
:1016F000A687B78780E48A8B8F2D9927F901858388
:10170000E68280E8838312821482C1828D2D99271C
:1017100080832DEE3AE0832F9927FA01828B238B69
:10172000809100169091011699838883D0930116B9
:10173000C093001612E01F871E8A1D8A188E1F8A0A
:1017400062E076E1CE010E94D106E0910416F091AC
:101750000516309721F40FB6F8940F9260CF809160
:10176000021690910316E817F90741F017870FB694
:10177000F8940F920E94F50A0F900FBECE01DF91F0
:10178000CF911F910F91FF90EF90DF90CF90089530
:101790001F93182F60919314709194148091951455
:1017A0009091961420EA3FE040E050E00E942A7FAA
:1017B000822F932F0197F1F71A95D1F71F91089572
:1017C0006091931470919414809195149091961453
:1017D000089560E074E080E090E00895BC0187B770
:1017E0008D7F87BF80B7886080BF12BE82E083BFD5
:1017F00080B7992787709070892BD1F781E086BFD9
:101800000FB6F8940F9281E090E0A0E0B0E0B6B798
:10181000B170E9F3B6BF0894811D911DA11DB6B743
:10182000B170C9F3BB270F900FBE27E0880F991F37
:10183000AA1FBB1F2A95D1F78093931490939414F9
:10184000A0939514B093961487B78D7F87BF80B708
:10185000886080BF12BE89E083BF8FE181BF80B7FF
:10186000992787709070892BD1F782E086BF40E07E
:1018700050E089E393E00E940D71089528EE33E073
:1018800040E050E00E94EC7E3AE09695879577958F
:1018900067953A95D1F708959C01FB0187B7482FCA
:1018A00055274270507087B78D7F87BF2031310533
:1018B000D9F0213131053CF42115310581F0213079
:1018C000310551F40EC02231310571F1223131055B
:1018D000E4F020323105E1F02FEF3FEF1FC040E090
:1018E00050E082E086BF18C006B601FE05C081E068
:1018F00090E09183808302C011821082452BA1F079
:101900008081918180689183808320E030E008C0ED
:101910008EE090E09183808320E030E0452B31F031
:1019200087B7826087BF02C020E030E0C901089518
:101930001F920F920FB60F9211242F933F934F9344
:101940005F936F937F938F939F93AF93BF93EF9327
:10195000FF9389E393E00E94FF70FF91EF91BF91A5
:10196000AF919F918F917F916F915F914F913F9137
:101970002F910F900FBE0F901F901895559A89B711
:101980008F7E89BF0895CF93DF93DC01EC01EA815C
:10199000FB8120919814422F5527CA0180739070C3
:1019A000892B89F044FF04C083E18CB9206403C013
:1019B00081E18CB92F7B20939814809198148F7CAF
:1019C0008093981455C027FF02C0559851C0ED016F
:1019D0008A859B85892BB1F180919B14882339F0EE
:1019E0000C9B05C0559889B7806189BF41C0ED0146
:1019F0008A859B8501979B878A8780919914882384
:101A000011F0509A01C0509881918CB99F01FD014D
:101A1000868197812817390711F424813581ED01DA
:101A20003B832A832A853B858C859D85281739072A
:101A3000F9F4E889F989309769F08FEFEF3FF807FB
:101A4000B9F011C05598ED011B861A86E889F9890D
:101A5000309729F48FEF9FEF998B888B09C08FEF18
:101A6000EF3FF80729F0848195810196958384835F
:101A7000DF91CF910895CF93DF93DC013BB180914B
:101A80009714382B309397146CB12091981422231B
:101A900061F0633119F45598206804C0613129F46C
:101AA000559A2F77209398145DC0ED014A855B8588
:101AB000888599854817590720F038603093971426
:101AC00051C04F5F5F4F41305105A1F4ED01E889EE
:101AD000F989309729F48FEF9FEF998B888B2AC073
:101AE0008FEFEF3FF80731F184819581019695835F
:101AF000848320C0222399F0ED018E859F854817AD
:101B00005907C0F026FD16C05D9B05C083E18CB966
:101B100020642F7D01C02062209398140BC0809117
:101B20009A14882339F0FD0186859785481759074F
:101B300008F01A9AED91FC91119761931196FC931C
:101B4000EE932D913C911197ED018E819F81281785
:101B5000390729F48C819D8111969C938E93FD0108
:101B600053874287DF91CF910895529B03C089E04C
:101B700090E008958091950082FF0AC080919500C1
:101B800081FF03C088E090E0089587E090E0089529
:101B90008091950081FF03C086E090E0089585E084
:101BA00090E008958091950085FD03C080E090E06D
:101BB00008958091950084FF03C081E090E008952E
:101BC00082E090E008958091950083FF03C082E059
:101BD00090E0089581E090E00895EF92FF920F93D6
:101BE0001F9380919714682F7727CB0174E0969507
:101BF00087957A95E1F79C0144275527217030702D
:101C00004070507063FD226062FD246080919814E2
:101C1000882321F086FD426087FD48601A9B14C02E
:101C2000E12C62E0F62E012D112DE22AF32A042B7D
:101C3000152B80919A14882381F0E12C92E0F92EE3
:101C400092E0092F112D05C0E12C81E0F82E012D25
:101C5000112DE22AF32A042B152B0C9B0CC0A80192
:101C60009701386080919B14882341F0A801970167
:101C70003860426003C0A8019701346041FF4160B1
:101C800043FF446080919914882321F0CA01B9016F
:101C9000806403C0CA01B9018068589B02C080619A
:101CA00001C080621F910F91FF90EF900895EF9215
:101CB000FF920F931F937B018C01809198148823CE
:101CC000D9F00FB6F8940F9200FF02C08F7B03C0CB
:101CD00001FF03C080648093981402FF04C08091C8
:101CE00098148F7705C003FF05C080919814806811
:101CF000809398140F900FBE80919A14882321F03E
:101D000001FD1A9A00FD1A98F1FC1A9AF0FC1A9833
:101D100006FF03C081E08093991407FF02C0109270
:101D2000991404FD589A05FD5898E0FE05C080916D
:101D300097148F7E80939714E1FE05C080919714CD
:101D4000877F80939714E2FE05C0809197148B7F64
:101D5000809397140E94ED0D687F6E157F058007B4
:101D6000910719F08FEF9FEF02C080E090E01F9184
:101D70000F91FF90EF9008958091950086FF0BC022
:101D8000129B02C093E001C091E08091950080FF1A
:101D900007C0946005C0599B02C090E201C090E06A
:101DA000892F9927089580919814882329F020E29B
:101DB00030E040E050E004C020E030E040E050E09F
:101DC00080919A14882311F0216001C02E7F8091A8
:101DD0009B14882321F0CA01B90162600895CA01E9
:101DE000B9016D7F0895559A08959091981499239B
:101DF000A9F096FF13C00FB6F8940F925D9B04C034
:101E000081E18CB99F7E01C090619093981480917C
:101E100098148F79809398140F900FBE80919A1424
:101E200081111A9808950FB6F8940F925798569802
:101E300055980F900FBE8AE00E94C80B5498539893
:101E400008951F93182F0E94130F529880919500A8
:101E50008D7F80939500809195008B7F8093950076
:101E60001730A1F0183018F41630A9F405C0183056
:101E700041F0193081F404C080919500826009C05E
:101E8000529A809195008260809395008091950090
:101E90008460809395000FB6F8940F9288EB8AB90E
:101EA0000F900FBE0E94B50D811719F08FEF9FEFB5
:101EB00002C080E090E01F9108958F929F92AF92B0
:101EC000BF92CF92DF92EF92FF920F931F9389B050
:101ED000909090008091950086FF06C0B2E0AB2EF6
:101EE000B12CC12CD12C0DC0599B06C0A8E0AA2E44
:101EF000B12CC12CD12C05C0F0E1AF2EB12CC12CDE
:101F0000D12C0E94E00B7B018C01282D3327892DD9
:101F10009927982F8827282B392B442755272F5F5F
:101F20003F4F4F4F5F4FC601B5010E94EC7E9B01B2
:101F3000AC01C801B7010E942A7FCA01B9011F91F3
:101F40000F91FF90EF90DF90CF90BF90AF909F9058
:101F50008F90089540E050E060E070E08DE394E001
:101F60000E940D7140E050E060E070E083E494E096
:101F70000E940D7180919B14882359F010929B143C
:101F8000149840E050E060E070E089E494E00E9442
:101F90000D7180919A14882319F010929A14129856
:101FA00080E090E0089544E853E06BE37DE08DE34A
:101FB00094E00E940D71892B19F08FEF9FEF089527
:101FC00042E753E063EC7CE083E494E00E940D710F
:101FD000892B19F480E090E0089540E050E060E043
:101FE00070E08DE394E00E940D718FEF9FEF0895F4
:101FF000EF92FF920F931F937B018C0165FF0BC043
:1020000080919814882371F40FB6F8940F9281E4AC
:102010008093981405C00FB6F8940F9210929814FC
:102020000F900FBEE0FE06C01A9A129A81E08093CC
:102030009A1407C080919A14882319F010929A1468
:102040001298E1FE10C040E050E06EEB7CE089E4C5
:1020500094E00E940D71892BF9F41C9A149881E088
:1020600080939B140FC080919B14882359F0109289
:102070009B1440E050E060E070E089E494E00E944E
:102080000D7114980E94D30E6E157F05800791077D
:1020900019F480E090E002C08FEF9FEF1F910F9145
:1020A000FF90EF900895EF92FF920F931F937B01A3
:1020B0008C010E94130F8091950086FD11C0599BE1
:1020C00008C092E0EE0CFF1C001F111F9A95D1F77B
:1020D00007C083E0EE0CFF1C001F111F8A95D1F78B
:1020E0000E94E00BA80197010E942A7F2F5F3F4FBB
:1020F0004F4F5F4F56954795379527952150304064
:1021000029B9232F3327209390000FB6F8940F920C
:1021100088EB8AB90F900FBE80E090E01F910F917D
:10212000FF90EF9008951F93182F0E94130F812F97
:10213000992780FF13C081FF02C0129A01C0129834
:1021400082FF04C080919500816003C0809195005A
:102150008E7F8093950059985E9A0FC085FF02C0CC
:10216000599A01C05998809195008E7F809395006F
:10217000809195008F7B809395000FB6F8940F9215
:1021800088EB8AB90F900FBE0E94BC0E811719F020
:102190008FEF9FEF02C080E090E01F9108951F93A2
:1021A000182F0E94130F113071F0113018F01230F7
:1021B000C1F40DC0809195008F7E80939500809131
:1021C00095008F7D0CC080919500806103C0809147
:1021D00095008F7E8093950080919500806280931A
:1021E00095000FB6F8940F9288EB8AB90F900FBE46
:1021F0000E94D20D811719F08FEF9FEF02C080E08F
:1022000090E01F9108951F93182F0E94130F113013
:1022100021F480919500877F05C0123029F48091C8
:1022200095008860809395000FB6F8940F9288EB24
:102230008AB90F900FBE8091950083FF03C082E0A2
:1022400090E002C081E090E0181719F08FEF9FEF47
:1022500002C080E090E01F910895EAE9F0E08081FB
:102260008062808389B78F7D89BF08951F920F9206
:102270000FB60F9211242F933F938F939F93EF9359
:10228000FF93E091F003F091F1038091F8039091B6
:10229000F903892B09F44EC08091A014882359F0CA
:1022A0000D9B09C080919A008F7D80939A0089B719
:1022B000806289BF5EC08091F8039091F903019715
:1022C0009093F9038093F80380919E14882321F062
:1022D00080919A00816003C080919A008E7F8093E4
:1022E0009A00819180939C009F018091F4039091CA
:1022F000F503E817F90721F42091F2033091F30375
:102300003093F1032093F0032091F8033091F90307
:102310008091FA039091FB032817390751F5E0915A
:10232000FE03F091FF033097A1F08FEFEF3FF80726
:1023300001F11AC080919A008F7D80939A001092CB
:10234000F9031092F803E091FE03F091FF03309738
:1023500039F48FEF9FEF9093FF038093FE0309C042
:102360008FEFEF3FF80729F08481958101969583DF
:102370008483FF91EF919F918F913F912F910F90C7
:102380000FBE0F901F9018951F920F920FB60F92CD
:1023900011242F933F934F935F936F937F938F936A
:1023A0009F93AF93BF93EF93FF9360919C14A09181
:1023B0009F14B0E080919B00682B70919C0020914D
:1023C0000A0430910B0480910804909109042817A5
:1023D000390708F047C0A9014F5F5F4F41305105F1
:1023E00011F4B1E00AC0AA2341F080910E0490914B
:1023F0000F044817590708F0949AE0910004F091EF
:1024000001047193F0930104E0930004209100040F
:102410003091010480910604909107042817390730
:1024200041F48091040490910504909301048093F9
:10243000000450930B0440930A0480919B0087FD95
:10244000B9CF60939C14BB23D1F0E0911004F091BC
:102450001104309759F48FEF9FEF909311048093FC
:1024600010040DC0686060939C1409C08FEFEF3FAB
:10247000F80729F084819581019695838483FF91E3
:10248000EF91BF91AF919F918F917F916F915F91EC
:102490004F913F912F910F900FBE0F901F90189565
:1024A00080919A0082FF03C089E090E008958091B6
:1024B0009D0082FF0AC080919D0081FF03C088E0DB
:1024C00090E0089587E090E0089580919D0081FF5D
:1024D00003C086E090E0089585E090E00895809143
:1024E0009D0085FD03C080E090E0089580919D00EF
:1024F00084FF03C081E090E0089582E090E00895B9
:1025000080919D0083FF03C082E090E0089581E008
:1025100090E00895EF92FF920F931F9380919C1487
:10252000682F7727CB0174E0969587957A95E1F728
:102530009C0144275527217030704070507063FD16
:10254000226062FD246080919D14882321F086FD25
:10255000426087FD4860949B14C0E12C62E0F62E37
:10256000012D112DE22AF32A042B152B80919F14A3
:10257000882381F0E12C92E0F92E92E0092F112DB1
:1025800005C0E12C81E0F82E012D112DE22AF32A5D
:10259000042B152B0D9B0CC0A8019701386080916E
:1025A000A014882341F0A80197013860426003C05D
:1025B000A8019701346041FF416043FF446080916E
:1025C0009E14882311F0406401C0406880919B00F4
:1025D00080FF04C0CA01B901806103C0CA01B9010A
:1025E00080621F910F91FF90EF900895EF92FF92FC
:1025F0000F931F937B018C0180919D148823D9F048
:102600000FB6F8940F9200FF02C08F7B03C001FF4A
:1026100003C0806480939D1402FF04C080919D14C8
:102620008F7705C003FF05C080919D14806880935B
:102630009D140F900FBE80919F14882321F001FDFF
:10264000949A00FD9498F1FC949AF0FC949806FFFB
:1026500003C081E080939E1407FF02C010929E1475
:1026600004FF05C080919B00816080939B0005FF63
:1026700005C080919B008E7F80939B00E0FE05C08B
:1026800080919C148F7E80939C14E1FE05C0809104
:102690009C14877F80939C14E2FE05C080919C145B
:1026A0008B7F80939C140E948A12687F6E157F0531
:1026B0008007910719F08FEF9FEF02C080E090E054
:1026C0001F910F91FF90EF90089580919D0086FFDC
:1026D0000BC0129B02C093E001C091E080919D006D
:1026E00080FF09C0946007C080919B0081FF02C0F9
:1026F00090E201C090E0892F9927089580919D1460
:10270000882329F020E230E040E050E004C020E0DF
:1027100030E040E050E080919F14882311F0216068
:1027200001C02E7F8091A014882321F0CA01B90135
:1027300062600895CA01B9016D7F0895EAE9F0E089
:10274000808180628083089590919D149923C1F0C7
:1027500096FF16C00FB6F8940F9280919B0085FFEC
:1027600005C081E180939C009F7E01C090619093A1
:102770009D1480919D148F7980939D140F900FBEAE
:1027800080919F1481119498089580E090E00895BD
:102790000F931F930FB6F8940F920AE910E0F80117
:1027A00080818F77808380818F7B808380818F7D04
:1027B00080830F900FBE8AE00E94C80BF8018081D1
:1027C0008F7E80838081877F80831F910F91089502
:1027D0001F93182F0E94C81380919A008B7F8093BB
:1027E0009A0080919D008D7F80939D0080919D0037
:1027F0008B7F80939D001730C1F0183018F416308D
:10280000C9F405C0183061F01930A1F404C08091FA
:102810009D0082600DC080919A00846080939A0030
:1028200080919D00826080939D0080919D008460D6
:1028300080939D000FB6F8940F9288EB80939A00D6
:102840000F900FBE0E945012811719F08FEF9FEF6B
:1028500002C080E090E01F9108958F929F92AF9206
:10286000BF92CF92DF92EF92FF920F931F938090CF
:1028700099009090980080919D0086FF06C0B2E07C
:10288000AB2EB12CC12CD12C0FC080919B0081FFAD
:1028900006C0A8E0AA2EB12CC12CD12C05C0F0E1B5
:1028A000AF2EB12CC12CD12C0E94E00B7B018C01EE
:1028B000282D3327892D9927982F8827282B392BC6
:1028C000442755272F5F3F4F4F4F5F4FC601B5013C
:1028D0000E94EC7E9B01AC01C801B7010E942A7FD7
:1028E000CA01B9011F910F91FF90EF90DF90CF9037
:1028F000BF90AF909F908F9008958091A0148823EF
:1029000059F01092A014159840E050E060E070E09B
:1029100087E394E00E940D7180919F14882319F041
:1029200010929F148C9880E090E00895EF92FF92AF
:102930000F931F937B018C0165FF0BC080919D1449
:10294000882371F40FB6F8940F9281E480939D145C
:1029500005C00FB6F8940F9210929D140F900FBE01
:10296000E0FE06C0949A8C9A81E080939F1407C081
:1029700080919F14882319F010929F148C98E1FE87
:1029800010C040E050E06DE271E187E394E00E9406
:102990000D71892BF9F41D9A159881E08093A0148C
:1029A0000FC08091A014882359F01092A01440E029
:1029B00050E060E070E087E394E00E940D711598AC
:1029C0000E947E136E157F058007910719F480E041
:1029D00090E002C08FEF9FEF1F910F91FF90EF905B
:1029E0000895EF92FF920F931F937B018C010E9439
:1029F000C81380919D0086FD13C080919B0081FFCC
:102A000008C092E0EE0CFF1C001F111F9A95D1F731
:102A100007C083E0EE0CFF1C001F111F8A95D1F741
:102A20000E94E00BA80197010E942A7F2F5F3F4F71
:102A30004F4F5F4F5695479537952795215030401A
:102A400020939900232F3327209398000FB6F894F2
:102A50000F9288EB80939A000F900FBE80E090E079
:102A60001F910F91FF90EF9008951F93182F0E94D0
:102A7000C813812F992780FF1BC081FF02C0129AC3
:102A800001C0129882FF04C080919D00816003C044
:102A900080919D008E7F80939D0080919B008D7F13
:102AA00080939B0080919B00806480939B0015C065
:102AB00085FF04C080919B00826003C080919B00D1
:102AC0008D7F80939B0080919D008E7F80939D00E1
:102AD00080919D008F7B80939D000FB6F8940F929C
:102AE00088EB80939A000F900FBE0E9465138117A8
:102AF00019F08FEF9FEF02C080E090E01F910895E2
:102B00001F93182F0E94C813113071F0113018F064
:102B10001230C1F40DC080919D008F7E80939D0086
:102B200080919D008F7D0CC080919D00806103C0CD
:102B300080919D008F7E80939D0080919D0080629A
:102B400080939D000FB6F8940F9288EB80939A00C3
:102B50000F900FBE0E946F12811719F08FEF9FEF39
:102B600002C080E090E01F9108951F93182F0E94EB
:102B7000C813113021F480919D00877F05C0123069
:102B800029F480919D00886080939D000FB6F89491
:102B90000F9288EB80939A000F900FBE80919D005A
:102BA00083FF03C082E090E002C081E090E018174C
:102BB00019F08FEF9FEF02C080E090E01F91089521
:102BC000CF93DF93EA019C0140E050E0FB0110C08D
:102BD000D9010E949A7F802D9081981721F0D90108
:102BE000092E0E94A27F4F5F5F4F31962F5F3F4FAC
:102BF0004C175D0769F780E090E0DF91CF91089571
:102C0000CF93DF93EA01DC01FB01219724F00E94BE
:102C10009A7F0192FACF80E090E0DF91CF91089502
:102C20009C01FB0189B7482F55274072507089B726
:102C30008F7D89BF21313105D1F1223131054CF42D
:102C400021303105F9F020313105F9F0232BA1F0C5
:102C500066C02831310571F1293131052CF422315A
:102C6000310509F05CC063C029313105B9F120326A
:102C7000310509F054C023C08AB78B7F8ABF8AB759
:102C8000877F8ABF80E288BF1EC008B605FE05C0E8
:102C900081E090E09183808302C011821082452BF5
:102CA00009F445C08081918180689183808320E010
:102CB00030E039C08AB7982F987083FF07C085E04D
:102CC00090E09183808320E030E02BC0943019F4B1
:102CD00087E090E0F6CF81E090E0F3CF60817181F2
:102CE0006130710519F48AB78B7F05C067307105B3
:102CF00031F48AB784608ABF8AB7877F0EC0653097
:102D0000710519F48AB78B7F05C06630710539F4F7
:102D10008AB784608ABF8AB788608ABFD4CF2FEF12
:102D20003FEF452B31F089B7806289BF02C020E0B8
:102D300030E0C90108951F920F920FB60F9211242F
:102D40002F933F934F935F936F937F938F939F93B3
:102D5000AF93BF93EF93FF9387E394E00E94FF70DC
:102D6000FF91EF91BF91AF919F918F917F916F9163
:102D70005F914F913F912F910F900FBE0F901F9039
:102D800018959C01FB018AB1482F55274078507057
:102D9000579820313105D9F0213131053CF4211506
:102DA000310581F02130310551F40EC02231310559
:102DB00059F122313105DCF020323105D9F08FEFA5
:102DC0009FEF1EC040E050E08CB18CB117C05F9BFC
:102DD00005C081E090E09183808302C0118210825F
:102DE000452B91F08081918180689183808380E080
:102DF00090E008C080E190E09183808380E090E0E3
:102E0000452B21F0579A089580E090E008951F9295
:102E10000F920FB60F9211242F933F934F935F930E
:102E20006F937F938F939F93AF93BF93EF93FF9392
:102E30008DE394E00E94FF70FF91EF91BF91AF91FD
:102E40009F918F917F916F915F914F913F912F91C2
:102E50000F900FBE0F901F9018959C01FB018AB137
:102E6000482F55274072507055982131310519F17E
:102E7000223131053CF42115310551F12031310564
:102E800039F409C02231310519F120323105B1F090
:102E90008FEF9FEF19C05D9B05C081E090E09183AB
:102EA000808302C011821082452B91F08081918134
:102EB00080689183808380E090E008C080E190E0AA
:102EC0009183808380E090E0452B21F0559A08950E
:102ED00080E090E008951F920F920FB60F92112498
:102EE0002F933F934F935F936F937F938F939F9312
:102EF000AF93BF93EF93FF9383E494E00E94FF703E
:102F0000FF91EF91BF91AF919F918F917F916F91C1
:102F10005F914F913F912F910F900FBE0F901F9097
:102F200018959C01FB0189B7482F552740715070B7
:102F300089B78F7E89BF21313105D1F12231310529
:102F40004CF421303105F9F020313105F9F0232B13
:102F5000A1F069C02831310571F1293131052CF416
:102F60002231310509F05FC066C029313105B9F160
:102F70002032310509F057C053C08AB78E7F8ABF0F
:102F80008AB78D7F8ABF80E188BF1EC008B604FE65
:102F900005C081E090E09183808302C0118210829D
:102FA000452B09F448C0808191818068918380839A
:102FB00020E030E03CC08AB7982F927081FF07C0B4
:102FC00085E090E09183808320E030E02EC0913056
:102FD00019F487E090E0F6CF81E090E0F3CF6081D4
:102FE00071816130710519F48AB78E7F05C0673031
:102FF000710531F48AB781608ABF8AB78D7F0EC0B0
:103000006530710519F48AB78E7F05C06630710589
:1030100051F48AB781608ABF8AB782608ABFD4CFF1
:1030200084E090E0CFCF2FEF3FEF452B31F089B711
:10303000806189BF02C020E030E0C90108951F927D
:103040000F920FB60F9211242F933F934F935F93DC
:103050006F937F938F939F93AF93BF93EF93FF9360
:1030600089E494E00E94FF70FF91EF91BF91AF91CE
:103070009F918F917F916F915F914F913F912F9190
:103080000F900FBE0F901F901895FC0180819181C9
:103090000895CF92DF92EF92FF920F931F93CF93F9
:1030A000DF936C01CB010E94A01D7C018F5F9F4FBD
:1030B00071F440C00F5F1F4F32960830110559F46C
:1030C00087E190E0909368168093671633C003E021
:1030D00010E0E5E5F4E080819181892B59F787E0E4
:1030E00090E00E94291AEC01000F111F015B1B4F99
:1030F000D801CD93DC932097E9F0B701C6010E9477
:10310000BB1999838883D801ED91FC918F5F9F4F04
:1031100039F4CF010E94261AF801118210820AC0E8
:10312000F382E2821482D801ED91FC91168215821D
:10313000CF0102C080E090E0DF91CF911F910F910D
:10314000FF90EF90DF90CF9008959F92AF92BF9243
:10315000CF92DF92EF92FF920F931F93CF93DF9363
:103160005C01CB01EA010E94A01D6C018F5F9F4FA3
:1031700071F448C00F5F1F4F32960830110559F4A3
:1031800089E090E090936816809367163BC000E05A
:1031900010E0EFE4F4E0808191818C179D0751F7F6
:1031A00087E090E00E94291A7C01E801CC0FDD1F26
:1031B000C15BDB4FF982E882E114F10419F1B60139
:1031C000C5010E94BB19F70191838083E881F981D1
:1031D0008F5F9F4F71F4CF010E94261A82E0801703
:1031E00028F00F5F1F4F198308830CC019821882C3
:1031F00009C0D382C2821482E881F98116821582C5
:10320000CF0102C080E090E0DF91CF911F910F913C
:10321000FF90EF90DF90CF90BF90AF909F90089578
:10322000CF93DF93CDB7DEB722970FB6F894DEBF0A
:103230000FBECDBFFE01379661917191FA83E9838C
:10324000AF0180915104909152040E946519229619
:103250000FB6F894DEBF0FBECDBFDF91CF910895BA
:1032600060915104709152040E94F41D8F5F9F4F32
:1032700019F48FEF9FEF08956091510470915204FB
:103280008AE090E00E94CC1D80E090E00895CF930A
:10329000DF93CDB7DEB722970FB6F894DEBF0FBE2F
:1032A000CDBFAE01455F5F4F5A83498369857A85FB
:1032B0008F8198850E94701922960FB6F894DEBF10
:1032C0000FBECDBFDF91CF910895FC01CB019A01D4
:1032D00060817181AC0183E19AE10E945E1A0895D8
:1032E000CF93DF93CDB7DEB722970FB6F894DEBF4A
:1032F0000FBECDBF9A8389839A01AB01BE016F5F78
:103300007F4F81E999E10E945E1AE981FA8110827A
:1033100022960FB6F894DEBF0FBECDBFDF91CF91DE
:103320000895EF92FF920F931F937C018A01FC0195
:10333000808191810E94A77EF70180819181800F19
:10334000911F91838083C8011F910F91FF90EF908F
:103350000895CF93DF93EC01AA81BB81109719F4F4
:10336000EB85FC8504C0ED01ED89FE89CD01099551
:10337000DF91CF910895EF92FF920F931F93CF9318
:10338000DF93CDB7DEB729970FB6F894DEBF0FBE37
:10339000CDBF7B018C01FE013196AE01475F5F4FCF
:1033A00003C021930F5F1F4F302F381BD8012C9182
:1033B000222329F02A3319F0E417F50791F7CE01FB
:1033C0000196FC01E30FF11D10820E94FD03DC0158
:1033D000892B49F482E090E09093681680936716F9
:1033E0008FEF9FEF13C0F80180818A3319F060E0FE
:1033F00070E003C0B8016F5F7F4FFD01058D168D32
:1034000020E030E0A701CD01F801099529960FB61B
:10341000F894DEBF0FBECDBFDF91CF911F910F910A
:10342000FF90EF900895CF93DF93DC01EC01EA81E8
:10343000FB81309719F4EF81F88503C0018CF28D80
:10344000E02DCD010995DF91CF9108950E94C80824
:1034500008950E9455089C01892B31F48CE090E07E
:103460009093681680936716C9010895CF92DF92F2
:10347000EF92FF920F931F93CF93DF936C017B0129
:103480008A01E90107C040E150E0B801C701F60137
:1034900009956097C131D105B4F71C161D062CF4AF
:1034A000AE01B801C701F6010995DF91CF911F91D7
:1034B0000F91FF90EF90DF90CF9008952F923F9261
:1034C0004F925F926F927F928F929F92AF92BF9234
:1034D000CF92DF92EF92FF920F931F93CF93DF93E0
:1034E000CDB7DEB76B970FB6F894DEBF0FBECDBF7A
:1034F000998F888F7B8F6A8F1A0159011D8A1C8AC8
:10350000B10103C00894211C311CD101FC90FF20A3
:1035100019F0B5E2FB16B1F78101061B170B61F03C
:10352000A8018A8D9B8DE88DF98D09952C893D899F
:10353000200F311F3D8B2C8BFF2009F4E6C2F101D7
:103540003196198266241B8A1A8A4FEF442E542E14
:1035500002C05C01F101DF019D901D01B0E29B16EC
:1035600021F489818823B1F703C02BE2921611F46C
:103570009982F0CF3DE2931619F444E0642AEACF31
:1035800053E2951619F461E0662AE4CF70E39716CA
:1035900019F480E1682ADECF9CE6991619F4A8E0B8
:1035A0006A2AD8CFBAE79B16A9F22AE2921691F4BA
:1035B000C5010296D501AD90BC90BB8AAA8AB7FE20
:1035C000C8CFB4E06B2AF501F095E195FF4FFB8B76
:1035D000EA8BBFCF2EE2921691F581818A3219F0E3
:1035E000442455241FC00894211C311CD5014D9042
:1035F0005C90E2E0F0E0AE0EBF1E1BC08AE090E0FF
:10360000A201489F2001499F500C589F500C112443
:10361000822F992787FD9095480E591E60ED7FEF08
:10362000460E571E21813196822F80538A3030F307
:103630001F0157FE8FCF3FEF432E532E8BCF892D87
:103640008153893010F5892D9927C0979B8B8A8BE0
:103650002AE030E012C04A895B89429FD001439F33
:10366000B00D529FB00D1124892F992787FD909599
:10367000A80FB91FD097BB8BAA8B91813196892F48
:1036800080538A3040F31F0165CFF501792C57E64E
:103690005915E8F065E6961608F09FC170E5971693
:1036A000D1F1791548F085E4981609F496C197E4AC
:1036B000991609F096C191C1A3E69A1621F1A915B0
:1036C00008F472C0B8E59B1609F08BC128C120E749
:1036D000921609F424C1291548F039E6931609F425
:1036E00063C04FE6941609F07CC1CDC055E795162E
:1036F00009F459C068E7961609F411C173E79716E3
:1037000009F06FC124C082E090E0A80EB91E80814C
:103710008A8319826CC1A2E0B0E0AA0EBB1EE080D1
:10372000F180E114F10439F42FE5C22E24E0D22E09
:1037300093E7792E19C0C7010E94917E01960E94DD
:10374000291A8C01B7010E948A7E680106C022E016
:1037500030E0A20EB31EC080D180C114D10421F488
:103760008FE5C82E84E0D82E57FC12C0A20160E07D
:1037700070E0C6010E949A7E009711F4820111C088
:103780008C199D098201841595055CF48C0109C092
:10379000D6010D900020E9F78D01015010400C1961
:1037A0001D091982AAC1198263FE0CC024E030E011
:1037B000A20EB31EE080F1800281138135E79316DB
:1037C000B1F421C0D5011296F50100811181F5E710
:1037D0009F1631F45D01980179010027112713C06C
:1037E0005D01A8017A010027F7FC0095102F17FF53
:1037F0000AC010950095F094E094E11CF11C011DA5
:10380000111D8DE2898357FC02C05FEE6522E11431
:10381000F1040105110539F44114510451F402E198
:10382000C02ED12C0CC06AE0E616F104010511058A
:1038300048F48E2D805D898B11E1C12ED12CCC0EE8
:10384000DD1EC4C0B2E1CB2ED12CCC0EDD1EC801D2
:10385000B7012AE030E040E050E00E942A7F605D3E
:10386000D6016E936D01C801B7012AE030E040E057
:1038700050E00E942A7F79018A0121153105410516
:10388000510529F7A3C063FE09C024E030E0A20E71
:10389000B31E008111812281338109C042E050E0D2
:1038A000A40EB51E808191818C01222733271982B5
:1038B00057FC02C05FEE6522011511052105310597
:1038C00049F44114510431F4A2E1CA2ED12CCC0E9A
:1038D000DD1E1FC0F2E1CF2ED12CCC0EDD1E802FBD
:1038E0008770805DD6018E936D01E3E03695279554
:1038F00017950795EA95D1F70115110521053105B1
:1039000071F760FE06C0803321F080E3FD018293F1
:103910006F018E010C191D090E5E1F4F70C020E74C
:10392000921671F442E050E0A40EB51E80819181A0
:103930008C012227332751E0652A78E7972E14C09F
:1039400063FE09C064E070E0A60EB71E008111811D
:103950002281338109C082E090E0A80EB91E8081E7
:1039600091818C012227332757FC02C09FEE6922E8
:10397000A8E59A1619F046E654E002C047E754E07D
:10398000198262E1C62ED12CCC0EDD1EF801EF703B
:10399000F070E40FF51F8081F60182936F0194E0CF
:1039A00036952795179507959A95D1F70115110525
:1039B0002105310559F760FE09C0319790826F01EA
:1039C0000894C108D10880E3D6018C938E010C19AC
:1039D0001D090E5E1F4F792C12C0E4E0F0E0AE0E20
:1039E000BF1E992009F491C09A821982792C82E035
:1039F000C82ED12CCC0EDD1E01E010E07EC0780177
:103A0000041515050CF472018981882319F00894B6
:103A1000E11CF11C4201262D33273F8B2E8B2901FF
:103A200034E1432255244114510461F42A893B892D
:103A30002E193F0948E854E06A8D7B8D888D998D59
:103A40000E94361A8981882359F041E050E0BE0176
:103A50006F5F7F4F8A8D9B8DA88DB98DFD01099574
:103A6000B0E14B16510461F42A893B892E193F09B4
:103A700048E954E06A8D7B8D888D998D0E94361AB5
:103A8000801A910A940148E954E06A8D7B8D888DF3
:103A9000998D0E94361A0115110539F0A801B60159
:103AA0008A8D9B8DE88DF98D0995F0E57F1619F4C7
:103AB000C6010E94261A2E8922FF0CC02A893B8942
:103AC0002E193F0948E854E06A8D7B8D888D998DC9
:103AD0000E94361A4A895B894E155F053CF06C8955
:103AE0007D89640F751F7D8B6C8B0ACD8C899D89B8
:103AF0008E0D9F1D9D8B8C8B03CD780117FF02C00F
:103B0000EE24FF248824992486CF8C899D896B9686
:103B10000FB6F894DEBF0FBECDBFDF91CF911F91DE
:103B20000F91FF90EF90DF90CF90BF90AF909F905C
:103B30008F907F906F905F904F903F902F9008955F
:103B4000FC018081823759F0873719F08136B1F452
:103B500003C081E093E41BC088E091E418C080E0DA
:103B600090E415C02B3219F0223641F404C08E7F48
:103B7000826093600CC09F7B906809C086E190E0F2
:103B800090936816809367168FEF9FEF0895319694
:103B90002081222339F708950F931F93CF93DF934A
:103BA000CDB7DEB721970FB6F894DEBF0FBECDBFFD
:103BB0008C01FB01898341E050E0BE016F5F7F4FC4
:103BC000808191810E94131A019711F00FEF1FEF6E
:103BD000C80121960FB6F894DEBF0FBECDBFDF91AE
:103BE000CF911F910F910895FC01CB01DF010D9042
:103BF0000020E9F71197AE1BBF0BAD01BF01FC011F
:103C0000808191810E94131A08958F929F92AF92A2
:103C1000BF92CF92DF92EF92FF920F931F93CF93B9
:103C2000DF93CDB7DEB72C970FB6F894DEBF0FBE8B
:103C3000CDBF6C014B01142F9CE6A92E93E0B92E49
:103C4000AC0CBD1C96012F5E3F4F83E4E82EF12C97
:103C500003E0AB01BE016F5F7F4FC6010E943837A2
:103C60007C01F50180899189892B39F481E090E00C
:103C70000E945508F501918B808BF501A089B189CF
:103C80001C9381E0F601848B158B0FEF1FEF2CE066
:103C900033E4A401B701C6010E948C372C960FB6FD
:103CA000F894DEBF0FBECDBFDF91CF911F910F9172
:103CB000FF90EF90DF90CF90BF90AF909F908F904C
:103CC0000895AF92BF92CF92DF92EF92FF920F933F
:103CD0001F93CF93DF93CDB7DEB72C970FB6F89431
:103CE000DEBF0FBECDBF6C015B019C012F5E3F4F5D
:103CF00042E4E42EF12C03E0AB01BE016F5F7F4F85
:103D00000E943837F601148A0FEF1FEF2CE032E4DF
:103D1000A501BC01C6010E948C372C960FB6F89401
:103D2000DEBF0FBECDBFDF91CF911F910F91FF90EE
:103D3000EF90DF90CF90BF90AF9008958F929F92B9
:103D4000AF92BF92CF92DF92EF92FF920F931F93A9
:103D5000CF93DF93CDB7DEB72C970FB6F894DEBFC5
:103D60000FBECDBF6C014B01142F6CE6A62E63E095
:103D7000B62EA80EB91E9C012F5E3F4F55E4E52ECE
:103D8000F12C03E0A401BE016F5F7F4F0E94383722
:103D90007C01F50186859785892B39F481E090E0D7
:103DA0000E945508F50197878687F501A685B78596
:103DB0001C9381E0F601848B158B0FEF1FEF2CE035
:103DC00035E4A401B701C6010E948C372C960FB6CA
:103DD000F894DEBF0FBECDBFDF91CF911F910F9141
:103DE000FF90EF90DF90CF90BF90AF909F908F901B
:103DF0000895AF92BF92CF92DF92EF92FF920F930E
:103E00001F93CF93DF93CDB7DEB72C970FB6F894FF
:103E1000DEBF0FBECDBF6C015B019C012F5E3F4F2B
:103E200074E4E72EF12C03E0A501BE016F5F7F4F24
:103E30000E943837F601148A0FEF1FEF2CE034E4AC
:103E4000A501BC01C6010E948C372C960FB6F894D0
:103E5000DEBF0FBECDBFDF91CF911F910F91FF90BD
:103E6000EF90DF90CF90BF90AF9008952F923F9248
:103E70004F925F926F927F928F929F92AF92BF927A
:103E8000CF92DF92EF92FF920F931F93CF93DF9326
:103E9000CDB7DEB72D970FB6F894DEBF0FBECDBFFE
:103EA0006C011B014A012D87380127018CE6A82EE1
:103EB00083E0B82EAC0CBD1C96012F5E3F4F03E390
:103EC000E02EF12C03E0AB01BE016F5F7F4FC60116
:103ED0000E9438377C01F50184859585892B39F45A
:103EE00087E090E00E945508F50195878487F501E9
:103EF000A485B58511969C928E928D85FD01828355
:103F0000F501A485B585FD017482638256824582E0
:103F100087E0F601848B858A892D9927868B8D858C
:103F2000878B608E872D9927818F428E852D9927CB
:103F3000838F0FEF1FEF2CE033E3A101B701C60120
:103F40000E948C372D960FB6F894DEBF0FBECDBF02
:103F5000DF91CF911F910F91FF90EF90DF90CF9065
:103F6000BF90AF909F908F907F906F905F904F9099
:103F70003F902F9008958F929F92AF92BF92CF92D1
:103F8000DF92EF92FF920F931F93CF93DF93CDB702
:103F9000DEB72C970FB6F894DEBF0FBECDBF6C0115
:103FA0004B01142F2CE6A22E23E0B22EA80EB91E30
:103FB0009C012F5E3F4F91E3E92EF12C03E0AB0112
:103FC000BE016F5F7F4FC6010E9438377C01F5014B
:103FD00082859385892B39F481E090E00E94550811
:103FE000F50193878287F501A285B3851C9381E053
:103FF000F601848B158B0FEF1FEF2CE031E3A4014A
:10400000B701C6010E948C372C960FB6F894DEBF1C
:104010000FBECDBFDF91CF911F910F91FF90EF9019
:10402000DF90CF90BF90AF909F908F9008954F9268
:104030005F926F927F928F929F92AF92BF92CF9238
:10404000DF92EF92FF920F931F93CF93DF93CDB741
:10405000DEB72C970FB6F894DEBF0FBECDBF6C0154
:104060002B0149015A016CE6662E63E0762E680E3C
:10407000791E9C012F5E3F4F54E2E52EF12C03E0A8
:10408000A201BE016F5F7F4F0E9438377C01F301B0
:1040900082899389892B39F484E090E00E94550845
:1040A000F301938B828BF301A289B3898D929D9248
:1040B000AD92BC92139783E0F601848B858ABB276F
:1040C000AB2D9A2D892D868BC501AA27BB27878BFF
:1040D0000FEF1FEF2CE034E2A201B701C6010E94EE
:1040E0008C372C960FB6F894DEBF0FBECDBFDF9194
:1040F000CF911F910F91FF90EF90DF90CF90BF90E5
:10410000AF909F908F907F906F905F904F900895A9
:10411000AF92BF92CF92DF92EF92FF920F931F93D5
:10412000CF93DF93CDB7DEB72C970FB6F894DEBFF1
:104130000FBECDBF6C015B019C012F5E3F4F73E250
:10414000E72EF12C03E0A501BE016F5F7F4F0E94B7
:104150003837F601148A0FEF1FEF2CE033E2A50188
:10416000BC01C6010E948C372C960FB6F894DEBFB6
:104170000FBECDBFDF91CF911F910F91FF90EF90B8
:10418000DF90CF90BF90AF9008958F929F92AF92A3
:10419000BF92CF92DF92EF92FF920F931F93CF9334
:1041A000DF93CDB7DEB72C970FB6F894DEBF0FBE06
:1041B000CDBF6C014B01142FFCE6AF2EF3E0BF2EF8
:1041C000A80EB91E9C012F5E3F4FEAE1EE2EF12CA6
:1041D00003E0AB01BE016F5F7F4F0E9438377C0167
:1041E000F501828D938D892B39F481E090E00E9456
:1041F0005508F501938F828FF501A28DB38D1C9325
:1042000081E0F601848B158B0FEF1FEF2CE03AE174
:10421000A401B701C6010E948C372C960FB6F89402
:10422000DEBF0FBECDBFDF91CF911F910F91FF90E9
:10423000EF90DF90CF90BF90AF909F908F900895B8
:10424000AF92BF92CF92DF92EF92FF920F931F93A4
:10425000CF93DF93CDB7DEB72C970FB6F894DEBFC0
:104260000FBECDBF6C015B019C012F5E3F4FA9E1EA
:10427000EA2EF12C03E0AB01BE016F5F7F4F0E947D
:104280003837F601148A0FEF1FEF2CE039E1A50152
:10429000BC01C6010E948C372C960FB6F894DEBF85
:1042A0000FBECDBFDF91CF911F910F91FF90EF9087
:1042B000DF90CF90BF90AF9008956F927F928F92D2
:1042C0009F92AF92BF92CF92DF92EF92FF920F93A5
:1042D0001F93CF93DF93CDB7DEB72C970FB6F8942B
:1042E000DEBF0FBECDBF6C013B014A010CE6A02E24
:1042F00003E0B02EA80EB91E9C012F5E3F4F18E1BF
:10430000E12EF12C03E0AB01BE016F5F7F4F0E94F5
:1043100038377C01F50186899789892B39F482E049
:1043200090E00E945508F501978B868BF501A689D0
:10433000B7898D929C9282E0F601848B858A892DC3
:104340009927868B0FEF1FEF2CE038E1A301B7010F
:10435000C6010E948C372C960FB6F894DEBF0FBEB4
:10436000CDBFDF91CF911F910F91FF90EF90DF9024
:10437000CF90BF90AF909F908F907F906F90089557
:10438000AF92BF92CF92DF92EF92FF920F931F9363
:10439000CF93DF93CDB7DEB72C970FB6F894DEBF7F
:1043A0000FBECDBF6C015B019C012F5E3F4F87E1CB
:1043B000E82EF12C03E0AB01BE016F5F7F4FC60119
:1043C0000E943837F601148A0FEF1FEF2CE037E117
:1043D000A501BC01C6010E948C372C960FB6F8943B
:1043E000DEBF0FBECDBFDF91CF911F910F91FF9028
:1043F000EF90DF90CF90BF90AF9008956F927F9233
:104400008F929F92AF92BF92CF92DF92EF92FF92E4
:104410000F931F93CF93DF93CDB7DEB72C970FB6D3
:10442000F894DEBF0FBECDBF6C013B014A015CE6D4
:10443000A52E53E0B52EA80EB91E9C012F5E3F4F4E
:1044400046E1E42EF12C03E0AB01BE016F5F7F4F2C
:104450000E9438377C01F50182819381892B39F4E0
:1044600082E090E00E945508F50193838283F50174
:10447000A281B3818D929C9282E0F601848B858A21
:10448000892D9927868B0FEF1FEF2CE036E1A301D2
:10449000B701C6010E948C372C960FB6F894DEBF88
:1044A0000FBECDBFDF91CF911F910F91FF90EF9085
:1044B000DF90CF90BF90AF909F908F907F906F9044
:1044C0000895AF92BF92CF92DF92EF92FF920F9337
:1044D0001F93CF93DF93CDB7DEB72C970FB6F89429
:1044E000DEBF0FBECDBF6C015B019C012F5E3F4F55
:1044F00065E1E62EF12C03E0A501BE016F5F7F4F61
:104500000E943837F601148A0FEF1FEF2CE035E1D7
:10451000A501BC01C6010E948C372C960FB6F894F9
:10452000DEBF0FBECDBFDF91CF911F910F91FF90E6
:10453000EF90DF90CF90BF90AF9008954F925F9231
:104540006F927F928F929F92AF92BF92CF92DF92A3
:10455000EF92FF920F931F93CF93DF93CDB7DEB708
:104560002C970FB6F894DEBF0FBECDBF4C012B01C8
:104570003A01A22E9C012F5E3F4F74E1E72EF12CF1
:1045800003E0A201BE016F5F7F4F0E943837FC013C
:1045900071866086BB24CC24DD24A482B582C682C9
:1045A000D782F401148A0FEF1FEF2CE034E1A2014F
:1045B000BC01C4010E948C372C960FB6F894DEBF64
:1045C0000FBECDBFDF91CF911F910F91FF90EF9064
:1045D000DF90CF90BF90AF909F908F907F906F9023
:1045E0005F904F9008958F929F92AF92BF92CF921B
:1045F000DF92EF92FF920F931F93CF93DF93CDB78C
:10460000DEB72C970FB6F894DEBF0FBECDBF6C019E
:104610004B01142FFCE6AF2EF3E0BF2EA80EB91EFF
:104620009C012F5E3F4FEAE0EE2EF12C03E0AB0140
:10463000BE016F5F7F4F0E9438377C01F501808D8E
:10464000918D892B39F481E090E00E945508F501A5
:10465000918F808FF501A08DB18D1C9381E0F601C3
:10466000848B158B0FEF1FEF2CE03AE0A401B7010C
:10467000C6010E948C372C960FB6F894DEBF0FBE91
:10468000CDBFDF91CF911F910F91FF90EF90DF9001
:10469000CF90BF90AF909F908F900895AF92BF92B0
:1046A000CF92DF92EF92FF920F931F93CF93DF93FE
:1046B000CDB7DEB72C970FB6F894DEBF0FBECDBFD7
:1046C0006C015B019C012F5E3F4FA9E0EA2EF12CAB
:1046D00003E0AB01BE016F5F7F4F0E943837F601E8
:1046E000148A0FEF1FEF2CE039E0A501BC01C601D1
:1046F0000E948C372C960FB6F894DEBF0FBECDBF4C
:10470000DF91CF911F910F91FF90EF90DF90CF90AD
:10471000BF90AF900895AF92BF92CF92DF92EF9289
:10472000FF920F931F93CF93DF93CDB7DEB72C97F4
:104730000FB6F894DEBF0FBECDBF6C015B01FC016C
:10474000EB5BFD4F8081882329F06BEF7EEF8FEFCD
:104750009FEF1BC081E0808396012F5E3F4FB3E047
:10476000EB2EF12C03E0AB01BE016F5F7F4FC60162
:104770000E943837F601148A0FEF1FEF2CE033E068
:10478000A501BC01C6010E948C372C960FB6F89487
:10479000DEBF0FBECDBFDF91CF911F910F91FF9074
:1047A000EF90DF90CF90BF90AF9008952F923F92FF
:1047B0004F925F926F927F928F929F92AF92BF9231
:1047C000CF92DF92EF92FF920F931F93CF93DF93DD
:1047D000CDB7DEB72E970FB6F894DEBF0FBECDBFB4
:1047E0006C017E876D8729013A01470158015CE61B
:1047F000252E53E0352E280E391E9C012F5E3F4F8B
:1048000041E0E42EF12C03E0AB01BE016F5F7F4F6E
:104810000E9438377C01F10180859185892B39F41C
:1048200088E090E00E945508F10191878087F101AE
:10483000A085B1854D925D926D927C921397FD019A
:1048400084829582A682B78288E0F601848B858A6D
:10485000BB27AB2D9A2D892D868BC501AA27BB2797
:10486000878B8B2D9927AA27BB27808F418EBB274B
:10487000A72D962D852D828FC301AA27BB27838F55
:10488000872D9927AA27BB27848F0FEF1FEF2CE0D6
:1048900031E04D855E85B701C6010E948C372E96AA
:1048A0000FB6F894DEBF0FBECDBFDF91CF911F9141
:1048B0000F91FF90EF90DF90CF90BF90AF909F90BF
:1048C0008F907F906F905F904F903F902F900895C2
:1048D0004F925F926F927F928F929F92AF92BF9210
:1048E000CF92DF92EF92FF920F931F93CF93DF93BC
:1048F000CDB7DEB72C970FB6F894DEBF0FBECDBF95
:104900006C012B013A014901BA010E941B375C017D
:104910008FEFA8168FEFB80629F46DEF7EEF8FEFBB
:104920009FEF21C096012F5E3F4FE7E3EE2EF12C63
:1049300003E0A201BE016F5F7F4FC6010E943837BE
:1049400024E0F601248BA58A2B2D3327268B878A1A
:10495000292D3327208F83012CE037E3A201BC01EE
:10496000C6010E948C372C960FB6F894DEBF0FBE9E
:10497000CDBFDF91CF911F910F91FF90EF90DF900E
:10498000CF90BF90AF909F908F907F906F905F90EF
:104990004F9008956F927F928F929F92AF92BF92A5
:1049A000CF92DF92EF92FF920F931F93CF93DF93FB
:1049B000CDB7DEB72C970FB6F894DEBF0FBECDBFD4
:1049C0006C013B014A01BA010E941B375C018FEF69
:1049D000A8168FEFB80629F46DEF7EEF8FEF9FEFEB
:1049E0001DC096012F5E3F4FB6E3EB2EF12C03E086
:1049F000A301BE016F5F7F4FC6010E94383722E0DE
:104A0000F601248BA58A2B2D3327268B84012CE0DD
:104A100036E3A301BC01C6010E948C372C960FB669
:104A2000F894DEBF0FBECDBFDF91CF911F910F91E4
:104A3000FF90EF90DF90CF90BF90AF909F908F90BE
:104A40007F906F9008956F927F928F929F92AF9216
:104A5000BF92CF92DF92EF92FF920F931F93CF936B
:104A6000DF93CDB7DEB72C970FB6F894DEBF0FBE3D
:104A7000CDBF6C013B014A010E941B375C018FEFE7
:104A8000A8168FEFB80629F46DEF7EEF8FEF9FEF3A
:104A900026C096012F5E3F4F85E3E82EF12C03E000
:104AA00040E050E0BE016F5F7F4FC6010E94383783
:104AB00085E0F601848B81E0858BA68A8B2D992772
:104AC000878B808E892D9927818F83012CE035E398
:104AD00040E050E060E070E0C6010E948C372C9608
:104AE0000FB6F894DEBF0FBECDBFDF91CF911F91FF
:104AF0000F91FF90EF90DF90CF90BF90AF909F907D
:104B00008F907F906F9008956F927F928F929F9277
:104B1000AF92BF92CF92DF92EF92FF920F931F93CB
:104B2000CF93DF93CDB7DEB72C970FB6F894DEBFE7
:104B30000FBECDBF6C013B015A012CE6822E23E053
:104B4000922E880E991E9C012F5E3F4F93E1E92E15
:104B5000F12C03E0AB01BE016F5F7F4FC6010E94E5
:104B600038377C01F40184899589892B59F489EFC0
:104B700090E00E945508DC01F401958B848BA850CD
:104B8000BF4F1C92F50101900020E9F73197EA1917
:104B9000FB09E83FF10518F049EF50E003C0AF0111
:104BA0004F5F5F4FB501F401848995890E94A77E0C
:104BB00088EFF601848BF50120E030E0D6015596B0
:104BC000922F80818D938081882351F09F5F2F5F8A
:104BD0003F4F3196283F310599F7983F09F497EFF9
:104BE000F601E90FF11D158A0FEF1FEF2CE033E1FD
:104BF000A301B701C6010E948C372C960FB6F8941A
:104C0000DEBF0FBECDBFDF91CF911F910F91FF90FF
:104C1000EF90DF90CF90BF90AF909F908F907F905C
:104C20006F9008958F929F92AF92BF92CF92DF9232
:104C3000EF92FF920F931F93CF93DF93CDB7DEB721
:104C40002C970FB6F894DEBF0FBECDBF6C014B01A1
:104C50005A019C012F5E3F4F45E0E42EF12C03E00A
:104C6000AB01BE016F5F7F4F0E9438377C01F501B9
:104C7000408155274F5F5F4FB501C60144960E94A2
:104C8000A77E0FEF1FEF2CE035E0A401B701C601AE
:104C90000E948C372C960FB6F894DEBF0FBECDBFA6
:104CA000DF91CF911F910F91FF90EF90DF90CF9008
:104CB000BF90AF909F908F900895AF92BF92DF9278
:104CC000EF92FF920F931F93CF93DF93CDB7DEB791
:104CD00022970FB6F894DEBF0FBECDBFAE84BF845F
:104CE000DA88BCE6EB2EB3E0FB2EEA0CFB1CCE010F
:104CF00043969A838983F70186819781892B39F4BA
:104D00008CE090E00E945508F70197838683F701B5
:104D100086819781DC011196FC01D182BD016F5F14
:104D20007F4FF7012681378181E0F90180838D2D46
:104D30008150823008F069C0E981FA813296FA83A5
:104D4000E98332978081FD0181836F5F7F4F8130DE
:104D500079F0813040F0823009F443C06EEE7FEF8D
:104D60008FEF9FEF6CC0F701A681B78182E04CC046
:104D7000E981FA813496FA83E98352914291329122
:104D80002291FB0121938F01BB27A52F942F832F05
:104D9000FB018183B8016F5F7F4F9A01442755273C
:104DA000F80121838B010F5F1F4FE981FA8134964F
:104DB000FA83E983B291A29192918291FB0181835E
:104DC000B8016F5F7F4F292F3A2F4B2F5527F801DE
:104DD0002183CD01AA27BB27FB0181836E5F7F4F13
:104DE0000FC0E981FA813296FA83E983CB01B2914F
:104DF000A29126E00D90FC010192CF012150D1F744
:104E0000F701A681B78188E08C93F2E0DF1679F490
:104E1000E981FA813296FA83E98332978081FB0136
:104E20008083F701A681B7818C918F5F8C93F70106
:104E30004681578168897989C5010E941226229688
:104E40000FB6F894DEBF0FBECDBFDF91CF911F919B
:104E50000F91FF90EF90DF90BF90AF9008958F92E9
:104E60009F92AF92BF92CF92DF92EF92FF920F93F9
:104E70001F93CF93DF93CDB7DEB72C970FB6F8947F
:104E8000DEBF0FBECDBF6C015B014A019C012F5EEE
:104E90003F4F89E0E82EF12C04E0AB01BE016F5FCB
:104EA0007F4FC6010E943837FC0191868086F6014B
:104EB000148A0FEF1FEF20E139E0A501BC01C60104
:104EC0000E948C372C960FB6F894DEBF0FBECDBF74
:104ED000DF91CF911F910F91FF90EF90DF90CF90D6
:104EE000BF90AF909F908F900895AF92BF92CF9256
:104EF000DF92EF92FF920F931F93CF93DF93CDB783
:104F0000DEB72C970FB6F894DEBF0FBECDBF6C0195
:104F10005B019C012F5E3F4F95E0E92EF12C04E0F0
:104F2000AB01BE016F5F7F4FC6010E943837F601AB
:104F3000148A0FEF1FEF20E135E0A501BC01C60187
:104F40000E948C372C960FB6F894DEBF0FBECDBFF3
:104F5000DF91CF911F910F91FF90EF90DF90CF9055
:104F6000BF90AF900895AF92BF92CF92DF92EF9231
:104F7000FF920F931F93CF93DF93CDB7DEB72C979C
:104F80000FB6F894DEBF0FBECDBF6C015B019C0174
:104F90002F5E3F4F44E0E42EF12C04E0AB01BE0154
:104FA0006F5F7F4F0E943837F601148A0FEF1FEFB3
:104FB00020E134E0A501BC01C6010E948C372C968B
:104FC0000FB6F894DEBF0FBECDBFDF91CF911F911A
:104FD0000F91FF90EF90DF90CF90BF90AF9008952A
:104FE0008F929F92AF92BF92CF92DF92EF92FF92F9
:104FF0000F931F93CF93DF93CDB7DEB72C970FB6E8
:10500000F894DEBF0FBECDBF6C015B014A019C016D
:105010002F5E3F4F53E0E52EF12C04E0AB01BE01C3
:105020006F5F7F4F0E943837FC0191868086F601C2
:10503000148A0FEF1FEF20E133E0A501BC01C60188
:105040000E948C372C960FB6F894DEBF0FBECDBFF2
:10505000DF91CF911F910F91FF90EF90DF90CF9054
:10506000BF90AF909F908F900895AF92BF92CF92D4
:10507000DF92EF92FF920F931F93CF93DF93CDB701
:10508000DEB72C970FB6F894DEBF0FBECDBF6C0114
:105090005B019C012F5E3F4F62E0E62EF12C04E0A5
:1050A000A501BE016F5F7F4F0E943837F601148A59
:1050B0000FEF1FEF20E132E0A501BC01C6010E9405
:1050C0008C372C960FB6F894DEBF0FBECDBFDF91A4
:1050D000CF911F910F91FF90EF90DF90CF90BF90F5
:1050E000AF9008958F929F92AF92BF92CF92DF922E
:1050F000EF92FF920F931F93CF93DF93CDB7DEB75D
:105100002C970FB6F894DEBF0FBECDBF6C014B01DC
:105110005A019C012F5E3F4F71E0E72EF12C04E015
:10512000A401BE016F5F7F4F0E943837FC01B1863A
:10513000A0861482158216821782F601148A0FEF58
:105140001FEF20E131E0A401BC01C6010E948C37B1
:105150002C960FB6F894DEBF0FBECDBFDF91CF9176
:105160001F910F91FF90EF90DF90CF90BF90AF9085
:105170009F908F9008956F927F928F929F92AF929F
:10518000BF92CF92DF92EF92FF920F931F93CF9334
:10519000DF93CDB7DEB72C970FB6F894DEBF0FBE06
:1051A000CDBF6C013B014A01BA010E941B375C0173
:1051B0008FEFA8168FEFB80629F46DEF7EEF8FEF13
:1051C0009FEF1DC096012F5E3F4F46E0E42EF12C6D
:1051D00002E0A301BE016F5F7F4FC6010E94383716
:1051E00022E0F601248BA58A2B2D3327268B840100
:1051F00028E036E0A301BC01C6010E948C372C9642
:105200000FB6F894DEBF0FBECDBFDF91CF911F91D7
:105210000F91FF90EF90DF90CF90BF90AF909F9055
:105220008F907F906F9008952F923F924F925F9250
:105230006F927F928F929F92AF92BF92CF92DF92A6
:10524000EF92FF920F931F93CF93DF93CDB7DEB70B
:105250002C970FB6F894DEBF0FBECDBF6C011B01BB
:105260002A0149013801BA010E941B375C018FEF06
:10527000A8168FEFB80629F46DEF7EEF8FEF9FEF42
:1052800025C096012F5E3F4FE5E0EE2EF12C02E0A7
:10529000A101BE016F5F7F4FC6010E94383726E033
:1052A000F601248BA58A2B2D3327268B878A292D5F
:1052B0003327208F618E272D3327228F820128E00C
:1052C00035E0A101BC01C6010E948C372C960FB6B7
:1052D000F894DEBF0FBECDBFDF91CF911F910F912C
:1052E000FF90EF90DF90CF90BF90AF909F908F9006
:1052F0007F906F905F904F903F902F9008956F92A6
:105300007F928F929F92AF92BF92CF92DF92EF9255
:10531000FF920F931F93CF93DF93CDB7DEB72C97F8
:105320000FB6F894DEBF0FBECDBF6C013B014A0142
:10533000BA010E941B375C018FEFA8168FEFB806E9
:1053400029F46DEF7EEF8FEF9FEF1DC096012F5E6A
:105350003F4FB4E0EB2EF12C02E0A301BE016F5FE2
:105360007F4FC6010E94383722E0F601248BA58AC0
:105370002B2D3327268B840128E034E0A301BC01C8
:10538000C6010E948C372C960FB6F894DEBF0FBE74
:10539000CDBFDF91CF911F910F91FF90EF90DF90E4
:1053A000CF90BF90AF909F908F907F906F90089517
:1053B0002F923F924F925F926F927F928F929F9225
:1053C000AF92BF92CF92DF92EF92FF920F931F9313
:1053D000CF93DF93CDB7DEB760970FB6F894DEBFFB
:1053E0000FBECDBF5C017E876D87588B4F8749010B
:1053F000380127011601BA010E941B376C018FEF9B
:10540000C8168FEFD80629F46DEF7EEF8FEF9FEF70
:1054100030C095012F5E3F4F53E0E52EF12C02E0A6
:105420004D855E85BE016F5F7F4FC5010E94383795
:105430002AE0F501248BC58A2D2D3327268B878AF8
:10544000292D3327208F618E272D3327228F438EDE
:10545000252D3327248F258E232D3327268F0F8547
:10546000188928E033E04D855E85BC01C5010E94A6
:105470008C3760960FB6F894DEBF0FBECDBFDF91BC
:10548000CF911F910F91FF90EF90DF90CF90BF9041
:10549000AF909F908F907F906F905F904F903F90D4
:1054A0002F9008952F923F924F925F926F927F922A
:1054B0008F929F92AF92BF92CF92DF92EF92FF9224
:1054C0000F931F93CF93DF93CDB7DEB72C970FB613
:1054D000F894DEBF0FBECDBF6C011B012A0149014C
:1054E0003801BA010E941B375C018FEFA8168FEFBD
:1054F000B80629F46DEF7EEF8FEF9FEF25C0960180
:105500002F5E3F4FB1E0EB2EF12C02E0A101BE0176
:105510006F5F7F4FC6010E94383726E0F601248B6B
:10552000A58A2B2D3327268B878A292D3327208F79
:10553000618E272D3327228F820128E031E0A101DF
:10554000BC01C6010E948C372C960FB6F894DEBFC2
:105550000FBECDBFDF91CF911F910F91FF90EF90C4
:10556000DF90CF90BF90AF909F908F907F906F9083
:105570005F904F903F902F900895AF92BF92CF923F
:10558000DF92EF92FF920F931F93CF93DF93CDB7EC
:10559000DEB72C970FB6F894DEBF0FBECDBF6C01FF
:1055A0005B019C012F5E3F4F1EE0E12EF12C02E0DB
:1055B000AB01BE016F5F7F4F0E943837F601148A3E
:1055C0000FEF1FEF28E03EE0A501BC01C6010E94DD
:1055D0008C372C960FB6F894DEBF0FBECDBFDF918F
:1055E000CF911F910F91FF90EF90DF90CF90BF90E0
:1055F000AF9008954F925F926F927F928F929F9299
:10560000AF92BF92CF92DF92EF92FF920F931F93D0
:10561000CF93DF93CDB7DEB72C970FB6F894DEBFEC
:105620000FBECDBF6C012B013A014901BA010E94A6
:105630001B375C018FEFA8168FEFB80629F46DEFCA
:105640007EEF8FEF9FEF21C096012F5E3F4F4DE021
:10565000E42EF12C02E0A201BE016F5F7F4FC60174
:105660000E94383724E0F601248BA58A2B2D33279E
:10567000268B878A292D3327208F830128E03DE060
:10568000A201BC01C6010E948C372C960FB6F8947B
:10569000DEBF0FBECDBFDF91CF911F910F91FF9065
:1056A000EF90DF90CF90BF90AF909F908F907F90C2
:1056B0006F905F904F9008956F927F928F929F921C
:1056C000AF92BF92CF92DF92EF92FF920F931F9310
:1056D000CF93DF93CDB7DEB72C970FB6F894DEBF2C
:1056E0000FBECDBF6C013B014A01BA010E941B37BE
:1056F0005C018FEFA8168FEFB80629F46DEF7EEFEF
:105700008FEF9FEF1DC096012F5E3F4F6CE0E62E9E
:10571000F12C02E0A301BE016F5F7F4FC6010E9422
:10572000383722E0F601248BA58A2B2D3327268BD0
:10573000840128E03CE0A301BC01C6010E948C3733
:105740002C960FB6F894DEBF0FBECDBFDF91CF9180
:105750001F910F91FF90EF90DF90CF90BF90AF908F
:105760009F908F907F906F9008956F927F928F920D
:105770009F92AF92BF92CF92DF92EF92FF920F93E0
:105780001F93CF93DF93CDB7DEB72C970FB6F89466
:10579000DEBF0FBECDBF6C013B014A01BA010E94C2
:1057A0001B375C018FEFA8168FEFB80629F46DEF59
:1057B0007EEF8FEF9FEF1DC096012F5E3F4FE9E018
:1057C000EE2EF12C02E0A301BE016F5F7F4FC601F8
:1057D0000E94383722E0F601248BA58A2B2D33272F
:1057E000268B840128E039E0A301BC01C6010E9498
:1057F0008C372C960FB6F894DEBF0FBECDBFDF916D
:10580000CF911F910F91FF90EF90DF90CF90BF90BD
:10581000AF909F908F907F906F9008956F927F923E
:105820008F929F92AF92BF92CF92DF92EF92FF92B0
:105830000F931F93CF93DF93CDB7DEB72C970FB69F
:10584000F894DEBF0FBECDBF6C013B014A011CE6E0
:10585000A12E13E0B12EA80EB91E9C012F5E3F4F62
:10586000BFE0EB2EF12C02E0AB01BE016F5F7F4F7A
:105870000E9438377C01F50184819581892B39F4A8
:1058800082E090E00E945508F50195838483F5013C
:10589000A481B5818D929C9282E0F601848B858AE9
:1058A000892D9927868B0FEF1FEF28E03FE0A3019A
:1058B000B701C6010E948C372C960FB6F894DEBF54
:1058C0000FBECDBFDF91CF911F910F91FF90EF9051
:1058D000DF90CF90BF90AF909F908F907F906F9010
:1058E00008958F929F92AF92BF92CF92DF92EF92E4
:1058F000FF920F931F93CF93DF93CDB7DEB72C9713
:105900000FB6F894DEBF0FBECDBF6C014B015A013C
:10591000122FBA010E941B378F5F9F4F29F46DEF42
:105920007EEF8FEF9FEF23C096012F5E3F4F0BE07E
:10593000E02EF12C02E0A401BE016F5F7F4FC60193
:105940000E9438377C0187E0F601848BA6014B5E0C
:105950005F4FB501C6010E94BC2DF601138F850172
:1059600028E03BE0A401B701C6010E948C372C96C9
:105970000FB6F894DEBF0FBECDBFDF91CF911F9160
:105980000F91FF90EF90DF90CF90BF90AF909F90DE
:105990008F900895FC01E758FD4F20E030E0DC01D6
:1059A000A757BD4F8189853071F480819181861719
:1059B000970749F48C9182958F708370682F7727B1
:1059C0008827992708952F5F3F4F579677962A305B
:1059D000310541F76DEF7EEF8FEF9FEF0895CF9385
:1059E000DF93FC01E758FD4F20E030E0EC01C557A4
:1059F000DD4F81898530B1F48081918186179707C9
:105A000089F489819A81AA27BB272227382F492F19
:105A10005A2F88819927AA27BB27282B392B4A2B55
:105A20005B2B0BC02F5F3F4F679677962A3031056F
:105A300001F72DEF3EEF4FEF5FEFCA01B901DF91A4
:105A4000CF910895FC01E758FD4F20E030E0DC01E4
:105A5000AB57BD4F8189853051F480819181861784
:105A6000970729F46D917D918D919C9108952F5FF9
:105A70003F4F579677962A30310561F76DEF7EEFED
:105A80008FEF9FEF0895DC01A758BD4F30E020E075
:105A9000FD018189853079F46115710559F0E22F96
:105AA000FF27EE0FFF1FE60FF71F8D919C911197B7
:105AB000918380832F5F3F5F57963A3049F7622F7B
:105AC0007727882799270895CF93DF93DB01FC017F
:105AD000E358FD4F20E030E0AC0147585D4F85852D
:105AE000853009F590818C919817E9F49181ED0149
:105AF00089819817C1F492818A819817A1F49381C2
:105B00008B81981781F494818C81981761F4958129
:105B10008D81981741F4FA01808191819C01B9012E
:105B2000882799270CC02F5F3F4F495E5F4F7796BC
:105B30002A303105A1F66DEF7EEF8FEF9FEFDF91F9
:105B4000CF910895FC01E758FD4F20E08189853011
:105B500051F4808191818617970729F460E070E005
:105B600080E090E008952F5F77962A3079F76DEF07
:105B70007EEF8FEF9FEF0895FC01E758FD4FA0E007
:105B8000B0E09C0123583D4F8189853089F48081A4
:105B900091818617970761F4DA01F90186E0019097
:105BA0000D928150E1F760E070E080E090E00895B0
:105BB0001196295E3F4F7796AA30B10529F76DEF10
:105BC0007EEF8FEF9FEF0895DB01FC01EA59FC4F58
:105BD00086E001900D928150E1F760E070E080E096
:105BE00090E00895CB01089508950895FC01E95DC2
:105BF000FD4F619371933183208376975183408366
:105C00000895FC01ED5BFD4F718360833C975183E8
:105C100040830895FC01EB58FD4F619371935183CC
:105C200040830895FC01EE59FC4F619371935183B9
:105C300040830895AF92BF92CF92DF92EF92FF928E
:105C40000F931F93CF93DF936C01A42EB22EFC0110
:105C5000E758FD4F20E0808191818617970731F04A
:105C60002F5F77962A3009F44BC0F5CF822F992702
:105C700027E130E0829FE001839FD00D929FD00DFD
:105C80001124CC0DDD1DC657DD4F8881CA58D24086
:105C90008530B1F5C601815E9D4F0E946F49FE01BE
:105CA000E257FD4F80818F5F808382E0F701808320
:105CB000FE01E558FD4F8081E701898321818A2D0E
:105CC00099278370907034E0880F991F3A95E1F717
:105CD000282BBB0CBB0CBB0CBB0CBB0CBB0C2B2973
:105CE0002A830B83812F99278C83B701C6010E94D9
:105CF0009C32FC01BF01882777FD8095982F04C056
:105D00006DEF7EEF8FEF9FEFDF91CF911F910F919E
:105D1000FF90EF90DF90CF90BF90AF900895CF921B
:105D2000DF92EF92FF920F931F93CF93DF93EC01DB
:105D30005CE6C52E53E0D52EC80ED91E60E070E09B
:105D40000E948B23F601A085B185109751F0FD01CB
:105D5000E480F580068117812D913D914D915C91F4
:105D60000CC04FEFE42E4FEFF42E4FEB042F4FEF0C
:105D7000142F2FEF3FE140E050E060E070E0CE01F3
:105D80000E94D623F601468157814115510531F015
:105D900060E070E0CE010E94122626C01F921F9282
:105DA00081E08F931F921F92DF93CF930E945D2615
:105DB00082E090E09F938F931F921F9282E08F93D7
:105DC0001F921F92DF93CF930E945D26CE59DC4F26
:105DD00019821882C256D3408DB79EB740960FB62F
:105DE000F8949EBF0FBE8DBFF601A281B3811097BC
:105DF00019F04D915C9102C040E45FE160E070E019
:105E0000CE010E94FE21F601A689B789109719F0EC
:105E10004D915C9102C040E050E260E070E0CE0144
:105E20000E945D21F601A28DB38D109711F04C9167
:105E300001C043E060E070E0CE010E94C520F601A1
:105E4000A285B385109711F04C9101C040E060E04D
:105E500070E0CE010E94BB1FF601A685B7851097A2
:105E600011F04C9101C041E060E070E0CE010E9471
:105E70009E1EF601A089B189109711F04C9101C0C6
:105E800041E060E070E0CE010E94051EF601A481B1
:105E9000B581109739F04D915C9160E070E0CE01D2
:105EA0000E940E2CF601A485B585109769F0FD01BE
:105EB000E580F680038114814D915C91228160E040
:105EC00070E0CE010E94361FF601A289B3891097B7
:105ED00049F02D913D914D915C9160E070E0CE01D3
:105EE0000E941720F601448955894115510529F072
:105EF00060E070E0CE010E948425F601A08DB18D96
:105F0000109731F04C9160E070E0CE010E94F322D6
:105F1000D601ED91FC91309711F0608101C063E0F2
:105F2000CE010E94444860E070E0CE010E947527D7
:105F3000DF91CF911F910F91FF90EF90DF90CF9065
:105F400008958F929F92AF92BF92DF92EF92FF924D
:105F50000F931F93CF93DF93EC01FC01EA5BFD4F9E
:105F600080819181892B09F096C0809104169091CF
:105F7000051691838083EDE0AE2EB12CAC0EBD1ED4
:105F8000C5010E946F497DE6E72E72E0F72EEC0E08
:105F9000FD1EC7010E946F498E01085B1D4FC8019D
:105FA0000E946F49C7010E946149C8010E9461496E
:105FB000FE01EE59FC4F8080918085EF9DE2918338
:105FC00080838A819B810E94451840E052EC61E009
:105FD00070E00E94FE3481E088870E94254ACF58F5
:105FE000DD4F19921882C257D24069E7E62E62E06F
:105FF000F62EEC0EFD1EDD24F70181898823A1F128
:106000008FEF9FEF93838283808191818F5F9F4F7A
:1060100049F1D7014D915C9100E01FEF2FEF3FEF69
:106020006FEF7FEFCE010E945B388C018F5F9F4F37
:1060300081F7F7018189853091F4FE01EB58FD4F1E
:10604000C958DD4F28813981C757D240D7014D91BA
:106050005C910190F081E02D68E083E00995F70103
:1060600011830083F701118AD39487E190E0E80E51
:10607000F91E9AE0D91609F0BFCFCE010E948F2EEB
:10608000CE59DC4F99828882C5010E946149CC516A
:10609000D14019821882DF91CF911F910F91FF900B
:1060A000EF90DF90BF90AF909F908F900895CF9327
:1060B000DF93CDB7DEB72C970FB6F894DEBF0FBED7
:1060C000CDBF4C01AE014D5F5F4FBE016F5F7F4F93
:1060D000C4010E94F8333C01009709F476C0DC014A
:1060E0008C91833009F448C0843021F0823009F06B
:1060F0006CC005C0B301C4010E94DD3C66C0F30161
:106100000281602F77276F707070762F66278181EC
:106110009927682B792BC4010E94FA36F3018183F9
:10612000492F55272281207F242B2283F401E95D0A
:10613000FD4FAB80BC80CD80DE80E980FA80029587
:106140000F70202F237049E252E0840E951E0190BB
:10615000F081E02D06950695AC01B301D4018D9137
:106160009C910995EAEEFFEF8E0E9F1ED4018D9350
:106170009C93EDEEFDEF27C0F301628177276F70EE
:106180007070762F662781819927682B792BC4013F
:106190000E94FA3623E432E0820E931ED401ED9180
:1061A000FC912DEB3DEF820E931E2981AC01B301D2
:1061B000C401099547E352E0840E951ED4018D93E6
:1061C0009C93E9ECFDEF8E0E9F1E21E732E0820EDC
:1061D000931ED4018C91EFE8FDEF8E0E9F1E882355
:1061E00009F440C0840106571D4FAA24BB248DE743
:1061F000C82E82E0D82EC80CD91CB9E8EB2EB2E02C
:10620000FB2EE80CF91CF4018785908918161906F5
:10621000D4F48385948518161906ACF4D8018C91B2
:10622000823089F484E08C93F701408142954F706D
:106230004370B601C4010E942346F401EF58FD4F9C
:106240008081815080830894A11CB11C27E130E03B
:10625000E20EF31EC20ED31E095E1F4F3AE0A316D4
:10626000B10489F642E752E0840E951ED4018C9168
:10627000EEE8FDEF8E0E9F1E882309F451C0A9E7BA
:10628000EA2EA2E0FA2EE80CF91CAA24BB24FDE7B2
:10629000CF2EF2E0DF2EC80CD91CF401878590893F
:1062A000181619067CF5838594851816190654F579
:1062B000F7018689882331F584E090E09A83898309
:1062C000DE011796F60186E001900D928150E1F70C
:1062D000D7016D917C9108EA14E02981AE01495FF4
:1062E0005F4FC4010E94F744611571058105910556
:1062F00049F483E0F701868BF401EE58FD4F80816D
:10630000815080830894A11CB11C27E130E0C20EAB
:10631000D31EE20EF31E3AE0A316B10409F0BDCF7E
:106320000E943D08CFCE0F931F938B01BA0141E02D
:1063300050E00E942325C8011F910F9108950F93EB
:106340001F93CF93DF938C0188E893E00E9441096B
:10635000009719F4C0E0D0E053C0EC011983088322
:1063600060E070E0815E9D4F0E94864960E070E0D1
:10637000CE01825C9D4F0E94864961E070E0CE01B3
:10638000885B9D4F0E948649CE010E94323581E094
:1063900090E090931E1680931D16CE010E94A638A1
:1063A000C95DDD4F83E991E389939993198218823E
:1063B000669719821882E09682EF9DE2998388831E
:1063C0002C9719821882EE9684EF9DE28993999317
:1063D00019821882C757D24020E034E0AE0167E549
:1063E00070E38DEA94E00E94340BCE010E948F2E60
:1063F000AE014A595C4F60E070E0CE010E942F2749
:10640000CE01DF91CF911F910F91089504960E94C4
:106410006149089504960E946F490895AF92BF9212
:10642000CF92DF92EF92FF920F931F93CF93DF9360
:10643000CDB7DEB763970FB6F894DEBF0FBECDBF02
:106440005C017B016A01DE011196E5EBF4E083E17A
:1064500001900D928150E1F78091A714882341F0BB
:1064600080ED90E09F938F930E949B740F900F900C
:1064700000E010E011C0C5010E944518A601401BB4
:10648000510BB701600F711F0E94131A2FEF8F3F3E
:10649000920781F1080F191F0C151D0560F38091FB
:1064A000A714882301F100E010E012C0F7018191E8
:1064B0007F0199279F938F9389EC90E09F938F930F
:1064C0000E949B740F5F1F4F0F900F900F900F90C3
:1064D0000C151D0559F787EC90E09F938F930E9450
:1064E0009B740F900F90C5010E94C5718F5F9F4FE5
:1064F00051F406C0BE016F5F7F4F8BE00E94455391
:106500008FEF9FEF02C080E090E063960FB6F894A3
:10651000DEBF0FBECDBFDF91CF911F910F91FF90D6
:10652000EF90DF90CF90BF90AF900895FC018281F3
:1065300093810E940E320895EF92FF920F931F9362
:10654000CF93DF937C018B01FB014081423029F125
:10655000433020F4413009F04BC006C0433041F1D4
:10656000443009F045C02AC0FB018381C82FDD27D4
:1065700023969281892F86958695833021F5892FE0
:106580009927982F882721813327822B932B93706B
:106590000397C9F4F701408716C0FB01848199274E
:1065A000D82FCC2783819927C82BD92B24960BC0B1
:1065B000FB018381C82FDD27239605C0FB01828163
:1065C000C82FDD272296C7010E940A322196AE010C
:1065D000B801C7010E9496328C01C7010E940632A1
:1065E0008FEFF701818B17FD03C080E090E002C0C0
:1065F0008FEF9FEFDF91CF911F910F91FF90EF9061
:1066000008954F925F926F927F928F929F92AF9276
:10661000BF92CF92DF92EF92FF920F931F93CF938F
:10662000DF93CDB7DEB7C954D0400FB6F894DEBFC4
:106630000FBECDBF3C012B015A01FC01E280F3806B
:10664000DE019296E8ECF4E082E101900D92815037
:10665000E1F7DE015396EAEDF4E08FE001900D9250
:106660008150E1F7DE01D496E9EEF4E086E1019095
:106670000D928150E1F7DE011596EFEFF4E08EE028
:1066800001900D928150E1F7CC24DD2462C0C70156
:106690000E944518A5014C195D09B2016C0D7D1DC4
:1066A0000E944E724C018F5F9F4F09F45DC0C7017D
:1066B0000E9445188E010F5F1F4FA8016AE071E02C
:1066C0000E94A919F3018085882369F087E090E092
:1066D000A0E0B0E089839A83AB83BC83C7010E94AA
:1066E0004518A80130C029813A814B815C81DA01CB
:1066F000C90187709070A070B0700097A105B105B6
:1067000031F120FF04C0BE016D5E7F4F0BC021FF41
:1067100004C0BE016C5C7F4F05C022FF06C0BE01F5
:106720006B5F7F4F8BE00E94455387E090E0A0E0D5
:10673000B0E089839A83AB83BC83C7010E9445186C
:10674000AE014F5F5F4F69E071E00E94A919C80C6C
:10675000D91CCA14DB0408F49ACF8091A7148823AB
:1067600061F480E090E02CC0BE016E5D7F4F8BE055
:106770000E9445538FEF9FEF23C000E010E07201AD
:1067800012C0F70181917F0199279F938F9384ED28
:1067900090E09F938F930E949B740F5F1F4F0F9009
:1067A0000F900F900F900A151B0559F782ED90E09E
:1067B0009F938F930E949B7480E090E00F900F90C6
:1067C000C75BDF4F0FB6F894DEBF0FBECDBFDF91C2
:1067D000CF911F910F91FF90EF90DF90CF90BF90DE
:1067E000AF909F908F907F906F905F904F900895A3
:1067F000CF92DF92EF92FF920F931F93CF93DF938D
:10680000CDB7DEB7A1970FB6F894DEBF0FBECDBFF0
:106810007C016B018A01FC0182819381DE01129669
:10682000EDE0F5E020E201900D922150E1F70E94A9
:10683000451841E050E0BE016F5F7F4F0E944E72ED
:10684000019709F0C9C08091A714882371F089814C
:1068500099279F938F9380EC90E09F938F930E9452
:106860009B740F900F900F900F9089818330C1F12E
:10687000843009F45FC0823009F096C00E946E0532
:10688000F801608371838283938323E132E0E20E17
:10689000F31EF701008111812DEE3DEFE20EF31E94
:1068A0008981F801819344E050E0BF01C7010E9453
:1068B0000133892B09F090C0F80184819927582F62
:1068C000442783819927482B592BF6015183408314
:1068D0004115510509F473C0B8016B5F7F4F23C0A8
:1068E00027E332E0E20EF31EF7010081118129EC6B
:1068F0003DEFE20EF31EF801819343E050E0BF014B
:10690000C7010E940133892B09F066C0F801838119
:10691000482F5527F60151834083882309F44FC03F
:10692000B8016C5F7F4FC7010E940133892B09F4C6
:1069300046C052C087010F5E1E4FF801819342E0AE
:1069400050E0BF01C7010E940133892B09F044C008
:10695000F8018281482F5527F6015183408388230F
:1069600041F0B8016D5F7F4FC7010E940133892B51
:1069700099F5F7018085882311F1F80181818E3026
:10698000F1F49581892F86958695C9F4892F9927E9
:10699000982F882724813327822B932B9370892B60
:1069A00071F4F70110860BC0F70180858823A1F4EC
:1069B000BE016E5F7F4F8CE00E9445530DC08091F9
:1069C000A714882359F08EEB90E09F938F930E9439
:1069D0009B740F900F9002C000E010E0C801A196D8
:1069E0000FB6F894DEBF0FBECDBFDF91CF911F91E0
:1069F0000F91FF90EF90DF90CF9008950F931F932A
:106A0000CF93DF93CDB7DEB724970FB6F894DEBFF0
:106A10000FBECDBF8C0149835A836B837C8340E0DA
:106A200050E060E070E00E94131A84E60E94C80BF8
:106A3000AE014F5F5F4F61E071E0C8010E94A9198C
:106A4000892B19F08FEF9FEF02C080E090E0249631
:106A50000FB6F894DEBF0FBECDBFDF91CF911F916F
:106A60000F9108952F923F924F925F926F927F9273
:106A70008F929F92AF92BF92CF92DF92EF92FF924E
:106A80000F931F93CF93DF93CDB7DEB724970FB645
:106A9000F894DEBF0FBECDBF2C0161E070E004961C
:106AA0000E94864940E060E070E0F20180819181BF
:106AB0000E941904892B09F01BC1F2018081918188
:106AC0006DE275E002960E944918F2019383828379
:106AD0000E944518181619060CF00AC1F2018281AD
:106AE00093810E94451840E052EC61E070E00E9402
:106AF000FE34892B09F0FCC019821A821B821C8289
:106B0000F201828193810E9445181E010894211C84
:106B1000311CA10165E071E00E94A919892B09F0DF
:106B2000E7C088E090E0A0E0B0E089839A83AB837F
:106B3000BC83F201828193810E944518A10163E028
:106B400071E00E94A919892B09F0D2C081E090E080
:106B5000A0E0B0E089839A83AB83BC83F201828199
:106B600093810E944518A10167E071E00E94A91974
:106B7000892B09F0BDC019821A821B821C82F20186
:106B8000828193810E944518A10163E171E00E9416
:106B9000A919892B09F0ACC083E090E0A0E0B0E037
:106BA00089839A83AB83BC83F201828193810E94A3
:106BB0004518A10161E171E00E94A919892B09F032
:106BC00097C0F2011086828193810E94451840E0AF
:106BD00050E060E070E00E944E7280E092E0A0E041
:106BE000B0E089839A83AB83BC83F2018281938175
:106BF0000E944518A1016BE171E00E94A9193C01B6
:106C0000882477FC8094982CF201828193810E94E1
:106C10004518A1016DE171E00E94A919AA2797FD0D
:106C2000A095BA2F680E791E8A1E9B1E84EF91E0F4
:106C3000A0E0B0E089839A83AB83BC83F2018281B8
:106C400093810E944518A10162E271E00E94A91996
:106C50007C01F201828193810E944518A10166E2C4
:106C600071E00E94A9195C01CC24B7FCC094DC2C13
:106C70000027F7FC0095102FAE0CBF1CC01ED11EC4
:106C800082EC91E0A0E0B0E089839A83AB83BC837F
:106C9000F201828193810E944518A10160E271E0B6
:106CA0000E94A919AA2797FDA095BA2F680E791EF0
:106CB0008A1E9B1EF201828193810E944518A101C8
:106CC00064E271E00E94A919AA2797FDA095BA2F46
:106CD000A80EB91ECA1EDB1E6A0C7B1C8C1C9D1CD8
:106CE000611471048104910419F480E090E002C001
:106CF0008FEF9EEF24960FB6F894DEBF0FBECDBF88
:106D0000DF91CF911F910F91FF90EF90DF90CF9087
:106D1000BF90AF909F908F907F906F905F904F90BB
:106D20003F902F9008950895CF93DF93FC01E45B8B
:106D3000FD4F20E030E0EC01C459DD4FDF018081E0
:106D40009181009731F46D937C93288380E090E0EB
:106D50000FC08617970719F48EEF9FEF09C02F5FBA
:106D60003F4F129632962031310549F78FEF9FEF52
:106D7000DF91CF910895DC01A45BBD4F20E0ED9140
:106D8000FC911197309751F0808191818617970778
:106D900029F4828193818417950731F02F5F129631
:106DA000203169F7E0E0F0E0CF010895DC01A6575B
:106DB000BD4F20E030E04FEF5FEFFC01E758FD4FA3
:106DC0008C91882361F481E0818B8089806F808B36
:106DD0005183408353834283158A168A09C02F5FEB
:106DE0003F4F779657962A30310551F72FEF3FEFF7
:106DF000C90108952FEF6F3F7207D1F0FC01E558EC
:106E0000FD4F20E030E0DC01A758BD4F878585307D
:106E100041F4808191818617970719F48D919C9197
:106E200008952F5F3F4F579677962A30310571F7B7
:106E30008FEF9FEF0895FC01E758FD4F20E030E011
:106E4000DC01A558BD4F8189853041F48081918155
:106E50008617970719F48D919C9108952F5F3F4FE6
:106E6000579677962A30310571F78FEF9FEF089587
:106E70008F929F92AF92BF92CF92DF92EF92FF924A
:106E80000F93CF93DF93EC014B015A016901CA5B69
:106E9000DD4F28813981C654D2402115310539F0A2
:106EA00080910416909105162817390721F0CE011C
:106EB0000D960E946F49033021F485E3E816F10432
:106EC00021F0CE0109960E946F4981E0F60180838E
:106ED000000F000F0283E182A114B10409F0450103
:106EE000C401DF91CF910F91FF90EF90DF90CF9091
:106EF000BF90AF909F908F9008959C01FC01E45942
:106F0000FD4F80818F3F39F08FEF8083C901835916
:106F10009D4F0E94614908958F929F92AF92BF92B8
:106F2000CF92DF92EF92FF920F931F93CF93DF9355
:106F3000EC017B014A016901672B99F18DE6A82ECE
:106F400082E0B82EAC0EBD1EC5010E946F49F7014C
:106F5000D182C0821383028313861286B701CE01C9
:106F60000E9494360097E9F0FFEF8F3F9F0739F4B6
:106F700068EE73E080E090E00E947B06EFCF8E5FCA
:106F80009F4F61F7CE010E949336C5010E9461496F
:106F9000CE010D960E94614960E07FEF8FEF9FEF79
:106FA0003BC0BE016F5E7F4FCE010E949C328C01C0
:106FB000CA5BDD4F28813981C654D2402115310585
:106FC00039F080910416909105162817390721F0A1
:106FD000CE010D960E9461490115110531F0B801ED
:106FE000882777FD8095982F17C0E114F10481F070
:106FF000892871F440E050E060E070E0C7010A9633
:107000000E946D0AF701648175818681978104C0B1
:1070100060E070E080E090E0DF91CF911F910F91F0
:10702000FF90EF90DF90CF90BF90AF909F908F90A8
:107030000895FF920F931F93CF93DF93EC01F62EE9
:10704000062F1127000F111F0C0F1D1F045B1D4F72
:10705000D801ED91FC912483358346835783CF017A
:107060000A960E94DA09D801ED91FC9111978FEFF1
:107070009FEF938782871D921C92C459DD4F8881B0
:10708000CC56D2408F1519F4CE010E947D37DF9186
:10709000CF911F910F91FF900895FC019A01AB01D0
:1070A000E459FD4F6081EC56F2406F3F19F0CF017B
:1070B0000E94193808956F927F928F929F92AF929B
:1070C000BF92CF92DF92EF92FF920F931F93CF93D5
:1070D000DF934C015B013A0168017901EC01C45B6B
:1070E000DD4F2FEF3FEF00E010E0E881F9813097AE
:1070F000B9F0828193818615970591F48FEFA816D8
:107100008FEFB80629F0808191818A159B0541F4A3
:10711000A7019601602FC4010E94193820E030E0D9
:107120000F5F1F4F229600311105F9F6C901DF915B
:10713000CF911F910F91FF90EF90DF90CF90BF9074
:10714000AF909F908F907F906F9008951F93CF93F3
:10715000DF93EC011FEF198B61E070E009960E944C
:107160008649CF5EDE4F1883C151D140FE01E45BFA
:10717000FD4F80E0119211928F5F8031D9F7DE01CF
:10718000A758BD4F20E030E04FEF5FEFBE016757DB
:107190007D4FFD01118A11965C934E935383428378
:1071A000FB0180818F7C80832F5F3F4F695E7F4F23
:1071B00057962A30310569F7CF58DD4F1882C157ED
:1071C000D24061E070E0CE010D960E94864960E0F9
:1071D00070E0CE0183599D4F0E948649CE010E94E6
:1071E0007D37FE01ED5EFD4FC75EDD4FD183C0836D
:1071F000C951D240CE01875C9D4FC95CDD4F998358
:107200008883DF91CF911F9108950F931F93CF93A0
:10721000DF93EC018B01FB014381442319F40E94AD
:107220007D370AC05527509541955F4F662757FD1A
:107230006095762F0E944D38F80164817727CE0142
:1072400009960E945449DF91CF911F910F910895A3
:107250003F924F925F926F927F928F929F92AF92E6
:10726000BF92CF92DF92EF92FF920F931F93CF9333
:10727000DF93CDB7DEB726970FB6F894DEBF0FBE0B
:10728000CDBF5C017B01FB0133968281382E3694A1
:1072900036949927D82ECC2481819927C82AD92AB7
:1072A0008FEF93E0C822D92293E0391609F4CCC0BD
:1072B000931538F0A1E03A1681F0A31508F455C0F3
:1072C00021C3B5E03B1609F463C23B1608F4AAC11A
:1072D000EFE33E1609F0FDC2E5C2FCE0CF16D10493
:1072E00009F43FC03DE0C316D10439F182E0C8166D
:1072F000D10409F0EEC218E4812E12E0912E8A0C1E
:107300009B1CC4010E940B494FEF5FEF64E071E0EA
:10731000C5010E94BB36FC01892B59F004811581FF
:10732000268137814FEF5FEF64E071E0C5010E9475
:107330005B38C4010E946149CCC24FEF5FEF64E04B
:107340007DE0C5010E94BB3620E030E0DE011196F1
:10735000F701379681918D932F5F3F4F263031058E
:10736000C9F7C5010E947D37B4C29DE0C916D1049A
:1073700009F440C0AEE0CA16D10450F4B9E0CB160F
:10738000D10481F0ECE0CE16D10409F0A2C219C0FC
:10739000FEE0CF16D104E9F13FE0C316D10409F0B5
:1073A00098C24BC0FB0180859927582E44248781C1
:1073B0009927482A592A8185682E77248824992478
:1073C0009FC2FB0180859927582E442487819927E5
:1073D000482A592A8681882309F0CAC282859927BA
:1073E000982F882721853327822B932B3C018824D3
:1073F0009924C2C2FB0180859927582E4424878195
:107400009927482A592A86819927909581959F4FD7
:10741000AEC0FB018681882309F0A7C28085992729
:10742000982F882727813327822B932B3C01882490
:1074300099244FEF442E542E9FC2FB018681992739
:10744000909581959F4F72C0F7E1CF16D10409F452
:1074500064C038E1C316D104D0F489E0C816D10461
:1074600009F48BC09AE0C916D10430F4A3E0CA161F
:10747000D10409F02EC229C0B4E1CB16D10409F41D
:1074800083C0E5E1CE16D10409F023C246C0F6E37D
:10749000CF16D10409F45AC037E3C316D10458F407
:1074A00089E1C816D10409F468C093E2C916D10471
:1074B00009F00FC215C0A7E3CA16D104E9F1B4E47C
:1074C000CB16D10409F005C228C0E5E4F2E0AE0E07
:1074D000BF1ED5011C92EBEBFDEFAE0EBF1EF9C136
:1074E000FB0180859927AA27BB276624782E892E41
:1074F0009A2E81859927AA27BB27DC0199278827FF
:107500002781332744275527822B932BA42BB52B78
:10751000682A792A8A2A9B2ADFC1F7018085992760
:10752000982F882727813327822B932B3C0188248F
:1075300077FC8094982CD0C1FB0180859927582E28
:10754000442487819927482A592AD7C1FB0180857D
:107550009927582E442487819927482A592A8285B9
:107560009927982F882721853327822B932B3C013D
:10757000882477FC8094982CC3C1F7018781682EFA
:10758000772488249924A8C14FEF5FEF6CE074E161
:10759000C5010E94BB369C01FC01008511858481D8
:1075A0009581A681B781893F9105A105B10544F078
:1075B00088EF90E0A0E0B0E084839583A683B78352
:1075C0006624772410C0492C5524D201AE0DBF1D6E
:1075D000FD018781400E511ED2018C930894611CDD
:1075E000711C882379F0962C462D5527662777271E
:1075F000F90184819581A681B781481759076A07E7
:107600007B070CF3F90184819581A681B781481726
:1076100059076A077B0709F49A94090D111DD801CF
:107620001C9257C1B3E0CB16D10409F44AC0E4E080
:10763000CE16D10430F4F1E0CF16D10409F049C1DF
:107640000BC035E0C316D10409F452C089E0C81656
:10765000D10409F03EC185C04FEF5FEF60E171E0FA
:10766000C5010E94BB36FC01A085B185F701878169
:107670008C932085332781859927982F8827282B5D
:10768000392BFD0132832183F7018285FD0183833C
:10769000F7012385332784859927982F8827282B5E
:1076A000392BFD0135832483F70125853327868512
:1076B0009927982F8827282B392BFD01378326837C
:1076C00008C14FEF5FEF60E173E0C5010E94BB3678
:1076D000FC0140855185D70114969A01285F3F4FE0
:1076E0008D91FA018193AF01E217F307C9F7F1C059
:1076F00083E292E0A80EB91EFB0180859927982F9E
:10770000882727813327822B932BD5018D939C9338
:10771000EFE1F0E0AE0EBF1EF7018185D5018C933D
:10772000EEEBFDEFAE0EBF1EF70163857727762FD8
:10773000662782859927682B792BC501815E9D4F2D
:107740000E945449F70165857727762F662784853F
:107750009927682B792BC501825C9D4F0E94544963
:10776000B8C04FEF5FEF60E179E0C5010E94BB3622
:10777000FC0140855185D70117969A012A5F3F4F3A
:107780008D91FA018193AF01E217F307C9F7A1C008
:10779000F5E0CF16D10419F137E0C316D10409F48E
:1077A00040C083E0C816D10409F0ACC0FB0180855D
:1077B0009927582E442487819927482A592AB201AB
:1077C000C5010E94FA36AC0164E173E0C5010E9474
:1077D000BB36FC01A085B185F70181858DC0FB0119
:1077E00080859927582E442487819927482A592A29
:1077F000B201C5010E94FA36AC0164E175E0C50131
:107800000E94BB36FC01A085B185F70182859927CE
:10781000982F882721853327822B932B8D939C9338
:107820006CC04FEF5FEF64E177E0C5010E94BB36AB
:10783000FC01A085B185109729F0F701858599276E
:107840008D939C93F70182859927AA27BB276624ED
:10785000782E892E9A2E2485332744275527522F98
:1078600044273327222783859927AA27BB27DC01B2
:1078700099278827282B392B4A2B5B2B8185992721
:10788000AA27BB27282B392B4A2B5B2B622A732A6A
:10789000842A952A62E0660C771C881C991C6A95DC
:1078A000D1F71AC0F2E1CF16D10499F4F501E45BE7
:1078B000FD4F20E0008111810115110531F0D80143
:1078C0008D919C918C5F924159F02F5F32962031BF
:1078D00089F76624772443015FEF452E552E10C0AB
:1078E000F80162817381C5010E941B372C01F801E8
:1078F000A085B185F70187818C93662477244301A5
:1079000011E007C06624772443014FEF442E542E24
:1079100010E0F7018681882349F099279095819599
:107920009F4F3C01882477FC8094982CFFEF4F16E2
:10793000FFEF5F0619F44FEF5FEF05C0B201C5011D
:107940000E94FA36AC011123C9F07C2D6627832DE5
:107950009927880F991F880F991F682B792B9401FD
:107960008301C5010E945B3809C08FEF482E582E55
:10797000F701868111E0D1CF11E0D8CFF701638103
:107980007727C50109960E94544926960FB6F894A8
:10799000DEBF0FBECDBFDF91CF911F910F91FF9042
:1079A000EF90DF90CF90BF90AF909F908F907F909F
:1079B0006F905F904F903F9008952F923F924F921B
:1079C0005F926F927F928F929F92AF92BF92CF926F
:1079D000DF92EF92FF920F931F93CF93DF93CDB778
:1079E000DEB72A970FB6F894DEBF0FBECDBF6C018D
:1079F0004B01FB018181833109F459C0843128F5A1
:107A0000853009F427C3863078F4823009F489C0C0
:107A1000833020F4813009F040C057C0833009F42E
:107A2000AEC18430D1F57EC28F3009F4FBC3803102
:107A300030F4873009F48AC38E3079F5EFC3803192
:107A400009F4DEC5823149F536C08B3109F4D8C559
:107A50008C3170F4863109F41CC5873118F48431F7
:107A6000E1F41FC0873109F424C58831B1F4C8C5D9
:107A7000823209F456C0833230F48C3109F429C5BE
:107A80008D3159F44CC58F3E19F08F3F31F419C038
:107A90008B0181E0E82EF12C8BC58401EE24FF24BC
:107AA00098C5D601A558BD4F60E070E086C48B0133
:107AB000EE24FF247BC4D601A358BD4F20E030E064
:107AC000B5C38B01EE24FF2462C5FB0103810023B3
:107AD00079F01127109501951F4F222717FD20954A
:107AE000322F4FEF5FEF64E071E0C6010E945B3818
:107AF0004FEF5FEF64E071E0C6010E94BB36FC010E
:107B000004811581268137814FEF5FEF64E071E0DA
:107B1000C6010E945B38C601885B9D4F0E94614987
:107B20006FC54FEF5FEF64E071E0C6010E94BB36A6
:107B30008C01FC01E084F184B401AA24BB241886E2
:107B40001F82B1E12B2E312C280C391C02C1F80107
:107B5000848195818A0D9B1D2FE030E0829FD001AA
:107B6000839FB00D929FB00D1124EF81F885E80D31
:107B7000F91DAE0DBF1D349686E001900D92815027
:107B8000E1F7F801848195818A0D9B1DAFE06A2E93
:107B9000712C869DD001879DB00D969DB00D11244E
:107BA000AE0DBF1DFB0192859F70FD018681807F18
:107BB000892B8683F801848195818A0D9B1D869D82
:107BC000D001879DB00D969DB00D1124AE0DBF1D47
:107BD000FB0193859295907FFD0186818F70892BA3
:107BE0008683F4018181F80144815581FB019585EB
:107BF0005684823209F052C04A0D5B1D469D9001A9
:107C0000479D300D569D300D11242E0D3F1D3A8796
:107C100029872485332744275527892F9927AA2781
:107C2000BB27BA2FA92F982F8827282B392B4A2B0F
:107C30005B2B852D9927AA27BB27DC01992788274D
:107C4000282B392B4A2B5B2BE985FA852783308734
:107C500041875287F801848195818A0D9B1D869DFD
:107C6000D001879DB00D969DB00D1124AE0DBF1DA6
:107C7000FB0120893327322F222787859927906897
:107C8000282B392BFD0134872387F1018081992727
:107C900087FD9095FD01968785874CC04A0D5B1D39
:107CA000469D9001479D300D569D300D11242E0D9F
:107CB0003F1D3A872987292F332744275527852DAC
:107CC0009927AA27BB27BA2FA92F982F8827282BB7
:107CD000392B4A2B5B2BFB0187859927AA27BB27CA
:107CE000DC0199278827282B392B4A2B5B2BE98528
:107CF000FA852783308741875287F80184819581EF
:107D00008A0D9B1D869DD001879DB00D969DB00D5F
:107D10001124AE0DBF1DFB0121893327322F2227ED
:107D2000808999279068282B392BFD013487238778
:107D3000168615860894A11CB11C2F813885225FF8
:107D40003F4F38872F838EE090E0280E391E625F08
:107D50007F4FF4012381822F9927A816B9060CF4CE
:107D6000F6CEF80184819581A681B781820F911D9D
:107D7000A11DB11D84839583A683B78341C48B0164
:107D80000A5F1F4FDE011196F80186E001900D9207
:107D90008150E1F7A9817A816B815C814D819E815F
:107DA000F601E358FD4F20E030E08585882391F00F
:107DB00080818A1779F48181871761F4828186171F
:107DC00049F48381851731F48481841719F48581FE
:107DD000891739F02F5F3F4F77962A30310529F701
:107DE00001C487E190E0289FD001299FB00D389F02
:107DF000B00D1124A758BD4FAC0DBD1DED90FC90EA
:107E0000119734C0C6010E94D6369C0197FDF8C375
:107E100087E190E0289FD001299FB00D389FB00DD9
:107E20001124A758BD4FAC0DBD1DCD010496A8016E
:107E300026E0FA010190AF01FC010192CF0121502F
:107E4000C1F784E0FD01818B80911D1690911E1673
:107E500011969C938E93019690931E1680931D16F7
:107E6000019720892F7C2061208B7C01FD01718985
:107E7000872F8350F4019381823008F045C0992305
:107E800061F0FD01118A8FEF9FEF8D939C93938397
:107E90008283F4018381992739C085E0FD01818BBC
:107EA000F4012481332785819927982F8827282B4F
:107EB000392BFD0133832283F40194859F70FD01EA
:107EC0008089807F892B808B128A86010B581D4FF9
:107ED00027E732E0C20ED31EF6012081318189E806
:107EE0009DEFC80ED91E4D915C9160E0733009F48E
:107EF00061E081E06827D801ED91FC9182E009956D
:107F00008701222733270AC0892F992790958195C9
:107F10009F4F8C01222717FD2095322FA70164E087
:107F200075E004C1E2E6F3E0CE0EDF1ED6018D91CE
:107F30009C91EEE9FCEFCE0EDF1E892B09F460C3A5
:107F40008B010D5F1F4FDE011196F80186E0019055
:107F50000D928150E1F7F401E184F284B384C6010B
:107F60000E94D636AC018F5F9F4F09F449C387E169
:107F700090E0489FD001499FB00D589FB00D11244B
:107F8000A358BD4FAC0DBD1DC80126E0FC010190FA
:107F9000CF010D922150D1F787E190E0489F300149
:107FA000499F700C589F700C11246C0C7D1C25E8A7
:107FB00032E0620E731E2E2D3327442755278F2D56
:107FC0009927AA27BB27BA2FA92F982F8827282BB4
:107FD000392B4A2B5B2B8B2D9927AA27BB27DC013A
:107FE00099278827282B392B4A2B5B2BD3012D93DC
:107FF0003D934D935C931397EBE7FDEF6E0E7F1E61
:10800000D301A757BD4FF40194859F708C91807F59
:10801000892B8C9380911D1690911E1629E732E0D2
:10802000620E731EF30191838083019690931E1656
:1080300080931D1621E130E0620E731E82E0F30191
:1080400081938C918F7C80618C931082F601EF5824
:10805000FD4F2BC2FB0185819927582F442784812E
:108060009927482B592BD601A558BD4F60E070E0E9
:10807000E9E7AE2EE2E0BE2EAC0CBD1C9501FD0181
:108080008785882371F08D919C91119784179507AE
:1080900041F4D901ED90FC90F4010381002371F0CB
:1080A00049C06F5F7F4F87E190E0A80EB91E295E3F
:1080B0003F4F57966A30710511F7A2C2F501118A38
:1080C0008FEF9FEF938382839183808380898F7C5E
:1080D000808BF601EB58FD4F27E732E0C20ED31E2E
:1080E000D6012D913C9189E89DEFC80ED91EA08143
:1080F000B181A701F401668183E0FD010995F401D6
:1081000003811127109501951F4F222717FD2095F8
:10811000322FA70164E076E0C6010E945B3806EFCB
:108120001EEF2FEF3FEFA7016FEF7FEFC6010E9419
:108130005B3866C21127109501951F4F222717FD46
:108140002095322FA70164E076E0F0CF4FEF5FEF8C
:1081500064E079E1C6010E94BB367C01FC014084E9
:10816000518484819581A681B781893F9105A105BC
:10817000B10544F088EF90E0A0E0B0E084839583FF
:10818000A683B783540100E010E020E030E011C086
:10819000F5018285F201E40FF51F80838A019B01BE
:1081A0000F5F1F4F2F4F3F4F0894A11CB11C882316
:1081B00069F03801B901A801F70184819581A68190
:1081C000B781481759076A077B0714F3F7018481C1
:1081D0009581A681B781481759076A077B0719F46B
:1081E000089461087108460C571CD2011C92F401D6
:1081F0000381002349F01127109501951F4F222775
:1082000017FD2095322F05C08301222717FD2095E9
:10821000322F4FEF5FEF64E079E188CFC6010E9413
:108220002839EEC1C6010E940539EAC1A4014D5F9B
:108230005F4F9C91FA0181819817F1F4FD019181C2
:10824000FA0182819817C1F4FD019281FA018381BC
:10825000981791F4FD019381FA018481981761F4D4
:10826000FD019481FA018581981731F4FD01958112
:10827000FA018681981739F02F5F3F4F57962A30C1
:108280003105A1F6BDC187E190E0289F7001299FCB
:10829000F00C389FF00C1124EC0CFD1C29E732E0A7
:1082A000E20EF31ED701AD90BC90E7E8FDEFEE0EB5
:1082B000FF1EF4010381002351F011271095019551
:1082C0001F4F222717FD2095322FA501ABC0D701E4
:1082D000A757BD4FF401928593709295907F8C9132
:1082E0008F7C892B8C930285112722273327A501A8
:1082F00068E07BE0C6010E945B382AE832E0E20ECB
:10830000F31ED7018C91853009F07AC1F601EB5844
:10831000FD4F27E732E0C20ED31ED6012D913C91CE
:1083200089E89DEFC80ED91EA081B181A50160E04A
:10833000F4018285FD01099563C1F8016781772702
:10834000762F662786819927682B792BC601815E57
:108350009D4F0E944549F80185819927382F222792
:1083600084819927282B392BD601A558BD4F40E091
:1083700050E0B60162577D4F8D919C911197821705
:10838000930739F4F8019681DB018C91891B8C935A
:1083900008C04F5F5F4F695E7F4F57964A30510567
:1083A00059F70894E11CF11C0C5F1F4FF401838105
:1083B0009927E816F9060CF223C18D919C9111972B
:1083C0005796F40125813327322F222744815527E0
:1083D000242B352B3F708217930731F06F5F7F4F4F
:1083E0006A30710551F70CC187E190E0689FD001B8
:1083F000699FB00D789FB00D1124AC0DBD1DA7581D
:10840000BD4F4D915C911197A957B240F401038182
:10841000002359F01127109501951F4F222717FDB2
:108420002095322F68E07BE081CEA557BD4FF40147
:1084300086818D938681882359F080859927982F8E
:10844000882727813327822B932B8D939C9302C0FF
:108450001D921C9287E190E0689FF001699FF00DEA
:10846000789FF00D1124EC0DFD1DE457FD4F0081A8
:10847000118122273327322F212F102F0027F401BB
:1084800086819927AA27BB27082B192B2A2B3B2B40
:108490004BCEDE011196FB01339686E001900D92E2
:1084A0008150E1F7F601EE58FD4F80818F5F8083A8
:1084B000A7C0DE011196FB01339686E001900D9274
:1084C0008150E1F7BE016F5F7F4FC6010E946A4590
:1084D00097C0FB0165817727762F662784819927CE
:1084E000682B792BC6010E94FA36AC01F401038196
:1084F000002329F01127109501951F4F09C0F401A1
:1085000007811127102F002786819927082B192B07
:10851000222717FD2095322F64E07FE107CEFB0173
:1085200065817727762F662784819927682B792B99
:10853000C6010E94FA36AC01F4010381002329F040
:108540001127109501951F4F09C0F40107811127CC
:10855000102F002786819927082B192B222717FD1A
:108560002095322F64E07FE0E1CDF80182819927E8
:108570009F938F9380E395E09F938F930E941019B0
:108580000894E11CF11C0F900F900F900F900F5F5B
:108590001F4FF40182819927E816F90634F330C0A1
:1085A000F801838199270E94F4710894E11CF11C61
:1085B0000F5F1F4FF40182819927E816F90684F3B3
:1085C0001FC0F801828199270E94F4710894E11C70
:1085D000F11C0F5F1F4FF40182819927E816F906FD
:1085E00084F30EC0E2E6F3E0CE0EDF1ED6018D91DD
:1085F0009C91EEE9FCEFCE0EDF1E892B09F402CC34
:1086000021E131E0C20ED31E8FEFD6018C932A9662
:108610000FB6F894DEBF0FBECDBFDF91CF911F9193
:108620000F91FF90EF90DF90CF90BF90AF909F9011
:108630008F907F906F905F904F903F902F90089514
:108640006F927F928F929F92AF92BF92CF92DF9262
:10865000EF92FF920F931F93CF93DF93CDB7DEB7C7
:108660002C970FB6F894DEBF0FBECDBF6C014B0147
:108670003A01BA010E941B375C018FEFA8168FEFF9
:10868000B80629F46DEF7EEF8FEF9FEF1EC09601C5
:108690002F5E3F4F4FE1E42EF12C01E0A401BE011B
:1086A0006F5F7F4FC6010E94383722E0F601248BAE
:1086B000A58A2B2D3327268B830124E03FE140E060
:1086C00050E0BC01C6010E948C372C960FB6F8947E
:1086D000DEBF0FBECDBFDF91CF911F910F91FF90F5
:1086E000EF90DF90CF90BF90AF909F908F907F9052
:1086F0006F9008950F931F938B0124E031E140E0C8
:1087000050E060E070E00E948C371F910F91089557
:108710004F925F926F927F928F929F92AF92BF9291
:10872000CF92DF92EF92FF920F931F93CF93DF933D
:10873000CDB7DEB72C970FB6F894DEBF0FBECDBF16
:108740006C014B012A013901BA010E941B375C01FF
:108750008FEFA8168FEFB80629F46DEF7EEF8FEF3D
:108760009FEF22C096012F5E3F4F7FE0E72EF12C56
:1087700001E0A401BE016F5F7F4FC6010E94383740
:1087800024E0F601248BA58A2B2D3327268B678ABC
:10879000272D3327208F820124E03FE040E050E086
:1087A000BC01C6010E948C372C960FB6F894DEBF30
:1087B0000FBECDBFDF91CF911F910F91FF90EF9032
:1087C000DF90CF90BF90AF909F908F907F906F90F1
:1087D0005F904F9008956F927F928F929F92AF9289
:1087E000BF92CF92DF92EF92FF920F931F93CF939E
:1087F000DF93CDB7DEB72C970FB6F894DEBF0FBE70
:10880000CDBF6C013B014A01122FBA010E941B37F8
:108810005C018FEFA8168FEFB80629F46DEF7EEF9D
:108820008FEF9FEF1EC096012F5E3F4FB6E0EB2EFD
:10883000F12C01E0A301BE016F5F7F4FC6010E94D2
:10884000383723E0F601248BA58A2B2D3327268B7E
:10885000178B840124E036E0A301BC01C6010E940D
:108860008C372C960FB6F894DEBF0FBECDBFDF91CC
:10887000CF911F910F91FF90EF90DF90CF90BF901D
:10888000AF909F908F907F906F900895AF92BF921E
:10889000CF92DF92EF92FF920F931F93CF93DF93CC
:1088A000CDB7DEB72C970FB6F894DEBF0FBECDBFA5
:1088B0006C015B019C012F5E3F4F12E0E12EF12C19
:1088C00001E0AB01BE016F5F7F4F0E943837F601B8
:1088D000148A0FEF1FEF24E032E0A501BC01C601AE
:1088E0000E948C372C960FB6F894DEBF0FBECDBF1A
:1088F000DF91CF911F910F91FF90EF90DF90CF907C
:10890000BF90AF9008952F923F924F925F926F92D7
:108910007F928F929F92AF92BF92CF92DF92EF920F
:10892000FF920F931F93CF93DF93CDB7DEB72D97B1
:108930000FB6F894DEBF0FBECDBF2C013B011A016C
:108940002D874801AE2C9C012F5E3F4F89E1E82E18
:10895000F12C01E040E050E0BE016F5F7F4FC201AB
:108960000E943837DC01FC0191868086BB24CC2430
:10897000DD24A482B582C682D7828AE0F201848B8C
:10898000C2014596A30126E0FA010190AF01FC0166
:108990000192CF012150C1F78D85F201838F148E92
:1089A000258E832D9927868F0FEF1FEF24E039E165
:1089B00040E050E0BD01C2010E948C372D960FB6F9
:1089C000F894DEBF0FBECDBFDF91CF911F910F9105
:1089D000FF90EF90DF90CF90BF90AF909F908F90DF
:1089E0007F906F905F904F903F902F9008954F929F
:1089F0005F927F928F929F92AF92BF92CF92DF92BF
:108A0000EF92FF920F931F93CF93DF93CDB7DEB713
:108A10002C970FB6F894DEBF0FBECDBF6C012B01B3
:108A20004A01722E58019C012F5E3F4F9DE0E92EB6
:108A3000F12C01E040E050E0BE016F5F7F4FC601C6
:108A40000E9438378C0187E1F601848BD601559658
:108A5000F40186E001900D928150E1F7F601738EEA
:108A6000A501D60160E070E0272D33270DC07A0103
:108A7000FA018191AF01FD01848F1196F701808188
:108A8000882329F06F5F7F4F6217730781F7F80122
:108A900091868086820124E03DE040E050E060E085
:108AA00070E0C6010E948C372C960FB6F894DEBF9A
:108AB0000FBECDBFDF91CF911F910F91FF90EF902F
:108AC000DF90CF90BF90AF909F908F907F905F90FE
:108AD0004F900895AF92BF92CF92DF92EF92FF92A4
:108AE0000F931F93CF93DF93CDB7DEB72C970FB6BD
:108AF000F894DEBF0FBECDBF5C016B019C012F5E01
:108B00003F4F4CE0E42EF12C01E040E050E0BE018C
:108B10006F5F7F4F0E94383786E0F501848BD50167
:108B20005596F60101900D928150E1F70FEF1FEF7E
:108B300024E03CE040E050E060E070E0C5010E94CD
:108B40008C372C960FB6F894DEBF0FBECDBFDF91E9
:108B5000CF911F910F91FF90EF90DF90CF90BF903A
:108B6000AF9008956F927F928F929F92AF92BF9233
:108B7000CF92DF92EF92FF920F931F93CF93DF93E9
:108B8000CDB7DEB72C970FB6F894DEBF0FBECDBFC2
:108B90006C013B015A0149010E941B378F5F9F4FB7
:108BA00029F46DEF7EEF8FEF9FEF38C096012F5EB7
:108BB0003F4F5BE0E52EF12C01E040E050E0BE01CC
:108BC0006F5F7F4FC6010E94383786E1F601848BC4
:108BD000D6015596F50186E001900D928150E1F79E
:108BE000A401D60120E030E0FA018081FD01838FED
:108BF000FA018081882341F02F5F3F4F4F5F5F4F25
:108C000011962F30310581F7830124E03BE040E0ED
:108C100050E060E070E0C6010E948C372C960FB6E1
:108C2000F894DEBF0FBECDBFDF91CF911F910F91A2
:108C3000FF90EF90DF90CF90BF90AF909F908F907C
:108C40007F906F900895AF92BF92CF92DF92EF9294
:108C5000FF920F931F93CF93DF93CDB7DEB72C977F
:108C60000FB6F894DEBF0FBECDBF5C016B01142FB1
:108C70009C012F5E3F4F69E0E62EF12C01E040E0C1
:108C800050E0BE016F5F7F4F0E94383787E0F501EB
:108C9000848BD5015596F60186E001900D928150A6
:108CA000E1F7F501138F0FEF1FEF24E039E040E00B
:108CB00050E060E070E0C5010E948C372C960FB642
:108CC000F894DEBF0FBECDBFDF91CF911F910F9102
:108CD000FF90EF90DF90CF90BF90AF9008958F926C
:108CE0009F92AF92BF92CF92DF92EF92FF920F933B
:108CF0001F93CF93DF93CDB7DEB72C970FB6F894C1
:108D0000DEBF0FBECDBF5C014B016A019C012F5E2F
:108D10003F4F78E0E72EF12C01E0A401BE016F5F28
:108D20007F4F0E943837BC0186E0F501848BD50166
:108D30005596F60101900D928150E1F70FEF1FEF6C
:108D400024E038E0A401C5010E948C372C960FB6B0
:108D5000F894DEBF0FBECDBFDF91CF911F910F9171
:108D6000FF90EF90DF90CF90BF90AF909F908F904B
:108D700008952F923F924F925F926F927F928F92BF
:108D80009F92AF92BF92CF92DF92EF92FF920F939A
:108D90001F93CF93DF93CDB7DEB72D970FB6F8941F
:108DA000DEBF0FBECDBF5C011B014A0139010D873B
:108DB00027011C2DBA010E94642D6D5F7E4F8F4FDD
:108DC0009F4F29F069EF7EEF8FEF9FEFDBC0F4013B
:108DD0004081D501A358BD4F20E030E08C9184172D
:108DE00049F5FD019181F4018181981719F5FD0183
:108DF0009281F40182819817E9F4FD019381F401D5
:108E000083819817B9F4FD019481F4018481981746
:108E100089F4FD019581F4018581981759F4FD01CC
:108E20008585833009F4A5C0823009F49DC0843063
:108E300009F49AC02F5F3F4F57962A30310571F6DB
:108E4000D501A657BD4F40E050E020E030E0F501ED
:108E5000E757FD4F8C91853039F4808182958F7072
:108E6000837011F44F5F5F4F2F5F3F4F7796579698
:108E70002A30310579F7473051050CF07FC0C50124
:108E80000E94D6366C018F5F9F4F09F477C0950121
:108E90002F5E3F4F05E0E02EF12C01E0A101BE0165
:108EA0006F5F7F4FC5010E943837BC018DE0F5012F
:108EB000848BD5015596F40186E001900D92815086
:108EC000E1F7F501638E872D9927848F2D85258FF6
:108ED000168E478E852D992780A311A387E190E0F8
:108EE000C89EF001C99EF00DD89EF00D1124E358E4
:108EF000FD4FEA0DFB1DD40186E00D9001928150DB
:108F0000E1F787E190E0C89EF001C99EF00DD89E80
:108F1000F00D1124EA0DFB1DE657FD4F83E0808321
:108F2000EA58F24080911D1690911E16DF01A75855
:108F3000BD4F11969C938E93019690931E1680932D
:108F40001D16E757FD4F1295110F110F107C8081F0
:108F50008F70812B80830D911C9124E035E0A1015D
:108F6000C5010E948C370EC067EF7EEF8FEF9FEF39
:108F700009C068EF7EEF8FEF9FEF04C06CEF7EEFCC
:108F80008FEF9FEF2D960FB6F894DEBF0FBECDBFCB
:108F9000DF91CF911F910F91FF90EF90DF90CF90D5
:108FA000BF90AF909F908F907F906F905F904F9009
:108FB0003F902F9008956F927F928F929F92AF92E1
:108FC000BF92CF92DF92EF92FF920F931F93CF93B6
:108FD000DF93CDB7DEB72C970FB6F894DEBF0FBE88
:108FE000CDBF4C013B01B42EA22E68019C012F5E27
:108FF0003F4F91E0E92EF12C01E0AB01BE016F5F24
:109000007F4FC4010E9438377C01C401885B9D4FAB
:109010000E946F49F7011482158216821782D18649
:10902000C08685E0F401848B83E3858B8BE8868B97
:109030008EE9878B8B2D813308F080E3F401808FDC
:10904000AA2011F481E0A82EF401A18E0FEF1FEFEA
:1090500024E031E0A301B701C4010E948C372C96B3
:109060000FB6F894DEBF0FBECDBFDF91CF911F9139
:109070000F91FF90EF90DF90CF90BF90AF909F90B7
:109080008F907F906F9008956F927F928F929F92B2
:10909000BF92CF92DF92EF92FF920F931F93CF93E5
:1090A000DF93CDB7DEB72C970FB6F894DEBF0FBEB7
:1090B000CDBF6C01B62E8C0104591C4FD8018D9187
:1090C0009C91892B39F481E090E00E945508F801C9
:1090D00091838083D801ED91FC91B082B2E0BB1600
:1090E000D9F1BB1538F0BB20C1F0E1E0BE1609F0A4
:1090F0007AC00AC0F4E0BF1609F1BF1628F185E076
:10910000B81609F070C012C0BAE0BB2E612CA4E8FA
:109110007A2EA3E08A2E912C27C0FCE0BF2E612C72
:10912000E8E07E2EE7E08E2E912C1EC073E0B72E75
:10913000612C6BE4762E812C912C16C0612C56E9A3
:10914000752E812C912C10C046E0B42E612C31EE8E
:10915000732E812C912C08C028E0B22E612C92EC49
:10916000792E91E0892E912C96012F5E3F4F8FE052
:10917000E82EF12C0FE340E050E0BE016F5F7F4F1F
:10918000C6010E9438377C0185E0F601848B83E0BC
:10919000858B168A178AB08E118E0FEF1FEF2CEF7A
:1091A0003FE0A701B701C6010E948C376115710528
:1091B00081059105C1F4F601828193810E944518D1
:1091C000B401A3010E94FE34892B69F440E050E011
:1091D00060E070E0C7010A960E946D0A60E070E0EE
:1091E00080E090E004C06FEF7EEF8FEF9FEF2C9652
:1091F0000FB6F894DEBF0FBECDBFDF91CF911F91A8
:109200000F91FF90EF90DF90CF90BF909F908F9045
:109210007F906F900895FC0182819381009719F4EB
:109220008FEF9FEF089501979383828380E090E012
:10923000089560E279E486E395E00E9486540895FB
:10924000CF93DF93C091A814D091A91419C0E881DD
:10925000F981828193819F938F93FF93EF938BE3A7
:1092600095E09F938F930E9444520A80DB81C02D2A
:109270008DB79EB706960FB6F8949EBF0FBE8DBFF2
:10928000209729F7DF91CF910895FC018281938186
:10929000680F791F73836283892B19F4CF010E94B1
:1092A000DA0980E090E00895FC0182819381738364
:1092B0006283892B19F4CF010E94DA0980E090E0E3
:1092C0000895FC01828193810196938382830197A3
:1092D00019F4CF010E948B0980E090E00895CF93AC
:1092E000DF93EC0107C040E050E060E070E0CE01A9
:1092F0000E946D0A8A819B810097A9F301979B8345
:109300008A8380E090E0DF91CF9108950F931F93BF
:10931000CF93DF938C01FC011182108273836283EF
:10932000C091A814D091A914209759F484E090E03A
:109330000E944109FC019093A9148093A8140CC0C9
:10934000EC018A819B810097D9F784E090E00E942C
:109350004109FC019B838A8311830083DF91CF91B4
:109360001F910F910895089584B7806884BF84BFCA
:10937000089584B78F7784BF84BF0895EAE9F0E049
:109380008081877F80838B9893988A9892988C9815
:10939000949815981D98A1E6B0E08C918F7B8C93E2
:1093A000E2E6F0E080818F7B80838C918F7D8C93CF
:1093B00080818F7D80838C918F7E8C9380818F7E46
:1093C00080830895EAE9F0E08081886080838B9A49
:1093D000939A8A98929A8C9A15980895882321F0E6
:1093E00084E00E946F4A089584E00E947C4A0895B8
:1093F000882321F085E00E946F4A089585E00E944D
:109400007C4A0895882321F087E00E947C4A0895D1
:1094100087E00E946F4A0895189A939A8B9A80E089
:109420000E94D1030895882321F086E00E946F4AAC
:1094300003C086E00E947C4A88E495E00E94BE4911
:1094400084B7806884BF84BF08950F931F9308E496
:1094500015E0C8010E94BE4984B7806884BF84BFFC
:1094600080E00E94134A81E00E94024A68EE73E0A5
:1094700080E090E00E947B0681E00E94134A64EF46
:1094800071E080E090E00E947B0680E00E94024A4A
:1094900084B78F7784BF84BFC8010E94E24960ED22
:1094A00077E080E090E00E947B061F910F91089585
:1094B0000FB6F8940F92E82FFF27FE2FEE2790812A
:1094C0009083C59A0000C5980F900FBE8093AA1490
:1094D0000895BD9A8091AA140E94584A089521E0E7
:1094E00030E002C0220F331F8A95E2F78091AA1460
:1094F000822B0E94584A089521E030E002C0220FDA
:10950000331F8A95E2F720958091AA1482230E9446
:10951000584A0895A0913716BB27FD01EE0FFF1F93
:10952000EE0FFF1FEF5DF94E80836183428323833B
:10953000CD01019665E070E00E94177F282F80938F
:10954000371680912016281749F4822F9927019603
:1095500065E070E00E94177F809320160895809345
:109560004D056093AB1440934E0508951F93182F3B
:1095700080913516882319F4812F0E94117681E09D
:1095800090E002C0880F991F1A95E2F7809520910C
:109590001F16282320931F161F9108951F93182F1D
:1095A00080913516882319F4812F0E941F7681E05F
:1095B00090E002C0880F991F1A95E2F720911F16BC
:1095C000282B20931F161F910895CF93DF93C82F48
:1095D000DD27C0FF04C080E00E941F7603C080E04A
:1095E0000E941176C1FF04C081E00E941F7603C073
:1095F00081E00E941176C2FF04C082E00E941F76C3
:1096000003C082E00E941176C3FF04C083E00E9481
:109610001F7603C083E00E941176DF91CF910895F9
:10962000CF93DF93C0E0D0E080911F1699270C2ED6
:1096300002C0959587950A94E2F780FF04C08C2FAD
:109640000E941F7603C08C2F0E9411762196C43091
:10965000D10551F7DF91CF9108958091371680930E
:1096600020160E94104B1092351608951F93182F44
:109670000E942D761092371610922016112351F069
:1096800020E034E040E050E06CE47BE489E495E0E5
:109690000E94340B1F91089586E90E94B907E0915A
:1096A000201680913716E81719F41092351645C028
:1096B000FF27EE0FFF1FEE0FFF1FEF5DF94E8081BA
:1096C0008093351600E010E0802F0E9411760F5F26
:1096D0001F4F04301105C1F780912016A82FBB271A
:1096E000FD01EE0FFF1FEE0FFF1FEF5DF94E8381AF
:1096F0008F3F11F081508383128180913516843021
:1097000009F469C0853060F4813009F449C08130C2
:10971000A0F0823009F452C0833009F062C187C0E2
:10972000863009F4CEC0863008F4A3C0873009F42F
:10973000F9C0883009F055C127C180914E058823B2
:1097400029F10E948A6920914D05EFE32E9F900137
:109750001124442755270E942A7F6F337105810504
:109760009105A0F46091AB14662321F021E04091B3
:109770004E0507C080911F16882331F421E041E097
:1097800061E084E00E948A4A109236168091361673
:109790008F5F809336166FE370E080E090E00BC03F
:1097A00081810E94E54A6FE3169FB001112488274A
:1097B00077FD8095982F0E947B061BC181810E94B6
:1097C000E54A8FE3189FC00111247C010027F7FCB4
:1097D0000095102F21C080E00E94E54A8FE3189F7A
:1097E000C00111247C010027F7FC0095102FC8014F
:1097F000B7010E947B0680913516882309F44FCF6C
:10980000E0912016FF27EE0FFF1FEE0FFF1FEF5D09
:10981000F94E81810E94E54AC801B7010E947B068A
:1098200080913516882309F43ACF80E01FC080E08C
:109830000E94E54A8FE3189FC00111247C01002794
:10984000F7FC0095102FC801B7010E947B0680919C
:109850003516882309F423CFE0912016FF27EE0F59
:10986000FF1FEE0FFF1FEF5DF94E81810E94E54A59
:10987000B5C080E00E941F76C12FDD278FE390E006
:109880009C01C29FC001C39F900DD29F900D1124D7
:109890007C010027F7FC0095102FDD24C801B701DB
:1098A0000E947B0680913516882391F18D2D0E94B0
:1098B0001176D3948D2D0E941F7633E0D31671F765
:1098C00027C083E00E941F76C12FDD278FE390E041
:1098D000FC01CE9FC001CF9F900DDE9F900D112403
:1098E0007C010027F7FC0095102F63E0D62EC801FD
:1098F000B7010E947B0680913516882349F08D2D93
:109900000E941176DA948D2D0E941F76DD2079F762
:109910008FE390E0C89FB001C99F700DD89F700D74
:10992000112445CF80E00E941F768FE3189FC0016D
:1099300011246C01EE24D7FCE094FE2C10E0C7014A
:10994000B6010E947B0680913516882349F0812F4D
:109950000E9411761F5F812F0E941F76133079F7C6
:1099600013E0C701B6010E947B068091351688235B
:1099700009F495CE812F0E9411761150812F0E94FB
:109980001F761123B1F1EDCF80E00E941F7681E0B8
:109990000E941F7682E00E94117683E00E94117679
:1099A0008FE3189FC00111247C010027F7FC00956C
:1099B000102FC801B7010E947B06809135168823BD
:1099C00009F46DCE80E00E94117681E00E9411764C
:1099D00082E00E941F7683E00E941F76C801B701D3
:1099E000EACEAA0FBB1FAA0FBB1FAF5DB94EFD0188
:1099F000138280913516882309F451CE8091201668
:109A0000282F3327F901EE0FFF1FEE0FFF1FEF5D29
:109A1000F94E8381882309F042CEC901019665E0A1
:109A200070E00E94177F2091371633278217930723
:109A300011F40E94104B809120169927019665E041
:109A400070E00E94177F8093201629CEE82F815066
:109A50008F3118F08FEF9FEF0895FF27E455FB4EED
:109A6000828199270895E82F81508F3120F4FF27B4
:109A7000E455FB4E628308959C018091D615909128
:109A8000D715892B19F08FEF9FEF08953093D715D5
:109A90002093D6157093D9156093D8155093D5158A
:109AA0004093D41580E090E008951092D71510925D
:109AB000D6151092D9151092D8151092D51510926E
:109AC000D415089581E08093DA1508951092D11588
:109AD0001092D0151092CF151092CE151092D3156A
:109AE0001092D2151092DA151092DC151092DB1537
:109AF00040E058EC60E074E082E090E00E949B500F
:109B00009093AD148093AC14EEEAF4E18FEF81935F
:109B100094E1EE3CF907D9F71092D7151092D615BB
:109B20001092D9151092D8151092D5151092D415FF
:109B300020E034E040E050E060EB7DE48FE495E02D
:109B40000E94340B08951092DA158091DB159091E4
:109B5000DC15892B21F08BED95E10E941A0A0895FE
:109B6000CF93DF93CDB7DEB7CB50D1400FB6F8948B
:109B7000DEBF0FBECDBF88EC0E94B90740E050E0C9
:109B800060E070E082ED95E10E946D0AAA24BB249A
:109B900001C057018091AC149091AD140E942750E0
:109BA0008C01E090D015F090D1150894E108F108EF
:109BB0008091DA15882311F140E050E060E070E018
:109BC0008BED95E10E946D0AC8010E949150882397
:109BD00089F4A090D015B090D1150894A108B108CF
:109BE000C8010E9463508091AC149091AD140E9402
:109BF00027508C0182ED95E10E948B094E0108945B
:109C0000811C911C4BE050E0B401C8010E94C3507C
:109C1000892B09F03FC089819A818A159B05D1F172
:109C20008091D6159091D715892B61F18B81E091A8
:109C3000D415F091D515E80FF11D208133278C81C3
:109C40009927019702C0359527958A95E2F720FF5D
:109C500019C049855A858CE0C82ED12CCC0EDD1E4A
:109C6000B601C8010E94C350892BA1F44091D815B8
:109C70005091D915E091D615F091D715B401C601D0
:109C8000099505C069857A85C8010E94F74F0E9431
:109C90003D088ECFC8010E9463508091D0159091ED
:109CA000D1150197E816F90609F073CF40E050E0AE
:109CB00060E070E082ED95E10E946D0A6ACF7F92CC
:109CC0008F929F92AF92BF92CF92DF92EF92FF92CC
:109CD0000F931F93CF93DF93CDB7DEB72B970FB6BC
:109CE000F894DEBF0FBECDBF6C018B014A01590154
:109CF0008091AC149091AD140E9427507C01892B67
:109D0000E9F10115110519F00C0D1D1D06C000919A
:109D1000D0151091D1150150104077244BE050E040
:109D2000BE016F5F7F4FC7010E94C350892B19F599
:109D300089819A818C159D05F1F049855A856EECD3
:109D400074E1C7010E94C350892BA9F489819A81CB
:109D50008017910719F491E0792E02C0772041F025
:109D6000A501BE016F5F7F4F8EEC94E1F401099570
:109D70000E943D08D3CFC7010E9463502B960FB6B7
:109D8000F894DEBF0FBECDBFDF91CF911F910F9131
:109D9000FF90EF90DF90CF90BF90AF909F908F900B
:109DA0007F9008954F925F926F927F928F929F92D1
:109DB000AF92BF92CF92DF92EF92FF920F931F93D9
:109DC000CF93DF93CDB7DEB72B970FB6F894DEBFF6
:109DD0000FBECDBF6C01562E442E39014801809133
:109DE000AC149091AD140E9427508C01892BE9F19D
:109DF000EE24FF245E010894A11CB11C4BE050E04E
:109E0000B501C8010E94C350892B61F549855A8567
:109E10006EEC74E1C8010E94C350892B19F55520DE
:109E200019F08B81851591F4242D33278C81992786
:109E3000019702C0359527958A95E2F720FF06C065
:109E4000A401B5018EEC94E1F30109950894E11C9D
:109E5000F11CC114D10419F0CE14DF0419F00E94D2
:109E60003D08C8CFC8010E9463502B960FB6F894E6
:109E7000DEBF0FBECDBFDF91CF911F910F91FF903D
:109E8000EF90DF90CF90BF90AF909F908F907F909A
:109E90006F905F904F9008958091AC149091AD14A5
:109EA0000E947C500895CF93DF932EEF30E0809195
:109EB000CE159091CF15281B390BEA0124173507D1
:109EC00008F4E9018091AC149091AD140E941A51EC
:109ED0008091CE159091CF158C0F9D1F9093CF152B
:109EE0008093CE15CE01DF91CF910895EF92FF922E
:109EF0000F931F93CF93DF93CDB7DEB72D970FB698
:109F0000F894DEBF0FBECDBFFE88EF88EF2DFF2790
:109F1000E455FB4E228133278E2D9927019702C0ED
:109F2000359527958A95E2F720FF54C00E948A69EB
:109F30006F83788789879A871092CF151092CE15F4
:109F40009E01265E3F4F3A832983488D598D60E0FC
:109F500070E083E59FE40E945E1A0091CE15109197
:109F6000CF150E3F110561F441E050E066E575E064
:109F70008091AC149091AD140E941A510FEF10E033
:109F800041E050E068E575E08091AC149091AD142B
:109F90000E941A518091D0159091D1159C838B838A
:109FA00001969093D1158093D015FD82EE820F5FBC
:109FB0001F4F1C870B874BE050E0BE016D5F7F4F4A
:109FC0008091AC149091AD140E941A5182ED95E1EC
:109FD0000E94DA092D960FB6F894DEBF0FBECDBFF2
:109FE000DF91CF911F910F91FF90EF900895CF9344
:109FF000DF93FC01A081B1818681823019F48DEF5D
:10A000009FEF22C0848195818617970728F482E00C
:10A0100086838EEF9FEF18C0861B970B95838483F2
:10A02000828193818617970738F4681B790BED01BD
:10A03000888599859383828382819381861B970B80
:10A040009383828380E090E0DF91CF910895CF9356
:10A05000DF93DC01EC018889882321F480E090E023
:10A0600020E012C0FD018789882321F481E090E07F
:10A0700021E00AC0ED018E8D882319F080E090E088
:10A080001FC082E090E022E0FC0133E0EE0FFF1FF2
:10A090003A95E1F7E81BF90BEA0FFB1FED018C8104
:10A0A0009D81958784878E819F819787868781E0B0
:10A0B000808B87E0289FC00111240A968A0F9B1F7E
:10A0C000DF91CF910895FC01892BA9F02081318186
:10A0D000C9010A968E179F0709F41682C901419695
:10A0E0008E179F0709F41682D9015896AE17BF073D
:10A0F00011F4FD0116820895FC018089813011F46C
:10A1000082E0808B8789813011F482E0878B868D95
:10A11000813011F482E0868F1582148217821682B4
:10A12000089520E030E0FC018681813011F421E0C7
:10A1300030E0C9010895CF92DF92EF92FF920F9322
:10A140001F937B018C016A018FE190E00E9441091D
:10A15000FC01E082F18202831383D186C0861582DE
:10A1600014821782168293878287108A928B818B42
:10A17000178A918F808F168E1F910F91FF90EF900D
:10A18000DF90CF900895CF92DF92EF92FF920F93DE
:10A190001F93CF93DF93EC016B018A01E880F98074
:10A1A0008E81823019F48DEF9FEF3BC08C819D81B1
:10A1B0008417950728F482E08E838EEF9FEF31C0DD
:10A1C000841B950B9D838C832A813B812417350743
:10A1D00088F4021B130BF701408151816281738166
:10A1E000C601800F911F0E941277F701808591852B
:10A1F0009B838A834A815B81401B510B5B834A832B
:10A2000066277727F70180819181A281B381480F6A
:10A21000591F6A1F7B1F9801C6010E94127780E0B8
:10A2200090E0DF91CF911F910F91FF90EF90DF9021
:10A23000CF900895CF92DF92EF92FF920F931F93EA
:10A24000CF93DF93EC016B017A01488559854E1558
:10A250005F0518F48EEF9FEF62C02E813F81CA0127
:10A260008E199F098217930718F45F834E8304C0E9
:10A270002E0D3F1D3F832E83FE0140E052E080897A
:10A280008130A1F42E813F8188859985281739076F
:10A2900069F4868597858E159F0520F4508B178667
:10A2A000168604C08E199F09978786874F5F379659
:10A2B000433029F74C815D8108851985041B150BF6
:10A2C0000E151F05A0F46627772788819981AA813A
:10A2D000BB81480F591F6A1F7B1F9801C6010E944E
:10A2E00071761D821C82E01AF10AC00ED11E4C81CB
:10A2F0005D816627772788819981AA81BB81480F74
:10A30000591F6A1F7B1F9701C6010E9471768C81BD
:10A310009D818E0D9F1D9D838C8380E090E0DF9159
:10A32000CF911F910F91FF90EF90DF90CF90089504
:10A330009C01E0913816F0913916E657FD4F808167
:10A340009181EA58F2408217930719F420E030E037
:10A350000EC0E157F94F80819181EF58F640821786
:10A36000930719F080E090E0089521E030E085E067
:10A3700094E0AC01249FC001259F900D349F900D67
:10A38000112486579D4F8E0F9F1F089580E090E007
:10A390000E949851FC01892B19F481E090E0089506
:10A3A000809104169091051691838083ED5FFB4F99
:10A3B0001182108280E090E00895809104169091BF
:10A3C00005160E949851FC01892B19F481E090E058
:10A3D000089581E08283ED5FFB4F1182108280E05F
:10A3E00090E0089580910416909105160E9498516E
:10A3F000DC01892B19F480E090E00895AD5FBB4F3C
:10A40000ED91FC911197A350B440EA0FFB1F13820A
:10A41000FD011282CD01039608950F931F93DC0175
:10A42000FC0101900020E9F731970E2F081B043141
:10A4300008F003E111278091381690913916A80190
:10A44000BD01805E924F0E94DD7E80913816909112
:10A450003916080F191F005E124FF80110821F9164
:10A460000F91089580913816909139168C5C924F17
:10A470000E94F66B089580913816909139168C5C85
:10A48000924F0E94136C08950F931F93CF93DF9305
:10A49000CDB7DEB722970FB6F894DEBF0FBECDBFA3
:10A4A00009851A8580910416909105160E9498518D
:10A4B000FC01892B71F08281882359F09E01255F70
:10A4C0003F4F3A832983A801BF018AE892E50E94A1
:10A4D0005E1ACE010B969A8389830E943B52AE018D
:10A4E000455F5F4F5A834983B80180913A16909136
:10A4F0003B160E9465198C010E943252C8012296B7
:10A500000FB6F894DEBF0FBECDBFDF91CF911F9184
:10A510000F9108950F931F93CF93DF938C010D5FDD
:10A520001B4FF80120813181CEEFD3E0C21BD30B4A
:10A530004C175D0708F4EA010396AE01820F931FE2
:10A540000E94A77EF801808191818C0F9D1F9183CD
:10A550008083CE01DF91CF911F910F910895EF92EB
:10A56000FF920F931F937C01062F809138169091D4
:10A5700039168C5C924F0E94136C80913A16909120
:10A580003B160E9445181127A801B7010E94131A13
:10A5900080913816909139168C5C924F0E94F66B20
:10A5A0001F910F91FF90EF900895EF92FF920F93FC
:10A5B0001F93CF93DF93CDB7DEB722970FB6F894F2
:10A5C000DEBF0FBECDBF8E01055F1F4FF801E190CA
:10A5D000F1908F0180913816909139168C5C924FD2
:10A5E0000E94136C1A830983A801B70180913A165F
:10A5F00090913B160E94BB748C018091381690910B
:10A6000039168C5C924F0E94F66BC80122960FB6E9
:10A61000F894DEBF0FBECDBFDF91CF911F910F9198
:10A62000FF90EF9008950F931F938C01809138163F
:10A63000909139168C5C924F0E94136C60913A167F
:10A6400070913B16C8010E94F41D809138169091BC
:10A6500039168C5C924F0E94F66B1F910F910895F2
:10A66000E0913816F0913916E256F24F24E641E0B7
:10A67000608182E00E948A4A809138169091391652
:10A68000865C924F0E94135308950F931F93982F47
:10A69000DB01E0913816F0913916E65CF24F8081CB
:10A6A000EA53FD40882321F5E256F24F9083FB01E7
:10A6B00001900020E9F731970E2F061B043608F0B1
:10A6C00003E611278091381690913916A801BD0133
:10A6D000865C924F0E94DD7E8091381690913916EB
:10A6E000080F191F065C124FF80110820E943053A8
:10A6F0001F910F9108958091381690913916805EC0
:10A70000924F0E94135308950E947B53E091381694
:10A71000F0913916DF01A15EB24FE25EF24F808107
:10A72000EE51FD4022E8829FC00111248C56954FC6
:10A730006C918E0F9F1F0E94AF520895CF93DF93AD
:10A74000EB0190933B1680933A168FE99DE00E94AF
:10A7500041099093391680933816009749F48BED90
:10A7600090E09F938F930E94D5520F900F902BC033
:10A77000FE0101900020E9F731974E2F4C1B453127
:10A7800008F044E15527BE01805E924F0E94DD7EB5
:10A7900020E030E08091381690913916FC013B960C
:10A7A000118210823D962F5F3F4F22333105C1F752
:10A7B0008C5C924F0E94DA6BE0913816F09139165A
:10A7C000E65CF24F1082DF91CF9108956F927F92F5
:10A7D0009F92AF92BF92CF92DF92EF92FF920F9330
:10A7E0001F93CF93DF937C01A0903816B090391659
:10A7F0006501662477248501962CF601838594856E
:10A80000892BF9F0E80109900020E9F72197C01B96
:10A81000D10BAE01B701C8010E94CF7E892B89F40C
:10A82000F701EC0FFD1F8081803209F44AC0F70167
:10A8300001900020E9F73197EE19FF09CE17DF07E5
:10A84000A1F093940894611C711C035F1F4F8DE06D
:10A8500090E0C80ED91E92E36916710469F6E2E32E
:10A860009E1619F481E090E043C0292D33278DE036
:10A8700090E0289FF001299FF00D389FF00D1124E2
:10A88000EA0DFB1DDF010D900020E9F71197AE1BCB
:10A89000BF0BAE0DBF1D8C91811111968DE090E024
:10A8A000289FF001299FF00D389FF00D1124EA0D2B
:10A8B000FB1D0384F485E02DCD01099580E090E037
:10A8C00017C0262D33278DE090E0289FF001299FA7
:10A8D000F00D389FF00D1124EA0DFB1DDF010D90E6
:10A8E0000020E9F71197AE1BBF0BAE0DBF1DD5CFF2
:10A8F000DF91CF911F910F91FF90EF90DF90CF905C
:10A90000BF90AF909F907F906F900895CF93DF930B
:10A91000EC01FC0101900020E9F73197E81BF90BED
:10A920003B97C0F09F938F9385EC91E09F938F931B
:10A930000E94D5528DEA91E09F938F930E94D55249
:10A940004DB75EB74A5F5F4F0FB6F8945EBF0FBE5C
:10A950004DBF3EC0A0913816B0913916FD0120E0E0
:10A9600083859485892BD9F02F5F3D962233C1F7DB
:10A97000DF93CF9389E991E09F938F930E94D55203
:10A980008EE791E09F938F930E94D5528DB79EB72B
:10A9900006960FB6F8949EBF0FBE8DBF19C0332721
:10A9A0008DE090E0FC012E9FC0012F9F900D3E9FF7
:10A9B000900D1124A80FB91FFD01748763872091A2
:10A9C000381630913916BE01820F931F0E94C87E3F
:10A9D000DF91CF9108952F923F924F925F926F92A5
:10A9E0007F928F929F92AF92BF92CF92DF92EF921F
:10A9F000FF920F931F93CF93DF93CDB7DEB72397CB
:10AA00000FB6F894DEBF0FBECDBF7C01062F498381
:10AA100022241FEF332444245524662477248824D9
:10AA20009924AA24BB24C0903816D0903916C501A9
:10AA30008C0D9D1D9B838A83FC0183859485892BC6
:10AA400009F45DC0402F5527B701CF010E94CF7E8A
:10AA5000892B09F054C0F981FF2349F11F3F19F0F8
:10AA600091E0392E08C08FED91E09F938F930E9463
:10AA7000D5520F900F908091381690913916880D0D
:10AA8000991D0E9413532394822D65E00E940B7F31
:10AA9000992319F48DED91E002C08BED91E09F9325
:10AAA0008F930E94D552102F0F900F9028C01F3FF8
:10AAB00011F0202F20C0EA81FB8101900020E9F7EE
:10AAC00031971E2F8A81181B6A817B81C7010E94E2
:10AAD000C87E15C0122F11C0822F9927D701A80F49
:10AAE000B91FF301EC0DFD1DE80FF91F9C9180814A
:10AAF000981781F72F5F211778F381E0382E08949B
:10AB0000411C511CEDE0F0E0AE0EBF1E8E0E9F1EEC
:10AB10006E0E7F1EF2E34F16510409F084CF1F3FE3
:10AB200019F4802F992723C0332031F4F701E10F66
:10AB3000F11D80E280831F5F8981882379F089ED90
:10AB400091E09F938F930E94D5520E947B53612F77
:10AB5000C7010E94AF520F900F9007C0612F601B7A
:10AB6000C701800F911D0E94AF52812F9927239614
:10AB70000FB6F894DEBF0FBECDBFDF91CF911F910E
:10AB80000F91FF90EF90DF90CF90BF90AF909F908C
:10AB90008F907F906F905F904F903F902F9008958F
:10ABA000DF92EF92FF920F931F93CF93DF93CDB776
:10ABB000DEB723970FB6F894DEBF0FBECDBF86E990
:10ABC0000E94B9070E948453EE24DD24FF24809163
:10ABD0003A1690913B160E94451841E050E0BE01A4
:10ABE0006F5F7F4F0E944E728F3F39F480E591E096
:10ABF0009F938F930E94D552E2C1813041F780919B
:10AC00003A1690913B160E9445180E94A07B88231B
:10AC100069F099279F938F938BE391E09F938F9394
:10AC20000E94D5520F900F900F900F9099819B31F9
:10AC300009F0BCC010E080913A1690913B160E943A
:10AC40004518212F332727FD309542E050E0421B65
:10AC5000530BBE016F5F7F4F620F731F0E944E72D6
:10AC6000180F123044F389818B3509F04BC08A816B
:10AC70008134D1F42E2D3327E0913816F091391616
:10AC8000E25EF24F80819927821B930B059665E067
:10AC900070E00E94177F0497A9F1DD2011F4EE20E7
:10ACA00089F1C90104960EC0E0913816F091391669
:10ACB000823471F4E25EF24F8081E81619F18E2D34
:10ACC0009927019665E070E00E94177FE82E1AC070
:10ACD000E25EF24FE08016C081508C9388E090E0F5
:10ACE0009F938F939F938F9385E391E09F938F938F
:10ACF0000E94D5528DB79EB706960FB6F8949EBFA8
:10AD00000FBE8DBFE0913816F0913916DF01A15EBC
:10AD1000B24F8C91882301F7E25EF24F4081EE51F1
:10AD2000FD40E41609F452CF2E2D332782E890E03F
:10AD3000289F8001299F100D389F100D11240C565B
:10AD4000154FBF01600F711F32E8F32E4F9DC001F8
:10AD500011248C56954F42E850E08E0F9F1F0E94A1
:10AD6000DD7E8091381690913916800F911F0E94D8
:10AD700013538091381690913916825E924FDC0100
:10AD8000EC918E519D40EF9DF0011124EC56F54F52
:10AD9000E80FF91FDF010D900020E9F71197AE1BB6
:10ADA000BF0B815E924FFC01A08310CF9A3019F047
:10ADB0009D3009F08FC0A0913816B0913916A15E70
:10ADC000B24F4C918E91AE51BD40992722E830E0B0
:10ADD000829FF001839FF00D929FF00D1124EA0FE6
:10ADE000FB1FE40FF11DEC56F54F108283E391E059
:10ADF0009F938F930E94D552E0913816F0913916A7
:10AE0000E15EF24F0F900F908081EF51FD4088235B
:10AE100009F45DC0E25EF24F80818F010E511D404A
:10AE200022E8829FC00111248C56954F080F191FEC
:10AE3000C8010E94E653882361F01F930F938CE1B1
:10AE400091E09F938F930E94D5520F900F900F9097
:10AE50000F90E0913816F0913916E25EF24F808142
:10AE60008F5F8083E0913816F0913916E25EF24FE1
:10AE70008081853019F4108221E0D22EE0913816BD
:10AE8000F0913916E25EF24FE190108220E030E05E
:10AE900042E850E0A0913816B0913916A25EB24F48
:10AEA0008C91AE51BD409927849FF001859FF00D94
:10AEB000949FF00D1124EA0FFB1FE20FF31FEC56D5
:10AEC000F54F10822F5F3F4F2238310519F70E944E
:10AED0007B537CCE983019F09F3709F044C0E09145
:10AEE0003816F0913916E15EF24F8081882309F41B
:10AEF0006DCE88E090E09F938F939F938F9386E130
:10AF000091E09F938F930E94D552E0913816F09173
:10AF10003916E15EF24F808181508083A09138160E
:10AF2000B0913916A15EB24F4C918E91AE51BD4099
:10AF3000992722E830E0829FF001839FF00D929FD5
:10AF4000F00D1124EA0FFB1FE40FF11DEC56F54F35
:10AF50001082FF248DB79EB706960FB6F8949EBF59
:10AF60000FBE8DBF34CEE0913816F091391699306E
:10AF7000C9F48F01015E124FE25EF24F8081EE5103
:10AF8000FD4022E8829FC00111248C56954F4F2D21
:10AF9000D8016C918E0F9F1F0E94EB54F8018083A3
:10AFA000F39415CEE15EF24F80818F3759F483E040
:10AFB00091E09F938F930E94D5520E9484530F90EB
:10AFC0000F9005CE892F99279F938F9380E091E072
:10AFD0009F938F930E94D552A0913816B091391645
:10AFE000A15EB24F4C918E91AE51BD40992722E89F
:10AFF00030E0829FF001839FF00D929FF00D1124AD
:10B00000EA0FFB1FE40FF11DEC56F54F8981808399
:10B01000E0913816F0913916E15EF24F80818F5F32
:10B020008083FF240F900F900F900F90D0CD9B0145
:10B03000882359F420503C4F40E050E068E278E526
:10B040008AE595E00E94340B08950E94D05508953A
:10B050000E94D055FFCF69E671E685E695E00E9433
:10B06000865408950F931F938C0187EC90E00E9403
:10B070004109FC0190933D1680933C16ED55FF4F1E
:10B0800085E08083E0913C16F0913D16EB53FF4F35
:10B09000118300831F910F910895CF93DF93CDB754
:10B0A000DEB728970FB6F894DEBF0FBECDBFE09194
:10B0B0003C16F0913D16EB53FF4FAE014F5F5F4FD3
:10B0C00060E070E0808191810E94F0278885992757
:10B0D0009F938F938F8199279F938F938E81992729
:10B0E0009F938F938D8199279F938F938C8199271D
:10B0F0009F938F938B8199279F938F938A81992711
:10B100009F938F93898199279F938F9388E695E0EA
:10B110009F938F930E9444528DB79EB742960FB66D
:10B12000F8949EBF0FBE8DBF28960FB6F894DEBF71
:10B130000FBECDBFDF91CF9108958FEA95E09F9329
:10B140008F930E94445289E596E09F938F930E94CB
:10B1500044520F900F900F900F900895FC01808142
:10B1600099279F938F93818199279F938F938281B2
:10B1700099279F938F93838199279F938F9384819E
:10B1800099279F938F93858199279F938F9387EC1E
:10B1900096E09F938F930E9444528DB79EB70E9670
:10B1A0000FB6F8949EBF0FBE8DBF089585EE96E052
:10B1B0009F938F930E944452E0913C16F0913D166C
:10B1C000EB53FF4F808191818A599C4F0E94AE586A
:10B1D00085EF96E09F938F930E9444520F900F90BB
:10B1E0000F900F9008950F931F93CF93DF93E091EB
:10B1F0003C16F0913D16EE55FF4F8081992787FD53
:10B2000090959F938F9387EF96E09F938F930E94E3
:10B210004452E0913C16F0913D16EE55FF4F0F90D1
:10B220000F900F900F90808187FF02C0108208C09E
:10B2300084E097E09F938F930E9444520F900F9069
:10B2400000E010E0C0E0D0E033C01F930F938CE229
:10B2500097E09F938F930E94445280913C16909167
:10B260003D168C0F9D1F0E94AE58E0913C16F09148
:10B270003D16EC0FFD1F858596859F938F938781E3
:10B280009085A185B285BF93AF939F938F9383E3FE
:10B2900097E09F938F930E9444520F5F1F4F2F960A
:10B2A0008DB79EB70C960FB6F8949EBF0FBE8DBF9C
:10B2B000E0913C16F0913D16EE55FF4F80819927A5
:10B2C00087FD9095081719070CF4BFCFDF91CF9138
:10B2D0001F910F910895CF93DF93CDB7DEB72897D5
:10B2E0000FB6F894DEBF0FBECDBFE0913C16F091D3
:10B2F0003D16EB53FF4FAE014F5F5F4F60E070E0D4
:10B30000808191810E9472288F8198859F938F936D
:10B310008D819E819F938F938C8199279F938F938B
:10B320008A819B819F938F93898199279F938F9384
:10B3300080E497E09F938F930E9444528DB79EB70D
:10B340000C960FB6F8949EBF0FBE8DBF28960FB611
:10B35000F894DEBF0FBECDBFDF91CF910895CF939C
:10B36000DF93CDB7DEB722970FB6F894DEBF0FBEDE
:10B37000CDBF9E012F5F3F4F3F932F932EE637E0C7
:10B380003F932F939F938F930E94FB712DB73EB7EE
:10B390002A5F3F4F0FB6F8943EBF0FBE2DBF0197F7
:10B3A00021F489818093A71402C00E949D5822969F
:10B3B0000FB6F894DEBF0FBECDBFDF91CF910895D9
:10B3C0000F931F93CF93DF93CDB7DEB724970FB6BC
:10B3D000F894DEBF0FBECDBF8C0143E050E061E7C3
:10B3E00077E00E94CF7E892BB9F5CE0101969F931D
:10B3F0008F9385E797E09F938F930C5F1F4F1F9369
:10B400000F930E94FB712DB73EB72A5F3F4F0FB6D7
:10B41000F8943EBF0FBE2DBF0197D9F429813A8120
:10B420004B815C81E0913C16F0913D16EB53FF4F50
:10B4300060E070E0808191810E94172061157105A4
:10B440008105910519F089E797E034C083E997E019
:10B4500031C083EA97E02EC043E050E062ED77E030
:10B46000C8010E94CF7E892B19F5E0913C16F0911E
:10B470003D16EB53FF4F60E070E0808191810E94A8
:10B48000882069837A838B839C839F938F937F9398
:10B490006F9386ED97E09F938F930E9444528DB7F0
:10B4A0009EB706960FB6F8949EBF0FBE8DBF08C01C
:10B4B0008AEE97E09F938F930E9444520F900F90D3
:10B4C00024960FB6F894DEBF0FBECDBFDF91CF91AB
:10B4D0001F910F9108950F931F93CF93DF93CDB7D3
:10B4E000DEB76E970FB6F894DEBF0FBECDBF8C01EE
:10B4F00043E050E061E777E00E94CF7E892BD1F4F2
:10B500000C5F1F4FE0913C16F0913D16EB53FF4F3F
:10B51000A80160E070E0808191810E94842561151E
:10B5200071058105910519F088E198E034C083E345
:10B5300098E031C043E050E062ED77E0C8010E943E
:10B54000CF7E892B31F5E0913C16F0913D16EB53FF
:10B55000FF4F2EE18E010F5F1F4FA80160E070E0EA
:10B56000808191810E949E2261157105810591055E
:10B5700019F084E498E00FC01F930F938EE598E0D4
:10B580009F938F930E9444520F900F900F900F90B3
:10B5900008C080E798E09F938F930E9444520F90D9
:10B5A0000F906E960FB6F894DEBF0FBECDBFDF9141
:10B5B000CF911F910F910895CF92DF92EF92FF925A
:10B5C0000F931F93CF93DF93E0913C16F0913D16BC
:10B5D000EB53FF4F0081118180EA98E09F938F9396
:10B5E0000E944452E801C758DD4FCC24DD240F905F
:10B5F0000F9089E8E82E82E0F82EE00EF11E035845
:10B600001D4F888199819F938F938DEC98E09F9334
:10B610008F930E9444528A819B819F938F9381EDE7
:10B6200098E09F938F930E944452C8010E94AE58A5
:10B63000898999279F938F9387ED98E09F938F93A4
:10B640000E944452F701808127E130E0E20EF31EB0
:10B6500082958F70837099279F938F938DED98E0DB
:10B660009F938F930E9410198DB79EB740960FB687
:10B67000F8949EBF0FBE8DBF8A89813051F0813012
:10B6800028F0823049F0833069F409C081EE98E0F7
:10B690000BC089EE98E008C08FEE98E005C086EFF9
:10B6A00098E002C08CEF98E09F938F930E944452E1
:10B6B0000F900F9085EF96E09F938F930E944452D6
:10B6C0000894C11CD11C095E1F4F67960F900F9004
:10B6D0009AE0C916D10409F094CFDF91CF911F9160
:10B6E0000F91FF90EF90DF90CF900895CF93DF936D
:10B6F000CDB7DEB722970FB6F894DEBF0FBECDBF31
:10B700009E012F5F3F4F3F932F932EE637E03F93ED
:10B710002F939F938F930E94FB712DB73EB72A5FA3
:10B720003F4F0FB6F8943EBF0FBE2DBF019759F59E
:10B7300089819A819F938F9385E099E09F938F935E
:10B740000E94445269817A81E0913C16F0913D1645
:10B75000EB53FF4F808191810E94CA2C0F900F9074
:10B760000F900F90611571058105910519F487E21D
:10B7700099E002C08FE299E09F938F930E94445218
:10B780000F900F9002C00E949D5822960FB6F89419
:10B79000DEBF0FBECDBFDF91CF910895CF93DF9372
:10B7A000CDB7DEB724970FB6F894DEBF0FBECDBF7E
:10B7B0009E012D5F3F4F3F932F939E012F5F3F4F81
:10B7C0003F932F9326E339E03F932F939F938F93DB
:10B7D0000E94FB712DB73EB7285F3F4F0FB6F8941C
:10B7E0003EBF0FBE2DBF029709F053C049815A8159
:10B7F000E0913C16F0913D16EB53FF4F2B8160E03A
:10B8000070E0808191810E94712C97FF1DC09B0187
:10B81000AC0188279927DC01821B930BA40BB50B85
:10B82000BF93AF939F938F938BE399E09F938F93F5
:10B830000E9444524DB75EB74A5F5F4F0FB6F8940F
:10B840005EBF0FBE4DBF2DC089819A819F938F939C
:10B850008EE599E09F938F930E94445269817A818B
:10B86000E0913C16F0913D16EB53FF4F80819181A2
:10B870000E94CA2C0F900F900F900F9061157105C8
:10B880008105910519F487E299E005C08FE299E0FE
:10B8900002C08DE799E09F938F930E9444520F90CE
:10B8A0000F9024960FB6F894DEBF0FBECDBFDF9188
:10B8B000CF9108950F931F93CF93DF93CDB7DEB74A
:10B8C00028970FB6F894DEBF0FBECDBF9E012F5F45
:10B8D0003F4F3F932F932EE637E03F932F939F9355
:10B8E0008F930E94FB712DB73EB72A5F3F4F0FB673
:10B8F000F8943EBF0FBE2DBF019709F072C0698159
:10B900007A81E0913C16F0913D16EB53FF4F808118
:10B9100091810E94A22D29813A81611571058105CD
:10B92000910529F03F932F9389EB99E01AC08E017E
:10B930000D5F1F4FE0913C16F0913D16EB53FF4F0A
:10B94000A801B901808191810E94BC2D611571050A
:10B950008105910579F089819A819F938F938FED6D
:10B9600099E09F938F930E9444520F900F900F90F5
:10B970000F9039C08FE09AE09F938F930E944452BA
:10B98000C8010E94AE5885EF96E09F938F930E9466
:10B99000445249815A81E0913C16F0913D16EB5397
:10B9A000FF4F23E160E070E0808191810E94EB43D2
:10B9B0000F900F900F900F90611571058105910503
:10B9C00039F089819A819F938F9385E29AE0C9CF5C
:10B9D00081E69AE09F938F930E9444520F900F90BC
:10B9E00002C00E949D5828960FB6F894DEBF0FBE85
:10B9F000CDBFDF91CF911F910F910895AF92BF926C
:10BA0000CF92EF92FF920F931F93CF93DF93CDB717
:10BA1000DEB728970FB6F894DEBF0FBECDBF7C010E
:10BA20008FEF9FEF9A83898380913C1690913D160A
:10BA30009C012B553F4F3F932F9389559F4F9F93C9
:10BA40008F9302969F938F9302969F938F93029664
:10BA50009F938F93265F3F4F3F932F9380E79AE00A
:10BA60009F938F93FF92EF920E94FB712DB73EB789
:10BA7000205F3F4F0FB6F8943EBF0FBE2DBF069715
:10BA8000C1F0CE0101969F938F938EE697E09F932E
:10BA90008F93FF92EF920E94FB714DB75EB74A5FA2
:10BAA0005F4F0FB6F8945EBF0FBE4DBF019709F010
:10BAB000C9C0E0913C16F0913D16EE55FF4F8081D4
:10BAC000992787FD909529813A81281739075CF0DD
:10BAD00088E89AE09F938F930E9444520E94F35803
:10BAE0000F900F90B1C08DEA9AE09F938F930E94C0
:10BAF000445289819A810F900F9020913C16309189
:10BB00003D165FEF8F3F9507A1F19CF10FE010E02C
:10BB1000AC01409FC001419F900D509F900D11249A
:10BB2000820F931F0E94AE5885EF96E09F938F93EC
:10BB30000E944452A0913C16B0913D1689819A8191
:10BB4000809FF001819FF00D909FF00D1124EA0F6E
:10BB5000FB1FE384F48406810F70AB53BF4F51E0A9
:10BB6000C52E28E134E0AF0160E070E08D919C913A
:10BB700033C01A821982F901EB55FF4F20E030E003
:10BB800043E0A42EB12CAC0EBD1ED50180818D9357
:10BB9000C90101969C01329686309105B9F79A83C6
:10BBA0008983C5010E94AE5885EF96E09F938F93DD
:10BBB0000E944452E0913C16F0913D16EB53FF4F2A
:10BBC00091E0C92EEE24FF2400E028E134E0A50135
:10BBD00060E070E0808191810E94B9460F900F90E3
:10BBE00097FF1DC09B01AC0188279927DC01821BB0
:10BBF000930BA40BB50BBF93AF939F938F938AEBDB
:10BC00009AE09F938F930E9444524DB75EB74A5F6C
:10BC10005F4F0FB6F8945EBF0FBE4DBF15C09F9328
:10BC20008F937F936F938DEC9AE09F938F930E94F5
:10BC300044528DB79EB706960FB6F8949EBF0FBEBE
:10BC40008DBF02C00E949D5828960FB6F894DEBFA3
:10BC50000FBECDBFDF91CF911F910F91FF90EF905D
:10BC6000CF90BF90AF900895CF92DF92EF92FF9266
:10BC70000F931F93CF93DF93CDB7DEB7A8970FB67F
:10BC8000F894DEBF0FBECDBF8C018FEF9FEF9A837C
:10BC900089839C838B8380913C1690913D169C01F7
:10BCA0002B553F4F3F932F9389559F4F9F938F93D2
:10BCB00002969F938F9302969F938F9302969F93E2
:10BCC0008F93265F3F4F3F932F9380E79AE09F9398
:10BCD0008F931F930F930E94FB712DB73EB7205F88
:10BCE0003F4F0FB6F8943EBF0FBE2DBF069779F1B8
:10BCF000CE0103969F938F9382EE9AE09F938F934A
:10BD00001F930F930E94FB712DB73EB72A5F3F4FE1
:10BD10000FB6F8943EBF0FBE2DBF0197C1F0CE0104
:10BD200001969F938F938EE697E09F938F931F9337
:10BD30000F930E94FB712DB73EB72A5F3F4F0FB69E
:10BD4000F8943EBF0FBE2DBF019709F0EFC02981C7
:10BD50003A81E0913C16F0913D16EE55FF4F8081FF
:10BD6000E25AF040992787FD9095281739074CF043
:10BD700086EE9AE09F938F930E9444520E94F3585C
:10BD8000DBC02F5F3F4F09F00CF43EC08DE09BE01D
:10BD90009F938F930E94445289819A810FE010E013
:10BDA0009C01209FC001219F900D309F900D112478
:10BDB00020913C1630913D16820F931F0E94AE5881
:10BDC00085EF96E09F938F930E944452A0913C167A
:10BDD000B0913D1689819A81809FF001819FF00D7D
:10BDE000909FF00D1124EA0FFB1F26812F704385D1
:10BDF0005485AB53BF4F1EE1E12E8E01055F1F4FEF
:10BE0000BF018D919C9158C06B817C813FEF6F3F4A
:10BE10007307D1F0CCF0EB53FF4FAE014B5F5F4F98
:10BE2000808191810E94BC2D6D5F7E4F8F4F9F4F0F
:10BE3000F1F48B819C819F938F938FE19BE09F9383
:10BE40008F930E9444526DC01A821982EB55FF4FA6
:10BE500020E030E0DE01159680818D93C9010196C6
:10BE60009C01329686309105B9F79A8389838DE0DB
:10BE70009BE09F938F930E94445275E0C72ED12C74
:10BE8000CC0EDD1EC6010E94AE5885EF96E09F9352
:10BE90008F930E944452E0913C16F0913D16EB5373
:10BEA000FF4F6EE1E62E8E01055F1F4F20E040E060
:10BEB00050E0B601808191810E9483447B018C0116
:10BEC0000F900F900F900F9097FF1AC08827992717
:10BED000DC018E199F09A00BB10BBF93AF939F9309
:10BEE0008F9384E49BE09F938F930E9444528DB77D
:10BEF0009EB706960FB6F8949EBF0FBE8DBF1EC0AC
:10BF000089E59BE09F938F930E9444526E2DCE0152
:10BF10000B960E94AF5287E69BE09F938F930E94FF
:10BF200044520F900F900F900F9008C08AE69BE04C
:10BF30009F938F930E9444520F900F90A8960FB634
:10BF4000F894DEBF0FBECDBFDF91CF911F910F914F
:10BF5000FF90EF90DF90CF900895EF92FF920F93B4
:10BF60001F93CF93DF93CDB7DEB722970FB6F89428
:10BF7000DEBF0FBECDBF8C0185E090E09A83898340
:10BF800044E050E06DEB7BE0C8010E94CF7E892B3E
:10BF900009F04AC0CE0101969F938F938EE697E0F9
:10BFA0009F938F930C5F1F4F1F930F930E94FB7102
:10BFB000E0913C16F0913D16ED55FF4F898180834D
:10BFC000E0913C16F0913D16ED55FF4F8081992789
:10BFD00087FD90959F938F9382EC9BE09F938F9327
:10BFE0000E944452E0903C16F0903D16F701EB534E
:10BFF000FF4F87012AE083EA90E0E80EF91ED7019F
:10C000004C9160E070E0808191810E94DB47F701F4
:10C0100062930E94F3588DB79EB70A960FB6F894B4
:10C020009EBF0FBE8DBFC5C045E050E065EE7BE012
:10C03000C8010E94CF7E892B09F04CC0E0913C16CC
:10C04000F0913D16EC55FF4F8081813019F48BEE55
:10C050009BE0A9C0CE0101969F938F938EE697E057
:10C060009F938F930B5F1F4F1F930F930E94FB7142
:10C07000E0913C16F0913D16ED55FF4F898180838C
:10C0800083E19CE09F938F930E944452E0913C1681
:10C09000F0913D16BF016A567F4FDF01AB53BF4F92
:10C0A0008F012AE0ED55FF4F40818D919C910E94B8
:10C0B000DB47E0913C16F0913D16EC55FF4F81E0D7
:10C0C0008083ADB7BEB718960FB6F894BEBF0FBE4B
:10C0D000ADBF6FC044E050E065E67CE0C8010E945F
:10C0E000CF7E892BC1F4E0913C16F0913D16EC55C2
:10C0F000FF4F8081E45AF040882311F1E056FF4F52
:10C10000808191818F5F9F4F19F482E99CE04BC041
:10C1100081EA9CE048C044E050E069EB7CE0C80163
:10C120000E94CF7E892BE9F500913C1610913D16B7
:10C130000C551F4FF8018081045A1040882319F4D0
:10C140008BE69CE030C00D551F4FD8016C917727CE
:10C1500067FD7095872F972F28EE33E040E050E081
:10C160000E94EC7EAB01BC01C80103970E946D0ADE
:10C17000E0913C16F0913D16E656FF4F80813896CF
:10C18000808382E99CE09F938F930E9444520E9497
:10C19000F358E0913C16F0913D16EC55FF4F10829C
:10C1A00006C080EC9CE09F938F930E9444520F90B6
:10C1B0000F9022960FB6F894DEBF0FBECDBFDF9171
:10C1C000CF911F910F91FF90EF900895CF93DF9340
:10C1D000CDB7DEB724970FB6F894DEBF0FBECDBF44
:10C1E0009E012D5F3F4F3F932F939E012F5F3F4F47
:10C1F0003F932F9326E339E03F932F939F938F93A1
:10C200000E94FB712DB73EB7285F3F4F0FB6F894E1
:10C210003EBF0FBE2DBF029709F050C089819A81A1
:10C220009F938F9380E39DE09F938F930E9444524E
:10C230002B813C8180E496E0A901489F9001499FB1
:10C24000300D589F300D112449815A81E0913C16E0
:10C25000F0913D16EB53FF4F60E070E080819181DB
:10C260000E9468240F900F900F900F9097FF1DC0B1
:10C270009B01AC0188279927DC01821B930BA40B3F
:10C28000B50BBF93AF939F938F9383E59DE09F93EF
:10C290008F930E9444524DB75EB74A5F5F4F0FB60F
:10C2A000F8945EBF0FBE4DBF0BC089E69DE09F9323
:10C2B0008F930E9444520F900F9002C00E949D588D
:10C2C00024960FB6F894DEBF0FBECDBFDF91CF919D
:10C2D0000895CF93DF93EC0144E050E06DE77DE0FB
:10C2E0000E94CF7E892B19F40E94D658B2C048E034
:10C2F00050E062E87DE0CE010E94CF7E892B19F4E8
:10C300000E94DC5AA6C049E050E06BE87DE0CE0117
:10C310000E94CF7E892B29F4CE010A960E94AF5944
:10C3200098C049E050E065E97DE0CE010E94CF7EF3
:10C33000892B29F4CE010A960E94E6608AC043E068
:10C3400050E06FE97DE0CE010E94CF7E892B29F479
:10C35000CE0104960E94FE5C7CC046E050E063EA99
:10C360007DE0CE010E94CF7E892B29F4CE01079675
:10C370000E945A5C6EC047E050E06AEA7DE0CE0160
:10C380000E94CF7E892B29F4CE0108960E94AD5FD2
:10C3900060C044E050E062EB7DE0CE010E94CF7EC1
:10C3A000892B29F4CE0105960E946B5A52C043E0B6
:10C3B00050E067EB7DE0CE010E94CF7E892B29F40F
:10C3C000CE0104960E94E05944C045E050E06BEB7A
:10C3D0007DE0CE010E94CF7E892B29F4CE01069606
:10C3E0000E94345E36C047E050E061EC7DE0CE0153
:10C3F0000E94CF7E892B29F4CE0108960E94CE5B45
:10C4000028C044E050E069EC7DE0CE010E94CF7E80
:10C41000892B29F4CE0105960E94765B1AC048E06C
:10C4200050E06EEC7DE0CE010E94CF7E892B19F4A6
:10C430000E944D580EC047E050E067ED7DE0CE0110
:10C440000E94CF7E892B19F40E946B5902C00E9472
:10C450009D58DF91CF91089569E372E68FED9DE0DD
:10C460000E94865469EF72E683EE9DE00E94865436
:10C470000895AF92BF92CF92DF92EF92FF920F9307
:10C480001F93CF93DF93CDB7DEB72A970FB6F894FB
:10C49000DEBF0FBECDBF8C011A86198629E0A22E01
:10C4A000B12CAC0EBD1EBF92AF92CE0101969F93F0
:10C4B0008F9395E0C92ED12CCC0EDD1EDF92CF924A
:10C4C000CE0103969F938F9387EE9DE09F938F936A
:10C4D0001F930F930E94FB712DB73EB7245F3F4F10
:10C4E0000FB6F8943EBF0FBE2DBF03973CF02D81D1
:10C4F0004B81698589810E948A4A6AC04AE050E07E
:10C5000067EF7DE0C8010E94CF7E892B19F40E945D
:10C510002D4B5EC087E0E82EF12CEC0EFD1EFF9245
:10C52000EF9282E09EE09F938F931F930F930E9460
:10C53000FB712DB73EB72A5F3F4F0FB6F8943EBF51
:10C540000FBE2DBF019721F48F810E94CE4A40C0BB
:10C55000FF92EF9287E09EE09F938F931F930F933C
:10C560000E94FB712DB73EB72A5F3F4F0FB6F8947C
:10C570003EBF0FBE2DBF019721F48F810E94B64AA6
:10C5800027C0DF92CF92FF92EF92BF92AF928DE0E1
:10C590009EE09F938F931F930F930E94FB712DB783
:10C5A0003EB7265F3F4F0FB6F8943EBF0FBE2DBF7C
:10C5B000039731F44D816F8189850E94AF4A08C08D
:10C5C00086E19EE09F938F930E9444520F900F90BC
:10C5D0002A960FB6F894DEBF0FBECDBFDF91CF9184
:10C5E0001F910F91FF90EF90DF90CF90BF90AF9091
:10C5F00008958AE090E00E94C4759C0168EE73E0A3
:10C600000E94177F6AE070E00E94177F7F936F930C
:10C61000C90168EE73E00E94177F7F936F9380EBF0
:10C620009EE09F938F930E9444528DB79EB70696CB
:10C630000FB6F8949EBF0FBE8DBF08956EE273E6ED
:10C640008DEC9EE00E948654089582E092E09F93D4
:10C650008F930E94D5520F900F900895CF93DF9340
:10C66000EC0147E050E061ED7EE00E94CF7E892B37
:10C6700039F480913A1690913B160E94C86A2AC0FC
:10C6800046E050E069ED7EE0CE010E94CF7E892B2E
:10C6900039F480913A1690913B160E94466A1AC06E
:10C6A00044E050E060EE7EE0CE010E94CF7E892B18
:10C6B00079F40E943C099F938F9381EE91E09F93C0
:10C6C0008F930E94D5520F900F900F900F9002C041
:10C6D0000E942563DF91CF910895E82F81508F311B
:10C6E00018F08FEF9FEF0895FF27E25CF94E628309
:10C6F00080E090E0089590933F1680933E16E0E42A
:10C70000F6E1119286E1E036F807D9F765E974E6BB
:10C7100085EE9EE00E948654089540E456E160E074
:10C7200070E089E895E60E943C4D089589EE9EE010
:10C730009F938F930E94445285EF9EE09F938F9327
:10C740000E94445289E19FE09F938F930E9444523C
:10C750008AE49FE09F938F930E94445281E59FE07B
:10C760009F938F930E9444528BE69FE09F938F93F9
:10C770000E94445289E79FE09F938F930E94445206
:10C7800085E99FE09F938F930E94445286EA9FE041
:10C790009F938F930E94445288EB9FE09F938F93C7
:10C7A0000E9444528DB79EB744960FB6F8949EBF30
:10C7B0000FBE8DBF08950F931F93CF93DF93CDB717
:10C7C000DEB724970FB6F894DEBF0FBECDBF8C0145
:10C7D0001A8219828FEF90E09C838B8342E050E0B5
:10C7E00067EC7FE0C8010E94CF7E892BB1F440E462
:10C7F00056E160E070E089E895E60E943C4D892BA7
:10C8000019F48AEC9FE002C089ED9FE09F938F931B
:10C810000E9444520F900F907DC044E050E061E0D0
:10C8200070E1C8010E94CF7E892B29F40E94554DEA
:10C8300085E090E1EBCF43E050E065E170E1C801B5
:10C840000E94CF7E892B29F40E94624D8BE190E1FA
:10C85000DDCF45E050E06EE270E1C8010E94CF7E7E
:10C86000892B29F40E94A34D85E390E1CFCFCE011F
:10C8700003969F938F93CE0101969F938F9389E4A4
:10C8800090E19F938F931F930F930E94FB712DB79D
:10C890003EB7285F3F4F0FB6F8943EBF0FBE2DBF87
:10C8A00082309105A1F4E981FA81CF0101974F9778
:10C8B00028F4E25CF94E8B8182830CC08EE490E117
:10C8C0009F938F930E9444520F900F9003C01816AD
:10C8D0001906F4F429813A81C90101974F97C0F4F0
:10C8E000F901E25CF94E828199279F938F933F93E0
:10C8F0002F9387E690E19F938F930E9444528DB7C8
:10C900009EB706960FB6F8949EBF0FBE8DBF02C0AD
:10C910000E94966324960FB6F894DEBF0FBECDBF7B
:10C92000DF91CF911F910F9108950F931F93CF9394
:10C93000DF93CDB7DEB728970FB6F894DEBF0FBEF2
:10C94000CDBF8C011A8219828FEF90E09C838B837C
:10C950001E821D8218861F8244E050E062E970E169
:10C96000C8010E94CF7E892B51F5CE0103969F937B
:10C970008F93CE0101969F938F93CE0105969F933F
:10C980008F9387E990E19F938F930C5F1F4F1F93C5
:10C990000F930E94FB7100E010E029E835E64B811F
:10C9A00069818D819E810E94D24E2DB73EB7265F50
:10C9B0003F4F0FB6F8943EBF0FBE2DBF9FC043E060
:10C9C00050E06EE970E1C8010E94CF7E892B41F5ED
:10C9D000CE0103969F938F93CE0101969F938F93E1
:10C9E000CE0105969F938F93CE0107969F938F93C9
:10C9F00082EA90E19F938F930D5F1F4F1F930F93D8
:10CA00000E94FB716D817E8120E030E049E855E6AF
:10CA10008F8198850E945F4E8DB79EB70C9658C047
:10CA200045E050E06BEA70E1C8010E94CF7E892B9F
:10CA300019F40E944C4F62C047E050E061EB70E196
:10CA4000C8010E94CF7E892B09F048C0CE01039611
:10CA50009F938F93CE0101969F938F9389E490E1EA
:10CA60009F938F93095F1F4F1F930F930E94FB713A
:10CA70002DB73EB7285F3F4F0FB6F8943EBF0FBEAD
:10CA80002DBF8230910529F46B8189810E94334D3D
:10CA900003C01816190684F589810E94264D9C83CF
:10CAA0008B8389819A819F938F9389EB90E19F93E8
:10CAB0008F930E9444528B819C819F938F9388EC2B
:10CAC00090E19F938F930E9444528DB79EB7089632
:10CAD0000FB6F8949EBF0FBE8DBF10C049E050E066
:10CAE0006FED70E1C8010E94CF7E892B29F4C80147
:10CAF0000A960E94DB6302C00E94966328960FB6D6
:10CB0000F894DEBF0FBECDBFDF91CF911F910F9183
:10CB10000895EF92FF920F931F93CF93DF937C01C1
:10CB20008B010E943B52E801EB81FF27EE0FFF1FB4
:10CB3000E350FF4E808191819F938F938A81992743
:10CB40009F938F938C819D81AE81BF81BF93AF9363
:10CB50009F938F93888199819F938F9389EE90E122
:10CB60009F938F9380913E1690913F169F938F9342
:10CB70000E94D67160913E1670913F16C7010E94C7
:10CB8000F41D0E943252EDB7FEB73E960FB6F894F0
:10CB9000FEBF0FBEEDBFDF91CF911F910F91FF90B0
:10CBA000EF900895E0913C16F0913D16EB53FF4F46
:10CBB00080819181009761F040E050E060E070E09A
:10CBC0000E941B796CE079E68FE191E10E94865426
:10CBD0000895CF93DF93EC018881882309F45DC029
:10CBE0008AE090E00E94F471E0913C16F0913D16CD
:10CBF000EB53FF4F0190F081E02D81E0818BE091BC
:10CC00003C16F0913D16EB53FF4F0190F081E02D63
:10CC10008CEF838BE0913C16F0913D16EB53FF4F68
:10CC20000190F081E02D86E0828BE0913C16F0913E
:10CC30003D16EB53FF4FA081B181FE010190002012
:10CC4000E9F78E2F8C1BFD01848BE0913C16F0914F
:10CC50003D16EB53FF4F0190F081E02D448955279D
:10CC6000BE01CF0145960E94DD7EE0913C16F09119
:10CC70003D16EB53FF4F80819181BC016F5E7F4F6A
:10CC80000E949C3268E873E180E090E00E947B069D
:10CC90008AE090E00E94F47108C083E291E19F93E2
:10CCA0008F930E9444520F900F90DF91CF9108957F
:10CCB00081E591E19F938F930E9444520F900F90D2
:10CCC0000895E0913C16F0913D16EB53FF4F8081A3
:10CCD00091810E94A12F0895E0913C16F0913D169C
:10CCE000EB53FF4F0190F081E02DEB5BFD4F808116
:10CCF000E554F240882349F08CED91E19F938F93A6
:10CD00000E9444520F900F90089562E0CF010E945C
:10CD10004448E0913C16F0913D16EB53FF4F808163
:10CD200091810E948F2E0895CF93DF93CDB7DEB708
:10CD300024970FB6F894DEBF0FBECDBF9E012D5FC6
:10CD40003F4F3F932F939E012F5F3F4F3F932F9372
:10CD500021EF31E13F932F939F938F930E94FB71BB
:10CD60002DB73EB7285F3F4F0FB6F8943EBF0FBEBA
:10CD70002DBF0297C9F489819A8182309105A0F470
:10CD80004B815C814230510578F4440F480FE091AB
:10CD90003C16F0913D16EB53FF4F60E070E0808150
:10CDA00091810E94C52008C086EF91E19F938F93E7
:10CDB0000E9444520F900F9024960FB6F894DEBF55
:10CDC0000FBECDBFDF91CF910895CF93DF93CDB745
:10CDD000DEB722970FB6F894DEBF0FBECDBF9E011F
:10CDE0002F5F3F4F3F932F9326E432E13F932F93E2
:10CDF0009F938F930E94FB712DB73EB72A5F3F4FE1
:10CE00000FB6F8943EBF0FBE2DBF019781F4898104
:10CE10009A818230910558F4009719F0019779F4BE
:10CE200003C00E943B7B0BC00E94617B08C089E469
:10CE300092E19F938F930E9444520F900F902296FD
:10CE40000FB6F894DEBF0FBECDBFDF91CF9108952E
:10CE50000F931F93CF93DF93CDB7DEB724970FB611
:10CE6000F894DEBF0FBECDBF9E012D5F3F4F3F93B5
:10CE70002F939E012F5F3F4F3F932F9321EF31E17F
:10CE80003F932F939F938F930E94FB719C01019777
:10CE90004DB75EB7485F5F4F0FB6F8945EBF0FBEE9
:10CEA0004DBF0297F0F449815A81E0913C16F09110
:10CEB0003D162130310549F4EB53FF4F60E070E03F
:10CEC000808191810E94BB2815C02B813C81EB534E
:10CED000FF4F890160E070E0808191810E941429F8
:10CEE00009C080E792E19F938F930E9444520F9074
:10CEF0000F9040C09B01AC012F3F8FEF38078FEFA1
:10CF000048078FEF5807E9F0E4F0BB2757FDBA95C3
:10CF1000A52F942F832F9F938F93C90190709F9378
:10CF20008F9384EB92E19F938F930E9444524DB76D
:10CF30005EB74A5F5F4F0FB6F8945EBF0FBE4DBF3E
:10CF400019C088279927DC01821B930BA40BB50B12
:10CF5000BF93AF939F938F9389ED92E19F938F93AC
:10CF60000E9444528DB79EB706960FB6F8949EBFA6
:10CF70000FBE8DBF24960FB6F894DEBF0FBECDBF97
:10CF8000DF91CF911F910F910895CF92DF92EF9291
:10CF9000FF920F931F93CF93DF93CDB7DEB7289700
:10CFA0000FB6F894DEBF0FBECDBF9E01295F3F4F85
:10CFB0003F932F939E012B5F3F4F3F932F939E01F3
:10CFC0002D5F3F4F3F932F939E012F5F3F4F3F9326
:10CFD0002F932EEF32E13F932F939F938F930E94D5
:10CFE000FB712DB73EB7245F3F4F0FB6F8943EBF9D
:10CFF0000FBE2DBF8130910519F0049731F50FC098
:10D0000049815A81E0913C16F0913D16EB53FF4F58
:10D0100060E070E0808191810E947F291FC02B8198
:10D020003C81CF80D884ED80FE8049815A81E09197
:10D030003C16F0913D16EB53FF4F890160E070E024
:10D04000808191810E94D82909C087E093E19F9354
:10D050008F930E9444520F900F9040C09B01AC01EF
:10D060002F3F8FEF38078FEF48078FEF5807E9F012
:10D07000E4F0BB2757FDBA95A52F942F832F9F93DC
:10D080008F93C90190709F938F938CE593E19F9349
:10D090008F930E9444522DB73EB72A5F3F4F0FB681
:10D0A000F8943EBF0FBE2DBF19C088279927DC0119
:10D0B000821B930BA40BB50BBF93AF939F938F93DE
:10D0C00082E893E19F938F930E9444528DB79EB75D
:10D0D00006960FB6F8949EBF0FBE8DBF28960FB66A
:10D0E000F894DEBF0FBECDBFDF91CF911F910F919E
:10D0F000FF90EF90DF90CF9008950F931F93CF9301
:10D10000DF93CDB7DEB724970FB6F894DEBF0FBE1E
:10D11000CDBF9E012D5F3F4F3F932F939E012F5F09
:10D120003F4F3F932F9321EF31E13F932F939F93F5
:10D130008F930E94FB712DB73EB7285F3F4F0FB60C
:10D14000F8943EBF0FBE2DBF029709F052C02B814D
:10D150003C8149815A81E0913C16F0913D16EB5398
:10D16000FF4F890160E070E0808191810E94522A26
:10D170009B01AC012F3F8FEF38078FEF48078FEFF0
:10D180005807E9F0E4F0BB2757FDBA95A52F942F77
:10D19000832F9F938F93C90190709F938F9385EAFC
:10D1A00093E19F938F930E9444522DB73EB72A5F1D
:10D1B0003F4F0FB6F8943EBF0FBE2DBF22C0882749
:10D1C0009927DC01821B930BA40BB50BBF93AF9384
:10D1D0009F938F9382E893E19F938F930E94445291
:10D1E0008DB79EB706960FB6F8949EBF0FBE8DBF43
:10D1F00008C08AEC93E19F938F930E9444520F9052
:10D200000F9024960FB6F894DEBF0FBECDBFDF910E
:10D21000CF911F910F910895CF93DF93EC0144E0DC
:10D2200050E065EF73E10E94CF7E892B29F4CE0197
:10D2300005960E947D6860C045E050E06AEF73E1AA
:10D24000CE010E94CF7E892B29F4CE0106960E9442
:10D25000C56752C044E050E060E074E1CE010E9436
:10D26000CF7E892B29F4CE0105960E94286744C001
:10D2700042E050E065E074E1CE010E94CF7E892B50
:10D2800029F4CE0103960E94E56636C044E050E0E2
:10D2900069E074E1CE010E94CF7E892B29F4CE0192
:10D2A00005960E94946628C045E050E06EE074E167
:10D2B000CE010E94CF7E892B19F40E946C661CC09F
:10D2C00048E050E064E174E1CE010E94CF7E892BFA
:10D2D00019F40E94616610C047E050E06DE174E10E
:10D2E000CE010E94CF7E892B29F4CE0108960E94A0
:10D2F000E96502C00E945866DF91CF91089560935E
:10D30000DD157093DE158093DF159093E015409343
:10D310006016089580916016813089F40E946E0530
:10D320009B01AC018091DD159091DE15A091DF1578
:10D33000B091E015280F391F4A1F5B1F10C00E94D3
:10D340006E059B01AC018091DD159091DE15A091D9
:10D35000DF15B091E015281B390B4A0B5B0BCA0196
:10D36000B90108950E946E050895009729F09093E1
:10D3700062168093611606C08091611690916216C4
:10D38000892B19F06093651608951092651608951B
:10D39000009729F0909364168093631606C08091DD
:10D3A000631690916416892B19F0609366160895A0
:10D3B000109266160895EF92FF920F931F93CF93EA
:10D3C000DF938C01BC018AE090E00E94CC1DC091EB
:10D3D0000816D0910916EE24FF2422C08881998175
:10D3E000E80EF91E9F938F93DF93CF9385E692E02B
:10D3F0009F938F931F930F930E946974CE01805661
:10D4000090402DB73EB7285F3F4F0FB6F8943EBF10
:10D410000FBE2DBF805A9F4728F40A80DB81C02DA4
:10D420002097E1F60E943C098E159F05A9F09F9375
:10D430008F93FF92EF9288E492E09F938F931F93D4
:10D440000F930E9469748DB79EB708960FB6F89433
:10D450009EBF0FBE8DBF13C09F938F9389E392E051
:10D460009F938F931F930F930E9469742DB73EB7BC
:10D470002A5F3F4F0FB6F8943EBF0FBE2DBFDF911E
:10D48000CF911F910F91FF90EF9008950F931F93ED
:10D49000CF93DF938C01C091FA15D091FB152097A3
:10D4A00009F471C0BC018BE892E00E948774888502
:10D4B0009985AA85BB85BF93AF939F938F938C81EA
:10D4C0009D81AE81BF81BF93AF939F938F93DF9375
:10D4D000CF938DE792E09F938F931F930F930E94BA
:10D4E00069748C859D852DB73EB7225F3F4F0FB67F
:10D4F000F8943EBF0FBE2DBF37E08A35930721F465
:10D50000B80186EB92E007C02AE08532920731F439
:10D51000B80186EA92E00E9487741AC0AA27BB2746
:10D52000880F991FAA1FBB1FBF93AF939F938F9321
:10D5300087E792E09F938F931F930F930E946974E4
:10D540008DB79EB708960FB6F8949EBF0FBE8DBFDD
:10D550008E859F859F938F938FE692E09F938F9305
:10D560001F930F930E9469740990D881C02D2DB725
:10D570003EB72A5F3F4F0FB6F8943EBF0FBE2DBF98
:10D58000209709F094CFDF91CF911F910F910895CB
:10D59000EF92FF920F931F93CF93DF937C01BC0117
:10D5A00084EC92E00E948774C0910016D09101161D
:10D5B0007AC0EB89FC8980819181A281B3818F5EE1
:10D5C0009E4BAD4ABE4D19F085E294E102C08AE25D
:10D5D00094E1288939894F89588D9F938F93C90188
:10D5E0008E1B9F0B9F938F933F932F938D899E89C3
:10D5F0009F938F935F934F93EF85FF27EE0FFF1F4E
:10D60000E05BFB4E808191819F938F938A8999275C
:10D610009F938F932696DF93CF932697DF93CF9395
:10D620008AEF92E09F938F93FF92EF920E9469742A
:10D630008F89988DEDB7FEB776960FB6F894FEBF3A
:10D640000FBEEDBF892B39F1EF89F88D0081118173
:10D65000FFEF0F3F1F07E1F4B7018DE294E10E9455
:10D66000F41D19C01F930F9384EF92E09F938F9343
:10D67000FF92EF920E946974F801028113812DB725
:10D680003EB72A5F3F4F0FB6F8943EBF0FBE2DBF87
:10D690000115110539F7B7018AE090E00E94CC1D11
:10D6A0000990D881C02D209709F083CFDF91CF91C9
:10D6B0001F910F91FF90EF9008950F931F93CF93B9
:10D6C000DF938C01EB016F5F7F4F09F06BC0BC01F2
:10D6D00086E394E10E94F41D68C0EB89FC89808197
:10D6E0009181A281B3818F5E9E4BAD4ABE4DF1F018
:10D6F00084819581A681B7818F5E9E4BAD4ABE4DD8
:10D70000A9F080859185A285B3858F5E9E4BAD4A39
:10D71000BE4D61F084859585A685B7858F5E9E4B4D
:10D72000AD4ABE4D19F085E294E102C08AE294E16F
:10D73000288939894F89588D9F938F93C9018E1BF2
:10D740009F0B9F938F933F932F938D899E899F93D8
:10D750008F935F934F93EF85FF27EE0FFF1FE05BE3
:10D76000FB4E808191819F938F938A8999279F9304
:10D770008F932696DF93CF932697DF93CF9381E203
:10D7800093E09F938F931F930F930E9469740A8075
:10D79000DB81C02D8DB79EB746960FB6F8949EBF1D
:10D7A0000FBE8DBF209709F098CFDF91CF911F91C9
:10D7B0000F910895FC011382128215821482118246
:10D7C00010820895FC0184819581892B61F022816A
:10D7D000338180910416909105162817390719F0A6
:10D7E0008FEF9FEF089580E090E00895FC01228183
:10D7F000338180910416909105162817390719F086
:10D800008FEF9FEF0895848195810197958384839D
:10D81000892B19F080E090E00895CF010E941A0A48
:10D8200080E090E00895CF93DF93EC012A813B8163
:10D8300080910416909105162817390741F40BC002
:10D8400040E050E060E070E0CE010E94D60A8C819A
:10D850009D81892BA9F780910416909105169B83D1
:10D860008A838C819D8101969D838C83DF91CF91EA
:10D870000895FC0184819581892B61F02281338197
:10D8800080910416909105162817390719F08FEF2B
:10D890009FEF0895CF010E94136C80E090E00895FF
:10D8A0000F931F93CF93DF93FC01C189D289EDA918
:10D8B000FEA909958C01892B49F4CF5BDF4FE881E4
:10D8C000F98160E072EC81E090E00995C801DF9198
:10D8D000CF911F910F910895CF93DF93EC01EA81CF
:10D8E000FB810188F289E02D0FB6F8940F9264A5B0
:10D8F00075A50F900FBE88279927DF91CF910895C6
:10D90000CF92DF92EF92FF920F931F93CF93DF930B
:10D91000EC018B017A0169018C819D812885398513
:10D920000FB6F8940F92198618860F900FBE26171F
:10D93000370789F0232B21F0009711F00E94261A57
:10D940000115110509F1C8010E94291A009729F44F
:10D950008FEF9FEF1BC0672BB9F09D838C8399835A
:10D9600088839B838A83800F911F9F838E83FD868C
:10D97000EC86DF86CE861B861A860FB6F8940F9249
:10D98000198708870F900FBE80E090E0DF91CF915C
:10D990001F910F91FF90EF90DF90CF900895CF925D
:10D9A000DF92EF92FF920F931F93CF93DF938A0141
:10D9B000DA01CD90DD90ED90FC902C2DFC01C18919
:10D9C000D289F1E067307F0709F464C081E06830F4
:10D9D0007807ECF491E06330790709F44AC0A1E0DC
:10D9E00064307A0754F4B1E061307B0799F1E1E0EB
:10D9F00062307E0709F0CCC030C0F1E065307F07AF
:10DA000009F442C0665071400CF041C03AC091E048
:10DA10006B30790709F4A8C0A1E06C307A0754F4A0
:10DA2000B1E069307B0709F441C06A5071400CF0E5
:10DA300076C033C0F1E06D307F0709F49FC081E00C
:10DA40006D3078070CF495C091E06E30790709F0DD
:10DA50009FC099C0CF5BDF4F5FC0CD5BDF4FE881D8
:10DA6000F9810995D8016D937D938D939C931397BC
:10DA700036C1CB5BDF4FE881F9818C2D09958C0194
:10DA800030C1C95BDF4F0BC0C75BDF4FF4CFC55B55
:10DA9000DF4F05C0C35BDF4FEECFC15BDF4FE881D7
:10DAA000F98109959927AA27BB2714C1C6FC03C091
:10DAB00000E010E011C0FE01B2962685378544854E
:10DAC000558560857185CF010E94806C8C01892B02
:10DAD00019F4EBADFCAD0995C7FE10C00115110599
:10DAE00009F0FFC0FE01709626853785448555856F
:10DAF00060857185CF010E94806C8C010115110534
:10DB000009F0EFC0CF5ADF4F8FE39FEFAFEFBFEFCA
:10DB1000C822D922EA22FB22E881F9815DC0CD5AD0
:10DB2000DF4FE881F981C355D04009959B01AC01D5
:10DB3000D8016D937D938D939C9313978CA59DA590
:10DB4000892B31F42064F80120833183428353838D
:10DB50008A8D9B8D892B09F0C2C0F801808191814B
:10DB6000A281B3818068B7C0C886D986EA86FB8661
:10DB7000B6C088859985AA85BB85ACC0CC86DD8674
:10DB8000EE86FF86ACC08C859D85AE85BF85A2C024
:10DB9000FB01EF50F140E931F10540F4EA5BFF4F42
:10DBA000EE0FFF1F0590F491E02D09940FEF1FEF8A
:10DBB00098C088819981AA81BB81222311F0806459
:10DBC00022C08F7B20C088819981AA81BB8186FF7A
:10DBD00027C021C0EDADFEADC701B60109954FCFFD
:10DBE000EF96E881F9810995F8016083718382835A
:10DBF000938375C088819981AA81BB81222311F00A
:10DC0000806801C08F7788839983AA83BB8367C0AC
:10DC1000888187FF05C081E090E0A0E0B0E05AC0B5
:10DC2000D8011D921D921D921C92139758C0CB5A79
:10DC3000DF4FE881F981822F21CFC95ADF4F2FCFE3
:10DC4000FE0170962685378544855585B601CF013E
:10DC50000E94806C8C01892B09F043C0EBADFCADB8
:10DC600009953FC0888D998D33C0FE01B2962685F7
:10DC7000378544855585B601CF010E94806CFFCE63
:10DC80008AA59BA525C00FB6F8940F92DD8ECC8E89
:10DC90001AC08C8D9D8D1CC00FB6F8940F92DF8E2C
:10DCA000CE8E11C08E8D9F8D13C00FB6F8940F923B
:10DCB000DFA6CEA608C08EA59FA50AC00FB6F89411
:10DCC0000F92D9AAC8AA0F900FBE09C088A999A916
:10DCD000AA27BB27F80180839183A283B38300E046
:10DCE00010E0C801DF91CF911F910F91FF90EF904D
:10DCF000DF90CF900895CF92DF92EF92FF920F9333
:10DD00001F93CF93DF936C018A01FC01C189D289F3
:10DD100083E0E82EF12CE422F522E114F10481F0F5
:10DD200028E330E048E250E060E470E0CE01409645
:10DD30000E94806C892BA1F4F1E0EF16F10499F0B8
:10DD400020EF30E040ED50E060E071E0CE018296DF
:10DD50000E94806C892B39F08C899D890E94261A3B
:10DD60000FEF1FEF2CC086E090E00E94291A009769
:10DD700039F48C899D890E94261A8EA19FA1EECF2D
:10DD80000070107C288139814A815B8100501048E5
:10DD900011F42F7701C02068288339834A835B837D
:10DDA0008C01FC0111821082D382C28215821482FE
:10DDB000F1E0EF16F10419F0EBADFCAD0995C801E7
:10DDC000DF91CF911F910F91FF90EF90DF90CF9057
:10DDD0000895CF93DF93DC01EC01EA81FB81C189D7
:10DDE000D28901978E5F9F4F18F08FEF9FEF19C078
:10DDF000CD010E94261A20E030E040E050E060E0D3
:10DE000070E0CE0140960E94806C20E030E040E05F
:10DE100050E060E070E0CE0182960E94806C80E06D
:10DE200090E0DF91CF910895CF92DF92EF92FF9231
:10DE30000F931F93CF93DF937C016A01EC016096EF
:10DE40000FB6F8940F928A859B85860F971F9B8744
:10DE50008A8713C0F70181AD92ADFC010995F701E6
:10DE60004485558566857785CE0140960E946D0A6A
:10DE7000892B51F40FB6F8940F920A851B850F90E9
:10DE80000FBEC016D10630F3C801DF91CF911F91AC
:10DE90000F91FF90EF90DF90CF9008956F927F9257
:10DEA0008F929F92AF92BF92CF92DF92EF92FF92AA
:10DEB0000F931F93CF93DF93CDB7DEB722970FB6A3
:10DEC000F894DEBF0FBECDBF4A015901FC01E188C5
:10DED000F288A0E16A2E712C6E0C7F1CF301808504
:10DEE0009185892B21F4FFEFCF2EDF2E9BC061158A
:10DEF000710549F440E050E060E070E0C7010E9425
:10DF0000146F6C018FC0F70180819181A281B38170
:10DF10009C01AD01E9E05695479537952795EA951F
:10DF2000D1F721702A8327E0B695A7959795879515
:10DF30002A95D1F7817089830FB6F8940F92F30177
:10DF4000428553850F900FBE8B0160E070E0CC24BA
:10DF5000DD2450C09A01260F371FF301868597856F
:10DF60002817390778F044855585C7010E94146F3A
:10DF7000AC01F301848595858417950708F452C098
:10DF800060E070E0A114B10419F0F801849102C0BE
:10DF9000D8018C91B981B13069F48A3081F4EA8179
:10DFA000E13019F0F2E0F98303C082E08A838983CB
:10DFB0008DE00AC09981923011F4A1E0A9830F5F2E
:10DFC0001F4F0894C11CD11CD301ED91FC911197F6
:10DFD00081931196FC93EE932D913C91F3018681F0
:10DFE00097812817390721F4848195819183808353
:10DFF0006F5F7F4FC814D9040CF4ACCF6115710565
:10E0000089F00FB6F8940F92F30182859385860FFD
:10E01000971F938782870F900FBEF70181AD92AD56
:10E02000FC010995C60122960FB6F894DEBF0FBE1B
:10E03000CDBFDF91CF911F910F91FF90EF90DF90B7
:10E04000CF90BF90AF909F908F907F906F900895EA
:10E0500021E030E0FC01828193810E944E6F08959F
:10E0600020E030E0FC01828193810E944E6F089590
:10E07000AF92BF92CF92DF92EF92FF920F931F93D6
:10E08000CF93DF937B015A01EC01EA81FB81018987
:10E090001289E801A296688579856115710519F4E0
:10E0A0008FEF9FEFA1C0E114F10461F42E853F854D
:10E0B0004C855D85CE010E94806CE801EBADFCAD26
:10E0C00009951AC00FB6F8940F926A857B850F9058
:10E0D0000FBE6115710599F4F80183AD94ADFC0193
:10E0E0000995F8014085518562857385CE0140967A
:10E0F0000E946D0A892B31F380E090E075C0D70152
:10E10000F801808187FF35C0CC24DD24EE24FF2474
:10E110005AE02BC0E616F70609F44FC0EA81FB81EE
:10E120004191FB83EA832A813B818E819F8128175D
:10E13000390721F48C819D819B838A834D3011F0B6
:10E140004A3051F4F80184A9882311F0841751F45E
:10E15000F80144AB5D9303C0F80114AA4D930894F1
:10E16000C11CD11C0894E11CF11CCA14DB0490F200
:10E1700021C06B01A616B70608F4650140E050E027
:10E18000D70114C0EA81FB8181918C93FB83EA83E0
:10E190002A813B818E819F812817390721F48C8148
:10E1A0009D819B838A834F5F5F4F11964C155D0560
:10E1B00049F77601E114F104B1F00FB6F8940F922B
:10E1C0008A859B858E199F099B878A870F900FBE32
:10E1D0002A853B858C859D852817390720F4E80121
:10E1E000EBADFCAD0995C601DF91CF911F910F9169
:10E1F000FF90EF90DF90CF90BF90AF900895CF93B6
:10E20000DF93DC01EC01EA81FB81309719F08D91FD
:10E210009C910995DF91CF910895EF92FF920F9312
:10E220001F93CF93DF93EC017B018A01EC81FD8189
:10E23000309719F480E090E005C060E070E080E085
:10E2400090E0099519830883FB82EA82DF91CF91E0
:10E250001F910F91FF90EF900895CF93DF93EC0102
:10E26000EC81FD81309719F48FEF9FEF05C060E0DE
:10E2700070E081E190E00995DF91CF910895CF930F
:10E28000DF93EC01EC81FD81309719F48FEF9FEF64
:10E2900005C060E070E082E190E00995DF91CF91E8
:10E2A00008950F931F93CF93DF93CDB7DEB72497D5
:10E2B0000FB6F894DEBF0FBECDBF8C017C836B839D
:10E2C000FC01248135812115310519F48FEF9FEF71
:10E2D00017C0BE016F5F7F4F80E290E0F9010995A2
:10E2E000009771F4F80124813581BE016D5F7F4F85
:10E2F00081E290E0F9010995009711F489819A81F2
:10E3000024960FB6F894DEBF0FBECDBFDF91CF913C
:10E310001F910F9108950F931F93CF93DF93CDB764
:10E32000DEB724970FB6F894DEBF0FBECDBF8C01C9
:10E330007C836B83FC01248135812115310519F41F
:10E340008FEF9FEF17C0BE016F5F7F4F88E190E0B6
:10E35000F9010995009771F4F80124813581BE0116
:10E360006D5F7F4F89E190E0F9010995009711F405
:10E3700089819A8124960FB6F894DEBF0FBECDBF77
:10E38000DF91CF911F910F910895FC0140E050E083
:10E3900060E070E0808191810E94131A892B19F04E
:10E3A0008FEF9FEF089580E090E00895CF93DF9383
:10E3B000CDB7DEB722970FB6F894DEBF0FBECDBF44
:10E3C000AE01455F5F4F5A83498369857A858F81A6
:10E3D00098850E94651922960FB6F894DEBF0FBE8D
:10E3E000CDBFDF91CF910895609151047091520497
:10E3F0000E94CC1D0895CF93DF93CDB7DEB722974F
:10E400000FB6F894DEBF0FBECDBFAE01455F5F4FC4
:10E410005A83498369857A858F8198850E943072F5
:10E4200022960FB6F894DEBF0FBECDBFDF91CF911D
:10E430000895CF93DF93EC0180E090E0DB0105C00D
:10E440002D933196F983E88301968417950729F077
:10E45000E881F9812081222399F7DF91CF910895F6
:10E46000CF93DF93CDB7DEB722970FB6F894DEBF18
:10E470000FBECDBF9A019A838983AB01BE016F5F46
:10E480007F4F89E192E70E94617222960FB6F8945D
:10E49000DEBF0FBECDBFDF91CF910895CF93DF9345
:10E4A000DC01EC01EA81FB81309719F4ED81FE81FA
:10E4B00003C00788F08DE02DCD010995DF91CF9144
:10E4C00008952F923F924F925F926F927F928F9218
:10E4D0009F92AF92BF92CF92DF92EF92FF920F93F3
:10E4E0001F93CF93DF93CDB7DEB763970FB6F89442
:10E4F000DEBF0FBECDBF3C014B012A0159012224D2
:10E500003324FF24D2011C91112309F494C10894EF
:10E51000411C511C812F99270E94857F892B99F0DE
:10E5200041E050E0BE016F5F7F4FC401F3010995E8
:10E53000019741F7898199270E94857F892B81F76F
:10E54000A1E0FA2EDFCF153289F0FF2059F441E027
:10E5500050E0BE016F5F7F4FC401F3010995019741
:10E5600009F0A5C08981811761F265C1F20181912D
:10E570002F01853291F4FF2059F441E050E0BE01B3
:10E580006F5F7F4FC401F3010995019709F08FC0B8
:10E590008981853209F4B5CF4EC1982FCC24DD2472
:10E5A00000E02AE030E09A3211F4026016C09C3696
:10E5B00011F4016012C0892F80538A3090F4A601B3
:10E5C000429F6001439FD00C529FD00C1124C90E72
:10E5D000D11C80ED9FEFC80ED91ED2019D912D0157
:10E5E000E2CF9F3609F450C1903748F4933609F4CE
:10E5F0004FC1993661F0992309F443C149C093375B
:10E6000021F0983709F044C005C012E042C013E081
:10E61000EE2441C0006113E0F0E1EF2E3CC001FDAB
:10E6200012C024C0FF2059F440E150E0BE016E5FEB
:10E630007F4FC401F301099518161906C4F5E0EFE0
:10E64000FFEFCE0EDF1EF1E1CF16D10458F7FF2009
:10E6500009F07EC0A601BE016E5F7F4FC401F301C9
:10E660000995181619060CF473C021C0FF2009F093
:10E670006EC0D5016D917C91A601C401F30109958D
:10E6800018161906A4F4E2E0F0E0AE0EBF1E5FC05B
:10E6900013E0EAE0EE2EFF2071F441E050E0BE010D
:10E6A0006F5F7F4FC401F3010995019721F022208C
:10E6B00009F4E7C0C0C0F9808F2D99270E94857F9B
:10E6C000892B59F7123009F048C0C114D10419F44C
:10E6D0007FEFC72ED72E01FF17C00894C108D108BD
:10E6E000C114D104A9F141E050E0BE016F5F7F4F3A
:10E6F000C401F3010995019759F5898199270E9471
:10E70000857F892B29F5E9CFD5010D911C91F80161
:10E71000F1928F010894C108D108C114D10489F085
:10E7200041E050E0BE016F5F7F4FC401F3010995E6
:10E73000019739F4F9808F2D99270E94857F892BC5
:10E7400031F342E050E0A40EB51ED8011C92339480
:10E750002394D7CE61E0F62E6AC0133009F0D1CEF3
:10E76000C60101970F9718F05FE0C52ED12C102F2E
:10E770001C62FE013296FB8BEA8B54C09981903368
:10E7800049F4EE2019F4106148E0E42E15FF20C092
:10E79000137D32C0892F8153873018F4EE20C1F4E5
:10E7A00006C0892F8853823048F4EE2019F43AE0ED
:10E7B000E32E0EC0F8E0FE15C8F50AC0892F81547B
:10E7C000863018F08052863028F44AE04E1570F5F5
:10E7D000137E12C09D3211F09B3221F412FF26C02D
:10E7E0001B7F0AC0983719F0983509F0B3CF14FF92
:10E7F0001DC01F7E20E1E22EAA89BB899D93BB8BA1
:10E80000AA8BB2E0CB16D10450F041E050E0BE013B
:10E810006F5F7F4FC401F3010995019739F40894A4
:10E82000C108D108C114D10409F0A8CFFF24012FD9
:10E83000112703FF03C0832D992732C001FD1FC09C
:10E84000EA89FB8910824E2D552760E070E0CE01E9
:10E8500002960E94507D95012E5F3F4F00FF08C039
:10E86000D501ED91FC91608371838283938305C010
:10E87000D501ED91FC917183608359013394239408
:10E8800041CE8FEF9FEF0CC013E098E0E92E03CF4D
:10E89000C114D10409F0C3CE81E0C82ED12CBFCE63
:10E8A00063960FB6F894DEBF0FBECDBFDF91CF9158
:10E8B0001F910F91FF90EF90DF90CF90BF90AF909E
:10E8C0009F908F907F906F905F904F903F902F9090
:10E8D0000895CF93DF93CDB7DEB722970FB6F894A4
:10E8E000DEBF0FBECDBFAE01455F5F4F5A83498388
:10E8F00069857A858F8198850E94BB7422960FB6B0
:10E90000F894DEBF0FBECDBFDF91CF910895EF9297
:10E91000FF920F931F938C017B010E94917EAC01AB
:10E92000B801F701808191810E94F4741F910F91C9
:10E93000FF90EF900895CF93DF93CDB7DEB7229786
:10E940000FB6F894DEBF0FBECDBFFE0137966191C2
:10E950007191FA83E983AF0180915104909152043F
:10E960000E94BB7422960FB6F894DEBF0FBECDBFD7
:10E97000DF91CF910895AF92BF92CF92DF92EF9245
:10E98000FF920F931F93CF93DF935C017B016A018A
:10E99000CB010E94917E8C010F5F1F4FC8010E9426
:10E9A0005508EC01009719F40FEF1FEF11C0A801F3
:10E9B000B7010E947D7EF501608171819601AE01F3
:10E9C00083E19AE10E945E1A8C01CE010E94C80880
:10E9D000C801DF91CF911F910F91FF90EF90DF90D1
:10E9E000CF90BF90AF900895CF93DF93DC01EC01FF
:10E9F000EA81FB81309719F4E985FA8503C0038C1D
:10EA0000F48DE02DCD010995DF91CF9108950F93FD
:10EA10001F9300E010E023E030E046E050E060E0CB
:10EA200070E080E090E00E94697B9093E315809312
:10EA3000E21581E08093E1151F910F9108956F9287
:10EA40007F928F929F92AF92BF92CF92DF92EF927E
:10EA5000FF920F931F93CF93DF93CDB7DEB7C456CA
:10EA6000D0400FB6F894DEBF0FBECDBF8091E11548
:10EA7000882311F40E9407758E010F5F1F4F80914C
:10EA8000E2159091E3150E94817BF80181939193A7
:10EA90008F010E943D08CE018B599F4F081719071F
:10EAA00071F720E030E040E050E0FE013196B8011F
:10EAB00081919191AA27BB27280F391F4A1F5B1FFD
:10EAC000E617F707A9F7CA01B90122E330E040E0F1
:10EAD00050E00E944C7F49015A01CA01B90128EC5B
:10EAE00039E140E050E00E94EC7E2AE09595879560
:10EAF000779567952A95D1F7645F71408040904083
:10EB00005CF1EE24FF2487016E010894C11CD11C26
:10EB100085E6682E712C6C0E7D1EF6018191919117
:10EB20006F01AA27BB27A5019401281B390B4A0BAB
:10EB30005B0BCA01B9010E94EC7EE60EF71E081FAE
:10EB4000191FC614D70449F780E090E0F2E3EF16EE
:10EB5000F1040105110514F481E090E0CC59DF4F78
:10EB60000FB6F894DEBF0FBECDBFDF91CF911F91DE
:10EB70000F91FF90EF90DF90CF90BF90AF909F905C
:10EB80008F907F906F900895CF92DF92EF92FF92D7
:10EB90000F931F93CF93DF93EC010E940775CE0173
:10EBA0000A978B35910510F0CAE0D0E0CC24DD2423
:10EBB000EE24FF24870111C08091E2159091E315A6
:10EBC0000E94817BAA27BB27E80EF91E0A1F1B1F84
:10EBD0000E943D080894C11CD11CCC16DD0664F3CC
:10EBE000C801B70128EC39E140E050E00E94EC7E1A
:10EBF0009E01442737FD4095542F0E944C7FDA0137
:10EC0000C9013AE0B595A795979587953A95D1F7BB
:10EC1000DF91CF911F910F91FF90EF90DF90CF90F8
:10EC20000895882321F0813011F0823019F40E9478
:10EC30007C4A0895833011F40E947C4A0895882309
:10EC400021F0813011F0823019F40E946F4A08954A
:10EC5000833011F40E946F4A08950E94694A80E04F
:10EC60000E94117681E00E94117682E00E94117666
:10EC700083E00E9411760895DC01CB0120E030E0B2
:10EC800066277727480F591F6A1F7B1F40505D4C2E
:10EC90006240704010F021E030E0C901089520E0AA
:10ECA0003FEE40E050E00E942A7F2F5F822F99279D
:10ECB000089520E03FEE40E050E00E942A7FDC0112
:10ECC000CB0180509F4E089520E03FEE40E050E0A1
:10ECD0000E942A7F9B01AC0180E09FEE821B930B78
:10ECE00008957F928F929F92AF92BF92CF92DF92C0
:10ECF000EF92FF920F931F93CF93DF93EC015A0192
:10ED00006B014901790100271127E40EF51E061F4A
:10ED1000171F20E0E2162DECF20622E0020720E0A9
:10ED2000120708F05FC061C0272D33278F2D992768
:10ED300001972817390709F055C0C601B5010E948F
:10ED400064768C01C601B5010E94597622E07216E4
:10ED500061F023E0721671F021E0721609F042C0F2
:10ED6000A801BE010E94767809C0A801BE010E94D8
:10ED7000867804C0A801BE010E949678272D33270B
:10ED80008F2D992701972817390749F582E0F81642
:10ED900089F023E0F216C9F081E0F81619F5801A1F
:10EDA000910AC00FD11FA401BE0180E091E10E9431
:10EDB000767815C0801A910AC00FD11FA401BE0138
:10EDC00080E091E10E9486780AC0801A910AC00F03
:10EDD000D11FA401BE0180E091E10E94967880E0FD
:10EDE00090E012C081E090E00FC0CB01BA010E9418
:10EDF0004F76782EC801B7010E944F76F82E78160C
:10EE000009F092CF84019ECFDF91CF911F910F9196
:10EE1000FF90EF90DF90CF90BF90AF909F908F903A
:10EE20007F9008957F928F929F92AF92BF92CF92E0
:10EE3000DF92EF92FF920F931F93CF93DF934C01DA
:10EE40005A016B01E901790100271127E40EF51E33
:10EE5000061F171F80E0E8168DECF80682E0080711
:10EE600080E0180708F060C062C0272D33278F2D7F
:10EE7000992701972817390709F056C0C601B5012F
:10EE80000E9464768C01C601B5010E945976BC01CE
:10EE900082E0781661F083E0781671F081E07816F0
:10EEA00009F042C0A801C4010E94A87809C0A801C5
:10EEB000C4010E94B87804C0A801C4010E94C878A7
:10EEC000272D33278F2D992701972817390749F5C3
:10EED00082E0F81689F083E0F816C9F081E0F816B0
:10EEE00019F5C01BD10BAE0160E071E1C401800FC8
:10EEF000911F0E94A87815C0C01BD10BAE0160E025
:10EF000071E1C401800F911F0E94B8780AC0C01B34
:10EF1000D10BAE0160E071E1C401800F911F0E942E
:10EF2000C87880E090E012C081E090E00FC0CB0193
:10EF3000BA010E944F76782EC801B7010E944F7621
:10EF4000F82E781609F091CF8E019DCFDF91CF91E9
:10EF50001F910F91FF90EF90DF90CF90BF90AF90F7
:10EF60009F908F907F9008952F923F924F925F9243
:10EF70006F927F928F929F92AF92BF92CF92DF92C9
:10EF8000EF92FF920F931F93CF93DF93CDB7DEB72E
:10EF9000E2970FB6F894DEBF0FBECDBF49015A010C
:10EFA000AB01BC01222433244BC082E3C82ED12CF8
:10EFB000E12CF12CC40ED51EE61EF71ED701C601AA
:10EFC0008C149D04AE04BF0410F4D501C4012C01BF
:10EFD0003D01441A550A660A770A92018E010F5FB5
:10EFE0001F4FC8010E94127740E050E060E070E0DF
:10EFF000D8011FC0FD01E40FF51F80812826222DB6
:10F0000022952225022E269526952025022E26952C
:10F0100020252770022C232C269507942795302C29
:10F02000222606942795302422264F5F5F4F6F4F8C
:10F030007F4F4415550566057705E1F6B701A60132
:10F04000481559056A057B0508F4AFCFC101E29662
:10F050000FB6F894DEBF0FBECDBFDF91CF911F91E9
:10F060000F91FF90EF90DF90CF90BF90AF909F9067
:10F070008F907F906F905F904F903F902F9008956A
:10F08000EF92FF920F931F93CF93DF93CDB7DEB72D
:10F0900022970FB6F894DEBF0FBECDBF79018A016B
:10F0A0000E94B4778983892F99278A8322E030E0F0
:10F0B000B801A701CE0101960E94717622960FB683
:10F0C000F894DEBF0FBECDBFDF91CF911F910F919E
:10F0D000FF90EF9008952E5F3F4F4F4F5F4F0E947C
:10F0E000B477009711F081E090E00895FB01DC0116
:10F0F000E89447F4689406C0F8940190C79A0D927A
:10F10000C798789441505040B8F70895FB01DC014E
:10F11000E89447F4689406C0F8940190C69A0D925A
:10F12000C698789441505040B8F70895FB01DC012F
:10F13000E89457F4689408C0F8940190C79AC69A66
:10F140000D92C798C698789441505040A8F70895FA
:10F15000FB01DC01E89447F4689406C0F894C79A70
:10F160000190C7980D92789441505040B8F7089597
:10F17000FB01DC01E89447F4689406C0F894C69A51
:10F180000190C6980D92789441505040B8F7089578
:10F19000FB01DC01E89457F4689408C0F894C79A1E
:10F1A000C69A0190C798C6980D92789441505040E5
:10F1B000A8F70895E091E415F091E51581E090E05D
:10F1C000A0E0B0E08787908BA18BB28B838B948B70
:10F1D000A58BB68B80E197E2A0E0B0E0878F90A38B
:10F1E000A1A3B2A388EE93E0A0E0B0E0838F948F58
:10F1F000A58FB68F84E690E0A0E0B0E0878B908F7B
:10F20000A18FB28F80E092E0A0E0B0E083A394A34E
:10F21000A5A3B6A388E090E0A0E0B0E087A390A704
:10F22000A1A7B2A780E190E0A0E0B0E083A794A7F7
:10F23000A5A7B6A70895EF92FF920F931F93CF93C0
:10F24000DF93EC017A018B018091E4159091E51533
:10F25000892B19F081E090E045C060E070E0CE01BC
:10F260000E94BD2A97FF03C08FEF9FEF3BC062FD56
:10F2700003C08EEF9FEF36C08FE290E00E945508EA
:10F28000FC019093E5158093E415892B19F48DEF1B
:10F290009FEF28C0D183C083E282F3820483158369
:10F2A000178216821486118610861586138612869A
:10F2B00016860E94DA7820E031E040E050E06AE40F
:10F2C0007AE788E594E10E94340B892B19F080E0FD
:10F2D00090E008C08091E4159091E5150E94C8085F
:10F2E0008CEF9FEFDF91CF911F910F91FF90EF90E7
:10F2F00008950F931F93CF93DF93EC01162F042FE4
:10F30000E091E415F091E515BC01808191810E94A6
:10F31000EF2C9B01AC012D3F8EEF38078FEF480794
:10F320008FEF580709F45CC0307040705070812F27
:10F33000992787FD9095A92FB92F281739074A07D4
:10F340005B0709F04DC00F3F09F44DC0E091E41593
:10F35000F091E515BE01808191810E94CA2C9B012C
:10F36000AC012D3F8EEF38078FEF48078FEF58071E
:10F37000E9F1307040705070802F992787FD90958B
:10F38000A92FB92F281739074A075B0779F5E091AC
:10F39000E415F091E51582819381A481B5810097F0
:10F3A000A105B10501F1BE01808191810E94222D4C
:10F3B0009B01AC012D3F8EEF38078FEF48078FEF91
:10F3C0005807B9F0E091E415F091E5158281938139
:10F3D000A481B581281739074A075B0751F403C098
:10F3E0008FEF90E008C080E090E005C08EEF90E0E5
:10F3F00002C08DEF90E0DF91CF911F910F910895A2
:10F40000EF92FF920F931F93CF93DF93CDB7DEB7A9
:10F4100064970FB6F894DEBF0FBECDBFE091E41540
:10F42000F091E515BE016F5F7F4F808191810E9451
:10F43000432DE62EFF241FC00F2D1127000F111F93
:10F44000CE010196080F191F4FEF62E0F80180818D
:10F4500091810E947979882369F4F8014081518172
:10F46000E091E415F091E51560E070E08081918114
:10F470000E947F29F394FE14F9F664960FB6F8946F
:10F48000DEBF0FBECDBFDF91CF911F910F91FF90D7
:10F49000EF900895CF93DF93CDB7DEB764970FB6A3
:10F4A000F894DEBF0FBECDBFE091E415F091E515F5
:10F4B00087890E94B907E091E415F091E515168659
:10F4C00040E050E060E070E0CF0106960E946D0AD7
:10F4D000E091E415F091E51581E08487E091E41571
:10F4E000F091E515BE016F5F7F4F808191810E9491
:10F4F000432D962EFF24AA2437C00F2D1127000F6D
:10F50000111FCE010196080F191FD8016D917C9132
:10F51000E091E415F091E515808191810E94EF2C36
:10F520006D3FBEEF7B07BFEF8B07BFEF9B07D9F0A7
:10F530006230C9F4F80160817181E091E415F091C5
:10F54000E515808191810E94CA2CE091E415F0912B
:10F55000E51523893489458956896217730784071D
:10F56000950709F4A394F394F91439F6BB2456C013
:10F57000E091E415F091E5152A2D3327442755270E
:10F5800087859089A189B289281739074A075B07BF
:10F5900008F047C00B2D1127000F111FCE01019657
:10F5A000080F191F438960E0D8018D919C910E943A
:10F5B0007979882391F5E091E415F091E515438D73
:10F5C000548D658D768DCF0108960E946D0AE0916D
:10F5D000E415F091E515892B61F486858823D1F532
:10F5E00040E050E060E070E0CF010A960E946D0AB2
:10F5F00018C023A134A1C3A4D4A4E7A0F0A4D801C7
:10F600004D915C91890160E070E0808191810E9460
:10F61000D82997FD02C0623021F0B394B91409F0E3
:10F62000A7CFE091E415F091E5158685882391F444
:10F63000478D50A161A172A1CF0108960E946D0A69
:10F64000892B09F04BCFE091E415F091E515868503
:10F65000882341F00E94007AE091E415F091E515CD
:10F66000148629CF40E050E060E070E0CF010A96B8
:10F670000E946D0A33CFE091E415F091E515848581
:10F68000882331F081E08687CF0108960E941A0A0C
:10F690000895E091E415F091E5158485882321F023
:10F6A000CF010A960E941A0A0895E091E415F0919C
:10F6B000E5158485882321F0CF0108960E941A0A57
:10F6C00008958091E4159091E51506960E941A0A16
:10F6D00008950F931F93682B642B202B0FB6F8947B
:10F6E0000F92379866B927B9379A0F900FBE822FBD
:10F6F0009927982F88277727862B972B1F910F9173
:10F700000895AC01692F77270FB6F8940F9287B14F
:10F7100026B1861719F42F76241721F0379846B9A9
:10F7200067B9379A369A3699FECF84B125B10F90D2
:10F730000FBE99273327322F2227822B932B089530
:10F74000DF92EF92FF920F931F93CF93DF93CDB78A
:10F75000DEB724970FB6F894DEBF0FBECDBF8C0185
:10F760007E010894E11CF11CA7016AE071E00E948F
:10F77000A91929813A814B815C81DA01C90187701D
:10F780009070A070B0700097A105B10511F4DD2450
:10F7900011C087E0D82ED22287E090E0A0E0B0E050
:10F7A00089839A83AB83BC83A70169E071E0C801B8
:10F7B0000E94A9198D2D992724960FB6F894DEBFC3
:10F7C0000FBECDBFDF91CF911F910F91FF90EF90B2
:10F7D000DF900895CF92DF92EF92FF920F931F93E5
:10F7E000CF93DF936C01EB01E42EFF243BC08E012D
:10F7F000020F131FC6010E94451841E050E0B801F6
:10F800000E944E72F8010081083011F00F3761F448
:10F81000FF2041F18CE594E19F938F930E94445225
:10F82000FA940F900F901EC00A3011F00D3049F479
:10F8300080E694E19F938F930E9444520F900F9023
:10F840001AC0802F992787FD90959F938F9382E60A
:10F8500094E19F938F930E944452F3940F900F90E2
:10F860000F900F902F2D33278E2D99270197281752
:10F8700039070CF4BCCFCF0DD11D1882F3948F2D16
:10F880009927DF91CF911F910F91FF90EF90DF901B
:10F89000CF900895FC01808199279F938F93818158
:10F8A00099279F938F93828199279F938F93838129
:10F8B00099279F938F93848199279F938F93858115
:10F8C00099279F938F9385E694E19F938F930E944E
:10F8D00044528DB79EB70E960FB6F8949EBF0FBEDA
:10F8E0008DBF08955F926F927F928F929F92AF9299
:10F8F000BF92CF92DF92EF92FF920F931F93CF931D
:10F90000DF934C013B01EC0101C0219688818032DC
:10F91000E1F3530195E0592E1881E12EFF24E7FC15
:10F92000F094C7010E947B7F892B89F10981C02E49
:10F93000DD24C7FCD094C6010E947B7F892B39F15E
:10F940001A3314F4105305C0C7010E94947F182F76
:10F9500017550A331CF4802F805304C0C6010E943F
:10F96000947F87551295107F182BF5011583CE01D2
:10F9700002965520A9F08A818A3349F423965A9435
:10F980000894A108B108FFEF5F1659F0C5CFF30145
:10F99000A1EAB4E186E00D900192815019F0FBCF0D
:10F9A000EC014E01C401DF91CF911F910F91FF90A7
:10F9B000EF90DF90CF90BF90AF909F908F907F900F
:10F9C0006F905F9008950F931F93FC01808199279A
:10F9D0009F938F93818199279F938F9382819927FA
:10F9E0009F938F93838199279F938F9384819927E6
:10F9F0009F938F93858199279F938F9385E694E1B9
:10FA00009F938F9306EE15E11F930F930E94471962
:10FA10008DB79EB740960FB6F8949EBF0FBE8DBFB0
:10FA2000C8011F910F910895AF92BF92CF92DF92BC
:10FA3000EF92FF920F931F93CF93DF937C015B01B3
:10FA40006A01EC0100E010E018C0EA0DFB1D8081A6
:10FA500099279F938F9383E894E19F938F93DF93EC
:10FA6000CF930E944719C80FD91F8DB79EB706962E
:10FA70000FB6F8949EBF0FBE8DBFE02FFF270F5F1C
:10FA80001F4FEC15FD0508F3C701DF91CF911F91C2
:10FA90000F91FF90EF90DF90CF90BF90AF900895BF
:10FAA0003F924F925F926F927F928F929F92AF920E
:10FAB000BF92CF92DF92EF92FF920F931F93CF935B
:10FAC000DF938C012B01EA016115710519F0FB012F
:10FAD00091838083209749F0CE010297839728F085
:10FAE00060E070E080E090E0F6C0F801E1908F0106
:10FAF0008E2D99270E94857F892BB9F7FDE2EF169D
:10FB000031F4F801E1908F0181E0382E07C0FBE26B
:10FB1000EF1619F4F801E1908F013324209719F0C2
:10FB2000C031D105C1F4F0E3EF1679F4F80180811A
:10FB3000883711F0883549F4F801E1800E5F1F4FD6
:10FB4000F2E03F2AC0E1D0E006C0209721F480E334
:10FB5000E816E9F427C0C830D10531F1C930D10524
:10FB600024F4C230D10531F50CC0CA30D10589F07A
:10FB7000C031D105F9F4A12CB12CC12CB8E0DB2E99
:10FB800026C0A12CB12CC12CA0E4DA2E20C0CAE0E2
:10FB9000D0E0FCECAF2EFCECBF2EFCECCF2EFCE05A
:10FBA000DF2E15C0C8E0D0E0A12CB12CC12CE0E1C3
:10FBB000DE2E0DC09E01442737FD4095542F60E096
:10FBC00070E080E090E80E942A7F59016A0120E0FD
:10FBD00030E040E050E060E03E01882477FC809413
:10FBE000982C70EDF72EFE0CE9E0EF1570F48E2DD9
:10FBF00081548A3118F499ECF92E06C08E2D815665
:10FC00008A3150F589EAF82EFE0C8F2D99278C1732
:10FC10009D0714F567FD1CC0A216B306C406D506E1
:10FC2000B0F0CA01B901A40193010E94EC7E9B01CE
:10FC3000AC012F0D311D411D511D2130F0E03F075A
:10FC4000F0E04F07F0E85F0710F461E001C06FEFEC
:10FC5000F801E1908F01C5CF4114510481F0662372
:10FC600031F001501040F2011183008308C031FED1
:10FC70001AC002501040F2011183008314C067FFC4
:10FC800012C030FE05C020E030E040E050E804C083
:10FC90002FEF3FEF4FEF5FE782E290E0909368161F
:10FCA0008093671616C030FE08C050954095309579
:10FCB00021953F4F4F4F5F4F0CC057FF0AC082E264
:10FCC00090E090936816809367162FEF3FEF4FEF09
:10FCD0005FE7CA01B901DF91CF911F910F91FF90AA
:10FCE000EF90DF90CF90BF90AF909F908F907F90DC
:10FCF0006F905F904F903F900895FB01DC0140FFB3
:10FD000005C002C005900D9205900D9242505040E2
:10FD1000C8F70895FB01DC0105900D920020E1F782
:10FD20000895FC0105900020E9F7809590958E0FCD
:10FD30009F1F0895FC014150504030F0019006167D
:10FD4000D1F73197CF010895882799270895FB01AE
:10FD5000DC0140FF05C002C001900D9201900D92A0
:10FD600042505040C8F70895DC0140FF03C001C075
:10FD70006D936D9342505040D8F70895FB01DC011C
:10FD80008D910190801911F40020D1F7990B0895FD
:10FD9000FB01DC0101900D920020E1F70895FB01C9
:10FDA000DC014150504030F08D910190801919F4E0
:10FDB0000020B9F7881B990B0895FB01DC01415025
:10FDC000504048F001900D920020C9F701C01D92EB
:10FDD00041505040E0F70895629FD001739FF001B9
:10FDE000829FE00DF11D649FE00DF11D929FF00DCB
:10FDF000839FF00D749FF00D659FF00D9927729F02
:10FE0000B00DE11DF91F639FB00DE11DF91FBD018C
:10FE1000CF0111240895991B79E004C0991F96170A
:10FE200008F0961B881F7A95C9F78095089597FB6F
:10FE3000092E07260AD077FD04D049D006D000202D
:10FE40001AF4709561957F4F0895F6F79095819516
:10FE50009F4F0895A1E21A2EAA1BBB1BFD010DC0E6
:10FE6000AA1FBB1FEE1FFF1FA217B307E407F5076A
:10FE700020F0A21BB30BE40BF50B661F771F881F46
:10FE8000991F1A9469F760957095809590959B01DC
:10FE9000AC01BD01CF01089597FB092E05260ED0B8
:10FEA00057FD04D0D7DF0AD0001C38F45095409598
:10FEB000309521953F4F4F4F5F4F0895F6F790953E
:10FEC0008095709561957F4F8F4F9F4F0895AA1B26
:10FED000BB1B51E107C0AA1FBB1FA617B70710F035
:10FEE000A61BB70B881F991F5A95A9F78095909567
:10FEF000BC01CD010895082E8062813624F087363A
:10FF00000CF408952BC0802D36C0911127C080328B
:10FF100051F08A3041F08C3031F08D3021F0893051
:10FF200011F08B3099F708958F931DD08F9109F0C0
:10FF300080620895E199FECFBFBBAEBBE09A1196F7
:10FF40000DB20895E199FECFBFBBAEBB0DBA1196BD
:10FF50000FB6F894E29AE19A0FBE08959927882780
:10FF6000089585FDFBCF80629111F8CF8136ECF3C7
:10FF70008B37DCF708959111F1CF80538A50E0F769
:02FF80000895E2
:10FF8200722B000A23202D2D2D2D2D2D2D2D2D2DC3
:10FF92002D2D2D2D2D2D2D2D2D2D2D2D2D2D2D2D8F
:10FFA2002D2D2D2D2D2D2D2D2D2D2D2D2D2D2D2D7F
:10FFB2002D2D2D2D2D2D2D2D2D2D2D2D000A2320D6
:10FFC20057656C636F6D6520746F2042546E757453
:10FFD20020286329203230303620455448205A7573
:10FFE200726963680032303036313231382D313542
:0EFFF200313800232062742D636D642070721C
:020000021000EC
:100000006F6772616D2076657273696F6E3A202535
:10001000730A002449643A2062742D636D642E6370
:100020002C7620312E343820323030362F31322F9A
:1000300031352031323A32343A31332079756563C3
:10004000656C6D20457870202400232025730A00FC
:10005000232072756E6E696E6720402025752E25EF
:10006000303475204D487A2C204E75744672657177
:100070003D25756C20487A0A0023202D2D2D2D2D2D
:100080002D2D2D2D2D2D2D2D2D2D2D2D2D2D2D2DA0
:100090002D2D2D2D2D2D2D2D2D2D2D2D2D2D2D2D90
:1000A0002D2D2D2D2D2D2D2D2D2D2D2D2D2D2D2D80
:1000B000000A626F6F74696E6720426C7565746FB9
:1000C0006F7468206D6F64756C652E2E2E00426C07
:1000D0007565746F6F7468204D414320616464726C
:1000E0006573733A20252E34783A252E34783A25D4
:1000F0002E34780A004843492076657273696F6E22
:100100003A20255820252E345820255820252E34D5
:100110005820252E34580A004C4D502066656174D5
:10012000757265733A20252E325820252E325820BC
:10013000252E325820252E325820252E32582025A3
:100140002E325820252E325820252E32580A004CA7
:100150006F63616C206E616D653A20272573270AF5
:100160000062742D636D642064656D6F006869744E
:100170002074616220747769636520666F72206104
:10018000206C697374206F6620636F6D6D616E649F
:1001900073005B62742D636D6440252E32783A25BE
:1001A0002E32785D24200065746865726E75740067
:1001B00069646C65006D61696E00FF000000004CB1
:1001C0000C00007561727430000000000500000032
:1001D00000006203506CCF6C3870307028707B6EFA
:1001E000E96E6C6C000000000000000000000000E0
:1001F00000000000000000000000000000000000FF
:1002000000000000000000000000000000000000EE
:10021000000000000000000000D30FAA0FF30EF54D
:100220000EF80FD30E53105D0F210FB50DCF10D266
:100230000D0311E30D570EED0D9310BC0E0000756C
:100240006172743100000000050100000000DE034F
:10025000506CCF6C3870307028707B6EE96E6C6CAF
:10026000000000000000000000000000000000008E
:10027000000000000000000000000000000000007E
:10028000000000000000000000000000000000006E
:100290000000000000C5137D149E13A41396147E65
:1002A00013F1142D14E813501280156F12B5158038
:1002B00012F6128A123515651300000000101600A0
:1002C000000000C116000000002D17000000009182
:1002D0001701000200030000000000000000000001
:1002E00000286E756C6C2900303132333435363766
:1002F00038396162636465660030313233343536D3
:1003000037383941424344454600202020202020F0
:10031000202020202020202020203030303030307D
:1003200030303030303030303030313233340042E1
:1003300054537461636B005F554152547772697412
:1003400065206572726F72210A005F5541525472C6
:10035000656164206572726F72210A006672616D58
:10036000696E67206572726F720A006275666665F3
:1003700072206F76657272756E206572726F720A86
:1003800000706172697479206572726F720A007010
:1003900061636B6574206F7574206F662073796E6E
:1003A0006320746F2042542075617274210A0072B8
:1003B0002B00307825580A0073656D610073656DF8
:1003C000612025703A2025640A00004C4544000F46
:1003D000014C6F67457674000A000000545F544575
:1003E000524D494E414C006274004C6F63616C2069
:1003F0004C4D5020737570706F7274656420666523
:100400006174757265733A20252E325820252E327C
:100410005820252E325820252E325820252E32588D
:1004200020252E325820252E325820252E32580ACB
:100430000062743A206572726F722075736167652D
:100440003A0A20627420616464720A206274206334
:100450006F6E7461626C650A2062742075617274DB
:100460006465627567203C303D6F66662C20313DC7
:100470006F6E3E0A20627420636874696D656F75E3
:1004800074203C68616E646C653E203C74696D65E7
:100490003E0A20627420636F6E203C696E712D6984
:1004A0006E6465783E207C2078783A78783A78785F
:1004B0003A78783A78783A78780A206274206469D1
:1004C00073636F6E203C68616E646C653E0A2062E7
:1004D0007420696E71756972790A00206274206EE9
:1004E000616D650A20627420636F640A2062742063
:1004F000726E616D650A20627420726F6C65203CBB
:1005000068616E646C653E0A20627420726F6C656F
:10051000736574203C68616E646C653E203C6D7947
:100520005F726F6C653A4D3D3020533D313E0A207D
:1005300062742066656174757265730A2062742046
:1005400076657273696F6E0A00252E32783A252E11
:1005500032783A252E32783A252E32783A252E32C4
:10056000783A252E3278004C6F63616C2062745F9C
:10057000616464723A20000A0044657669636573B9
:100580003A2025640A0044657669636520202020AE
:10059000202020202062745F6164647220636F6495
:1005A0002020202020202020525353490A005B2580
:1005B000645D3A2000203078252E386C7820256440
:1005C0000A004C6F63616C20484349207665727362
:1005D000696F6E20696E666F3A20255820252E348B
:1005E0005820255820252E345820252E34580A000E
:1005F00025750073657400256C75004552524F5285
:100600002077726974696E67206C6F63616C204338
:100610004F44210A004C6F63616C20434F442073A8
:100620006574210A004552524F52207772697469ED
:100630006E67206C6F63616C20434F443A20496CB5
:100640006C6567616C2076616C75652028256C751A
:10065000292E0A00676574004C6F63616C20434F5C
:10066000443A203078252E386C780A00636F643A5B
:10067000206572726F723A2075736167653A0A205D
:10068000636F6420736574203C76616C75653E0A07
:1006900020636F64206765740A004552524F5220F0
:1006A00077726974696E67206C6F63616C206E612C
:1006B0006D65210A004C6F63616C206E616D652071
:1006C000736574210A004552524F522061736B6961
:1006D0006E67206C6F63616C206E616D65210A002E
:1006E0004C6F63616C206E616D653A20272573271E
:1006F0000A006E616D653A206572726F723A2075FC
:10070000736167653A0A206E616D652073657420B8
:100710003C6E616D653E0A206E616D652067657493
:100720000A000A48646C204D68646C20416464725D
:100730002020202020202020202020202020537432
:1007400061746520526F6C65204D6F64650A0025E9
:1007500033640025203464200020253564200025E2
:10076000346400206163746976650020686F6C648E
:100770000020736E69666600207061726B002069EC
:100780006E76616C6964006D7920726F6C6520749F
:100790006F20636F6E20776974682068616E646C87
:1007A0006520256420697320004D41535445520A49
:1007B00000534C4156450A00257525750045525297
:1007C0004F5220726F6C65206368616E67653A20D6
:1007D0006572726F7220636F64653D256C640A00F8
:1007E000726F6C657365742068616E646C6520253A
:1007F000643A206D7920726F6C65206973200072F5
:100800006F6C657365743A206572726F723A207509
:10081000736167653A0A20726F6C65736574203C7A
:1008200068616E646C653E203C6D795F726F6C65CB
:100830003A4D3D3020533D313E0A00646973636F89
:100840006E3A206572726F723A206E6F20636F6E1F
:1008500020776974682068616E646C652025640A7D
:1008600000646973636F6E3A206572726F723A202A
:1008700063616E6E6F74206765742062745F61647B
:100880006472206F662068616E646C652025640A5E
:1008900000646973636F6E20636F6E6E6563746965
:1008A0006F6E20746F2000646973636F6E3A206509
:1008B00072726F723A2063616E6E6F742064697336
:1008C000636F6E6E65637420636F6E6E65637469CB
:1008D0006F6E20776974682068616E646C6520258E
:1008E000640A00646973636F6E6E65637465642186
:1008F0000A002532783A2532783A2532783A25327C
:10090000783A2532783A25327800636F6E3A20655E
:1009100072726F723A2064657620696E6465782021
:100920006F7574206F6620626F756E64730A006F56
:1009300070656E20636F6E20746F2000636F6E3A77
:10094000206572726F723A2028256C78290A006E31
:10095000657720636F6E212068616E646C65202569
:100960006C640A0068257500726E616D653A2065D9
:1009700072726F723A2064657620696E64657820C1
:100980006F7574206F6620626F756E64730A0067FE
:10099000657474696E6720726E616D65206F662084
:1009A00000726E616D653A206572726F723A206EE8
:1009B0006F20636F6E20776974682068616E646C65
:1009C000652025640A00726E616D653A2065727259
:1009D0006F723A20252E3278210A0072656D6F748D
:1009E00065206E616D653A2700270A00726E616DA1
:1009F000653A206572726F723A2075736167653A65
:100A00000A20726E616D652078783A78783A787845
:100A10003A78783A78783A78780A20726E616D651B
:100A2000203C696E712D696E6465783E0A20726E95
:100A3000616D6520683C68616E646C653E0A007398
:100A4000796E63005374617274696E672073796E96
:100A50006320696E717569727920666F72202564F2
:100A6000207365633A0A006173796E6300506C65A8
:100A70006173652063616C6C2066697273742027F2
:100A8000627420696E717569727920726573756C14
:100A90007427210A005374617274696E6720617350
:100AA000796E6320696E7175697279210A205573B8
:100AB00065206E6578742027627420696E7175698F
:100AC000727920636865636B2720616E642F6F7293
:100AD0002027627420696E7175697279207265735E
:100AE000756C74272E0A00636865636B00506C6533
:100AF0006173652063616C6C206669727374202772
:100B0000627420696E7175697279206173796E63A0
:100B100027210A00496E717569727920646F6E65CC
:100B2000210A00496E7175697279207374696C6C61
:100B30002072756E6E696E67210A00726573756C3E
:100B40007400696E71756972793A206572726F729C
:100B50003A2075736167653A0A20696E717569722A
:100B6000792073796E63205B74696D6520696E20EE
:100B70007365635D0A20696E7175697279206173AE
:100B8000796E63205B74696D6520696E207365639F
:100B90005D0A20696E717569727920726573756C72
:100BA000740A20696E717569727920636865636B78
:100BB0000A006368616E6765206469736320746905
:100BC0006D656F757420666F722068616E646C6508
:100BD0002025640A00636874696D656F75743A2036
:100BE0006572726F723D256C640A00636874696D8A
:100BF000656F7574206368616E676564210A0061C2
:100C000064647200636F6E7461626C65007561721A
:100C100074646562756700636874696D656F757487
:100C200000636F6E00646973636F6E00696E717547
:100C3000697279006E616D6500636F6400726E6148
:100C40006D6500726F6C6573657400726F6C650022
:100C500066656174757265730076657273696F6E2F
:100C6000006C656400626174007061747465726E1A
:100C70002575257525752575007061747465726E0E
:100C8000636C72006F6E2575006F6666257500686F
:100C9000622575257525750075736167653A0A20AB
:100CA0006C6564207061747465726E203C7370654D
:100CB00065643A312D31303E203C6475726174694F
:100CC0006F6E3E203C6E723A312D383E205B617271
:100CD000675D0A206C6564207061747465726E6370
:100CE0006C720A206C6564206F6E203C6E723A3024
:100CF0002D333E0A206C6564206F6666203C6E7260
:100D00003A302D333E0A206C6564206862203C70C6
:100D1000617573653E203C342D6269742070617486
:100D20007465726E3E203C6475726174696F6E3ECC
:100D30000A004261747465727920566F6C74616741
:100D4000653A2025642E2530326420560A0D006E47
:100D5000757400746872656164730074696D65729E
:100D6000730068656170006C6F67006C6F67207559
:100D7000736167653A0A0073686F77205B3C6E7237
:100D80005F6D7367733E205B3C636C6173733E20E1
:100D90005B3C6D61736B5D5D5D0A00676574205B34
:100DA0003C69645F6E657765723E205B3C6E725F86
:100DB0006D7367733E205B3C636C6173733E205BB5
:100DC0003C6D61736B3E5D5D5D5D0A00636C6561EA
:100DD000720A006C6F676D61736B203C636C6173AA
:100DE000733E205B3C6D61736B3E5D0A00766572FD
:100DF000626F73697479206F6E0A00766572626F34
:100E000073697479203C636C6173733E205B3C6D45
:100E100061736B3E5D0A00766572626F7369747907
:100E20002070617573650A00766572626F7369740C
:100E30007920726573756D650A00766572626F73ED
:100E4000697479206F66660A006F6E00766572625B
:100E50006F73697479206F6E210A006661696C6531
:100E6000643A206F74686572206C6F67206C6973D8
:100E700074656E6572207265676973746572656406
:100E8000210A006F666600766572626F7369747915
:100E9000206F6666210A0070617573650076657261
:100EA000626F73697479207061757365642E0A00CE
:100EB000726573756D6500766572626F73697479BA
:100EC00020726573756D65642E0A002564257800AF
:100ED0006572723A20696E76616C6964206C6F6726
:100EE00020636C617373210A006C6F6720636C610F
:100EF00073732025692C20766572626F736974792B
:100F0000206D61736B2073657420746F3A20252EF9
:100F100032580A0073686F770025752575257800AB
:100F200067657400257525752575257800636C65E2
:100F30006172006C6F676D61736B006C6F6720632B
:100F40006C6173732025692C2000206C6F676D61C4
:100F5000736B2073657420746F3A20252E32580A03
:100F600000766572626F7369747900253575202586
:100F700031306C752043252E32642C2025730000FF
:100F80000007110D11131119114552523A20005743
:100F9000524E3A2000494E463A20004442473A20F9
:100FA0000065627400636F6E736F6C653A206572E2
:100FB000726F723A2075736167653A0A20656274D0
:100FC00020636F6E736F6C65203C737472696E671B
:100FD0003E0A002065627420686F6C640A206562B6
:100FE0007420736E6966660A20656274207061728F
:100FF0006B0A20656274207363616E203C696E71B8
:10100000756972795F7363616E3E203C70616765DC
:101010005F7363616E3E0A206562742063706D20A9
:101020003C303D6F66662C20313D6F6E3E0A206578
:1010300062742072657365740A2065627420687733
:101040005F72657365740A2065627420636F6E73E6
:101050006F6C65203C737472696E673E0A0072653E
:10106000736574206E6F742066696E697368656459
:101070002E0A0025752575007363616E3A2065722E
:10108000726F723A2075736167653A0A2073636103
:101090006E203C696E7175697279207363616E3A76
:1010A00020303D6F66662C20313D6F6E3E203C70D7
:1010B000616765207363616E3A20303D6F66662C10
:1010C00020313D6F6E3E0A0025750063706D3A2039
:1010D0006572726F723A2075736167653A0A2063B0
:1010E000706D203C303D6F66662C20313D6F6E3E4A
:1010F0000A007061726B3A206572726F723A2075E5
:10110000736167653A0A207061726B203C68616E9A
:10111000646C653E203C696E74657276616C2D73FB
:101120006C6F74733E0A207061726B203C68616E54
:10113000646C653E0A007061726B3A206D6F646585
:10114000206368616E67653A2025642028696E74A3
:10115000657276616C202564290A004552524F520F
:10116000206D6F6465206368616E67652028657215
:10117000726F7220636F64653D256C64292E0A00CE
:10118000257525752575257500736E6966663A2087
:101190006572726F723A2075736167653A0A2073DF
:1011A0006E696666203C68616E646C653E203C69D1
:1011B0006E74657276616C3E203C617474656D700E
:1011C000743E203C74696D656F75743E0A20736EC1
:1011D000696666203C68616E646C653E0A00736EE9
:1011E0006966663A206D6F6465206368616E676545
:1011F0003A2025642028696E74657276616C20251A
:1012000064290A004552524F52206D6F6465206375
:1012100068616E67653A206572726F7220636F64F1
:10122000653D256C640A00686F6C643A206D6F64DC
:1012300065206368616E67653A2025642028696EC1
:1012400074657276616C202564290A00686F6C648D
:101250003A206572726F723A2075736167653A0A57
:1012600020686F6C64203C68616E646C653E203C55
:1012700074696D653E0A00686F6C6400736E696620
:1012800066007061726B0063706D007363616E0065
:1012900072657365740068775F7265736574006367
:1012A0006F6E736F6C65004641494C004F4B0053A5
:1012B00049474E414C4544005349474E414C4544F3
:1012C0000A0054524D0052554E0052445900534C9E
:1012D00050004014441448144C1443504D0008204E
:1012E00008000A00256300252E32783A252E327830
:1012F0003A252E32783A252E32783A252E32783A0F
:0C130000252E327800252E3278200000C7
:00000001FF
